 archba

 Timestamp is 5bb221b5 (Mon Oct  1 19:01:33 2018)

 Preferred load address is 0000000140000000

 Start         Length     Name                   Class
 0001:00000000 0001f860H .text$mn                CODE
 0001:0001f860 00000020H .text$mn$00             CODE
 0001:0001f880 00000430H .text$mn$21             CODE
 0001:0001fcb0 000099c8H .text$s                 CODE
 0002:00000000 000000c0H .idata$5                DATA
 0002:000000c0 00000010H .00cfg                  DATA
 0002:000000d0 000000b0H .gfids                  DATA
 0002:0000017c 00000000H .gfids$y                DATA
 0002:00000180 000006c0H .rdata                  DATA
 0002:00000840 000001b0H .rdata$zzzdbg           DATA
 0002:000009f0 000015b4H .xdata                  DATA
 0003:00000000 00000ae0H .data                   DATA
 0003:00000ae0 000002e8H .bss                    DATA
 0004:00000000 00000c9cH .pdata                  DATA
 0005:00000000 0000005cH INIT                    CODE
 0005:0000005c 0000003cH .idata$2                CODE
 0005:00000098 00000018H .idata$3                CODE
 0005:000000b0 000000c0H .idata$4                CODE
 0005:00000170 00000228H .idata$6                CODE
 0006:00000000 000000d0H .rsrc$01                DATA
 0006:000000d0 00001108H .rsrc$02                DATA

  Address         Publics by Value              Rva+Base               Lib:Object

 0000:00000000       __enclave_config           0000000000000000     <absolute>
 0000:00000000       ___safe_se_handler_table   0000000000000000     <absolute>
 0000:00000000       __guard_longjmp_table      0000000000000000     <absolute>
 0000:00000000       __dynamic_value_reloc_table 0000000000000000     <absolute>
 0000:00000000       __guard_longjmp_count      0000000000000000     <absolute>
 0000:00000000       ___safe_se_handler_count   0000000000000000     <absolute>
 0000:00000000       __hybrid_code_map_count    0000000000000000     <absolute>
 0000:00000000       __hybrid_auxiliary_iat     0000000000000000     <absolute>
 0000:00000000       __guard_iat_table          0000000000000000     <absolute>
 0000:00000000       __hybrid_code_map          0000000000000000     <absolute>
 0000:00000000       __guard_iat_count          0000000000000000     <absolute>
 0000:0000002b       __guard_fids_count         000000000000002b     <absolute>
 0000:00014500       __guard_flags              0000000000014500     <absolute>
 0000:00000000       __ImageBase                0000000140000000     <linker-defined>
 0001:00000000       DumpHandles                0000000140001000 f   rxdevice.obj
 0001:000003b0       DumpHandlesZeroPointer     00000001400013b0 f   rxdevice.obj
 0001:00000760       GetOutstandingIoCnt        0000000140001760 f   rxdevice.obj
 0001:00000770       NonMSIXInterruptHandler    0000000140001770 f   rxdevice.obj
 0001:00000b50       PMCDpcResponseHandler      0000000140001b50 f   rxdevice.obj
 0001:000012f0       PMCInterruptHandler        00000001400022f0 f   rxdevice.obj
 0001:000018f0       PMCPushMessageUnitQueueFib 00000001400028f0 f   rxdevice.obj
 0001:00001c10       RxAccessDeviceRegister     0000000140002c10 f   rxdevice.obj
 0001:00001db0       RxCheckAdapterHealth       0000000140002db0 f   rxdevice.obj
 0001:00001e20       RxCheckSyncCommandComplete 0000000140002e20 f   rxdevice.obj
 0001:00001f60       RxDpcInterruptHandler      0000000140002f60 f   rxdevice.obj
 0001:00001f60       _guard_check_icall_nop     0000000140002f60 f   BufferOverflowFastFailK:guard_support.obj
 0001:00001f70       RxGetIBW                   0000000140002f70 f   rxdevice.obj
 0001:00001fa0       RxGetOMRx0                 0000000140002fa0 f   rxdevice.obj
 0001:00001fd0       RxInterruptHandler         0000000140002fd0 f   rxdevice.obj
 0001:000022a0       RxMapMailBoxFirmwareBase   00000001400032a0 f   rxdevice.obj
 0001:00002390       RxNewCommProcessInterrupt  0000000140003390 f   rxdevice.obj
 0001:00002760       RxNotifyAdapter            0000000140003760 f   rxdevice.obj
 0001:000027e0       RxPullMessageUnitQueueCompletedFib 00000001400037e0 f   rxdevice.obj
 0001:00002980       RxPushMessageUnitQueueFib  0000000140003980 f   rxdevice.obj
 0001:00002a70       RxSendSynchCommand         0000000140003a70 f   rxdevice.obj
 0001:000036b0       RxStartAdapter             00000001400046b0 f   rxdevice.obj
 0001:00003d30       RxWaitForAdapterToBoot     0000000140004d30 f   rxdevice.obj
 0001:00003e20       RxWriteIBW                 0000000140004e20 f   rxdevice.obj
 0001:00003e50       RxWriteIDR                 0000000140004e50 f   rxdevice.obj
 0001:00003e80       RxWriteODR                 0000000140004e80 f   rxdevice.obj
 0001:00003ec0       RevCheckCompatibility      0000000140004ec0 f   revision.obj
 0001:00003f60       RevGetBuildNumber          0000000140004f60 f   revision.obj
 0001:00003f70       RevGetExternalRev          0000000140004f70 f   revision.obj
 0001:00003f80       CompareStrings             0000000140004f80 f   helpers.obj
 0001:00004000       GetDriverParameter         0000000140005000 f   helpers.obj
 0001:00004140       LongToAscii                0000000140005140 f   helpers.obj
 0001:000041f0       MatchRegistryString        00000001400051f0 f   helpers.obj
 0001:000042b0       ZeroStructure              00000001400052b0 f   helpers.obj
 0001:000042c0       NullTraceFunc              00000001400052c0 f i arcdebug.obj
 0001:000042d0       ArcPrintf                  00000001400052d0 f   arcdebug.obj
 0001:00004880       ProcessCompleteSrbToHost   0000000140005880 f   arcdebug.obj
 0001:00004890       RealSprintf                0000000140005890 f   arcdebug.obj
 0001:00004d40       CheckingFWAfterPowerStateChange 0000000140005d40 f   timer.obj
 0001:00005130       MainTimeThread             0000000140006130 f   timer.obj
 0001:00005de0       RequestTimer               0000000140006de0 f   timer.obj
 0001:00005eb0       Reset_IOP_CompletionTimer  0000000140006eb0 f   timer.obj
 0001:00006380       StopTimer                  0000000140007380 f   timer.obj
 0001:00006420       UpdateThorHBAMappingTable  0000000140007420 f   timer.obj
 0001:00006700       VMCloseAllCompletionTimer  0000000140007700 f   timer.obj
 0001:00006950       AllocateConsumerProducerCommArea 0000000140007950 f   arcinit.obj
 0001:00006cd0       AllocateMessageUnitQueueCommArea 0000000140007cd0 f   arcinit.obj
 0001:00007280       ArcLogEventString          0000000140008280 f   arcinit.obj
 0001:00007300       AtomicINTXReleaseSlot      0000000140008300 f   arcinit.obj
 0001:00007320       CheckMSIxPossibility       0000000140008320 f   arcinit.obj
 0001:00007530       CleanHostSideRRQ           0000000140008530 f   arcinit.obj
 0001:00007760       ConfigureContainersRuntime 0000000140008760 f   arcinit.obj
 0001:00009090       DecToHex                   000000014000a090 f   arcinit.obj
 0001:000090f0       DriverEntry                000000014000a0f0 f   arcinit.obj
 0001:00009310       DumpFibsSentToFW60SecondsBefore 000000014000a310 f   arcinit.obj
 0001:000095f0       DynamicallyThrottleLunQueueDepth 000000014000a5f0 f   arcinit.obj
 0001:00009820       EventTracingCleanup        000000014000a820 f   arcinit.obj
 0001:00009890       FindAdapter                000000014000a890 f   arcinit.obj
 0001:0000c2e0       GetElapsedSeconds          000000014000d2e0 f   arcinit.obj
 0001:0000c370       GetFreeSlot                000000014000d370 f   arcinit.obj
 0001:0000c3a0       GetThorHbaPhyDevInfo       000000014000d3a0 f   arcinit.obj
 0001:0000c8f0       HWSoftReset                000000014000d8f0 f   arcinit.obj
 0001:0000ca50       HandleAdapterCommitConfig  000000014000da50 f   arcinit.obj
 0001:0000cb20       HandleAdapterConfigIssues  000000014000db20 f   arcinit.obj
 0001:0000ccf0       HandleAdapterGetConfig     000000014000dcf0 f   arcinit.obj
 0001:0000ce00       HwInitializeAdapter        000000014000de00 f   arcinit.obj
 0001:0000d250       INTXGetFreeSlot            000000014000e250 f   arcinit.obj
 0001:0000d270       IOPReset                   000000014000e270 f   arcinit.obj
 0001:0000d7c0       InitializeConsumerProducerCommRegion 000000014000e7c0 f   arcinit.obj
 0001:0000da50       InitializeDPCs             000000014000ea50 f   arcinit.obj
 0001:0000e190       IsAdapterReadyForConfigCommand 000000014000f190 f   arcinit.obj
 0001:0000e2c0       LogSystemEvent             000000014000f2c0 f   arcinit.obj
 0001:0000e3a0       MapDeviceBase              000000014000f3a0 f   arcinit.obj
 0001:0000e930       ReleaseSlot                000000014000f930 f   arcinit.obj
 0001:0000e960       ResetAdapter               000000014000f960 f   arcinit.obj
 0001:0000f060       ReturnOutstandingFibOnTargetDevice 0000000140010060 f   arcinit.obj
 0001:0000f210       ReturningLocalOutstandingRequestsToOS 0000000140010210 f   arcinit.obj
 0001:0000f500       ReturningOutstandingSentToFWBeforeIOPResetToOS 0000000140010500 f   arcinit.obj
 0001:0000f6b0       SA4ACI2Interface           00000001400106b0 f   arcinit.obj
 0001:0000f840       SA4StatusBatching          0000000140010840 f   arcinit.obj
 0001:0000f9d0       SMCrashDumpModeInitAdapter 00000001400109d0 f   arcinit.obj
 0001:0000fc80       SMNormalModeInitAdapter    0000000140010c80 f   arcinit.obj
 0001:00010160       SendEvent2OS               0000000140011160 f   arcinit.obj
 0001:00010af0       SendEvent2OSChild          0000000140011af0 f   arcinit.obj
 0001:00010f80       SendEvent2OSDelayed        0000000140011f80 f   arcinit.obj
 0001:000116d0       SendInitStructure          00000001400126d0 f   arcinit.obj
 0001:00011aa0       SendWellnessCmnd           0000000140012aa0 f   arcinit.obj
 0001:00011ca0       SetArcsasFwTime            0000000140012ca0 f   arcinit.obj
 0001:00011d80       SetFwTime                  0000000140012d80 f   arcinit.obj
 0001:00012210       SetPciSlotNumber           0000000140013210 f   arcinit.obj
 0001:000122f0       StorWmiTraceMessage        00000001400132f0 f i arcinit.obj
 0001:00012350       WppTraceCallback           0000000140013350 f   arcinit.obj
 0001:000125d0       CompleteQueuedRequest      00000001400135d0 f   cmddelivery.obj
 0001:000126d0       DequeueCertainLD           00000001400136d0 f   cmddelivery.obj
 0001:00012780       DequeueRawIoReadWriteRequest 0000000140013780 f   cmddelivery.obj
 0001:000128a0       HandleInterrupt            00000001400138a0 f   cmddelivery.obj
 0001:000128c0       HandleMSIXInterrupt        00000001400138c0 f   cmddelivery.obj
 0001:000129a0       PollSmartHBAFIBCompletion  00000001400139a0 f   cmddelivery.obj
 0001:00012d40       PostProcessScsiCommand     0000000140013d40 f   cmddelivery.obj
 0001:00013090       ProcessContainerInquiry    0000000140014090 f   cmddelivery.obj
 0001:00013640       ProcessScsiCommand         0000000140014640 f   cmddelivery.obj
 0001:000142a0       QueuePrintf                00000001400152a0 f   cmddelivery.obj
 0001:00014360       QueueRawIoReadWriteRequest 0000000140015360 f   cmddelivery.obj
 0001:00014650       SaveNFHandle               0000000140015650 f   cmddelivery.obj
 0001:00014690       SendFib                    0000000140015690 f   cmddelivery.obj
 0001:00014cd0       SendRawIoFib               0000000140015cd0 f   cmddelivery.obj
 0001:00014eb0       SendSynchFib               0000000140015eb0 f   cmddelivery.obj
 0001:000150b0       StartIo                    00000001400160b0 f   cmddelivery.obj
 0001:00015b10       AdapterControl             0000000140016b10 f   cmdproc.obj
 0001:00016240       BuildHBAFib                0000000140017240 f   cmdproc.obj
 0001:00016730       BuildHBAIoctlFib           0000000140017730 f   cmdproc.obj
 0001:000169e0       BuildIo                    00000001400179e0 f   cmdproc.obj
 0001:000175c0       BuildRawIo2ScatterGather   00000001400185c0 f   cmdproc.obj
 0001:000177a0       BuildRawIo2ScatterGather4HBAIoctl 00000001400187a0 f   cmdproc.obj
 0001:00017970       BuildRawIoFib              0000000140018970 f   cmdproc.obj
 0001:00017cd0       BuildRawIoScatterGather    0000000140018cd0 f   cmdproc.obj
 0001:00017ec0       BuildReadWriteFib          0000000140018ec0 f   cmdproc.obj
 0001:00018290       BuildScatterGather         0000000140019290 f   cmdproc.obj
 0001:00018340       BuildScatterGather64       0000000140019340 f   cmdproc.obj
 0001:00018400       BuildSrbFib                0000000140019400 f   cmdproc.obj
 0001:000186a0       ConvertRawIo2ScatterGather 00000001400196a0 f   cmdproc.obj
 0001:000187e0       InitializeFib              00000001400197e0 f   cmdproc.obj
 0001:00018810       PrepareBMIC15              0000000140019810 f   cmdproc.obj
 0001:00018a50       BuildRawScatterGather      0000000140019a50 f   ioctl.obj
 0001:00018b00       BuildRawScatterGather64    0000000140019b00 f   ioctl.obj
 0001:00018bb0       CSMIGetRAIDConfig          0000000140019bb0 f   ioctl.obj
 0001:00018e20       CSMIGetRAIDInfo            0000000140019e20 f   ioctl.obj
 0001:000192e0       CSMISTPPassThru            000000014001a2e0 f   ioctl.obj
 0001:00019580       HandleCSMI                 000000014001a580 f   ioctl.obj
 0001:00019b80       ProcessIoctl               000000014001ab80 f   ioctl.obj
 0001:0001c500       AdapterIsAlive             000000014001d500 f   comm.obj
 0001:0001c540       CompleteAllSortingQueue    000000014001d540 f   comm.obj
 0001:0001c650       CompleteBufferedRequest    000000014001d650 f   comm.obj
 0001:0001c710       DeQueueSortingQueue        000000014001d710 f   comm.obj
 0001:0001c8a0       DpcDequeueRawIoReadWriteRequest 000000014001d8a0 f   comm.obj
 0001:0001c910       FreeConsumerProducerAif    000000014001d910 f   comm.obj
 0001:0001ca60       GetConsumerProducerCompletedFib 000000014001da60 f   comm.obj
 0001:0001caf0       GetMessageUnitQueueCompletedFib 000000014001daf0 f   comm.obj
 0001:0001cb10       ProcessAif                 000000014001db10 f   comm.obj
 0001:0001d440       ProcessHbaErrors           000000014001e440 f   comm.obj
 0001:0001da50       ProcessNormalFib           000000014001ea50 f   comm.obj
 0001:0001e550       QueueEvent                 000000014001f550 f   comm.obj
 0001:0001e5f0       SendConsumerProducerFib    000000014001f5f0 f   comm.obj
 0001:0001e6f0       SendMessageUnitQueueFib    000000014001f6f0 f   comm.obj
 0001:0001e760       ServiceHostCommandNormalQueue 000000014001f760 f   comm.obj
 0001:0001e850       ServiceHostResponseNormalQueue 000000014001f850 f   comm.obj
 0001:0001ec70       ServiceInternalAifQueue    000000014001fc70 f   comm.obj
 0001:0001ed40       SubDeQueueSortingQueue     000000014001fd40 f   comm.obj
 0001:0001ee40       HwScsiWmiExecuteMethod     000000014001fe40 f   wmi.obj
 0001:0001eee0       HwScsiWmiQueryDataBlock    000000014001fee0 f   wmi.obj
 0001:0001eee0       HwScsiWmiFunctionControl   000000014001fee0 f   wmi.obj
 0001:0001ef00       HwScsiWmiQueryReginfo      000000014001ff00 f   wmi.obj
 0001:0001ef10       HwScsiWmiSetDataBlock      000000014001ff10 f   wmi.obj
 0001:0001ef10       HwScsiWmiSetDataItem       000000014001ff10 f   wmi.obj
 0001:0001ef20       InitializeWmiInterface     000000014001ff20 f   wmi.obj
 0001:0001f030       ProcessWmi                 0000000140020030 f   wmi.obj
 0001:0001f0c0       __security_check_cookie    00000001400200c0 f   BufferOverflowFastFailK:amdsecgs.obj
 0001:0001f0e0       __report_gsfailure         00000001400200e0 f   BufferOverflowFastFailK:gs_report.obj
 0001:0001f0e8       __report_rangecheckfailure 00000001400200e8 f   BufferOverflowFastFailK:gs_report.obj
 0001:0001f0f0       __GSHandlerCheck           00000001400200f0 f   ntoskrnl:gshandler.obj
 0001:0001f110       __GSHandlerCheckCommon     0000000140020110 f   ntoskrnl:gshandler.obj
 0001:0001f170       ExSystemTimeToLocalTime    0000000140020170 f   ntoskrnl:ntoskrnl.exe
 0001:0001f176       RtlTimeToTimeFields        0000000140020176 f   ntoskrnl:ntoskrnl.exe
 0001:0001f17c       KeQueryPerformanceCounter  000000014002017c f   hal:HAL.dll
 0001:0001f184       ScsiPortWmiDispatchFunction 0000000140020184 f   scsiwmi:wmilib.obj
 0001:0001f224       ScsiPortWmiPostProcess     0000000140020224 f   scsiwmi:wmilib.obj
 0001:0001f260       ScsiWmipFindGuid           0000000140020260 f   scsiwmi:wmilib.obj
 0001:0001f2c0       ScsiWmipPostProcess        00000001400202c0 f   scsiwmi:wmilib.obj
 0001:0001f410       ScsiWmipProcessRequest     0000000140020410 f   scsiwmi:wmilib.obj
 0001:0001f870       _guard_dispatch_icall_nop  0000000140020870 f   BufferOverflowFastFailK:guard_dispatch.obj
 0001:0001f880       memmove                    0000000140020880 f   ntoskrnl:memcpy.obj
 0001:0001f880       memcpy                     0000000140020880 f   ntoskrnl:memcpy.obj
 0001:0001fbc0       memset                     0000000140020bc0 f   ntoskrnl:memset.obj
 0001:0001fcb0       ??_C@_0CJ@KAGJNHLI@OMR?5value?5in?5Check?5Adapter?5Healt@FNODOBFM@ 0000000140020cb0     rxdevice.obj
 0001:0001fce0       ??_C@_0DE@IHDJGLJF@This?5should?5not?5happen?4?5We?5only?5@FNODOBFM@ 0000000140020ce0     rxdevice.obj
 0001:0001fd20       ??_C@_0CP@PEAJGKJE@?$CK?5NonMSIXInterruptHandle?3?5pFibCo@FNODOBFM@ 0000000140020d20     rxdevice.obj
 0001:0001fd50       ??_C@_0EM@CCDNION@?$CK?5Start?5a?5timer?5to?5update?5contai@FNODOBFM@ 0000000140020d50     rxdevice.obj
 0001:0001fda0       ??_C@_0DL@ELHJEKAJ@?$CK?57?124?3?5pFibContext?$DNNULL?5?$CB?$CBline?5@FNODOBFM@ 0000000140020da0     rxdevice.obj
 0001:0001fde0       ??_C@_0DA@IEDLNFHE@?$CK?55?124?3?5?9VectorIndex?9?5?$CB?$CBline?5?$CFd?5@FNODOBFM@ 0000000140020de0     rxdevice.obj
 0001:0001fe10       ??_C@_0CN@FKDOCGDJ@?$CK?55?124?3?5OutStanding?5IO?5?$CB?$CBline?5?$CFd@FNODOBFM@ 0000000140020e10     rxdevice.obj
 0001:0001fe40       ??_C@_0CD@PAEIGALF@?$CK?57?124?3?5?$CB?$CBline?5?$CFd?5?$CIhandle?5?9?51?$CJ?5?$CF@FNODOBFM@ 0000000140020e40     rxdevice.obj
 0001:0001fe70       ??_C@_0ED@DAJFCMJP@?$CK?5Start?5a?5timer?5to?5update?5Contai@FNODOBFM@ 0000000140020e70     rxdevice.obj
 0001:0001fec0       ??_C@_0DK@JKKKPJCO@Dumping?5Normal?5Fib?5handles?0?5?5pDe@FNODOBFM@ 0000000140020ec0     rxdevice.obj
 0001:0001ff00       ??_C@_0DG@FEIEMBNE@?$CFd?3?5?$CFd?5?$CFd?5?$CFd?5?$CFd?5?$CFd?5?$CFd?5?$CFd?5?$CFd?5?$CFd?5?$CF@FNODOBFM@ 0000000140020f00     rxdevice.obj
 0001:0001ff40       ??_C@_0GP@CPJOGFCD@Dumping?5Free?5handle?5list?0?5?5pDevi@FNODOBFM@ 0000000140020f40     rxdevice.obj
 0001:0001ffb0       ??_C@_0DN@IDNOKJK@ZP?5Dumping?5Normal?5Fib?5handles?0?5?5@FNODOBFM@ 0000000140020fb0     rxdevice.obj
 0001:0001fff0       ??_C@_0DJ@BENIEDOK@ZP?5?$CFd?3?5?$CFd?5?$CFd?5?$CFd?5?$CFd?5?$CFd?5?$CFd?5?$CFd?5?$CFd?5?$CF@FNODOBFM@ 0000000140020ff0     rxdevice.obj
 0001:00020030       ??_C@_0HC@OLAIGIPB@ZP?5Dumping?5Free?5handle?5list?0?5?5pD@FNODOBFM@ 0000000140021030     rxdevice.obj
 0001:000200b0       ??_C@_0CG@KADALDIK@?$CK?5?$CFd?5call?5of?5CheckForDupHandles?5@FNODOBFM@ 00000001400210b0     rxdevice.obj
 0001:000200e0       ??_C@_0EK@CPNBBJGG@?$CK?5duplicated?5handle?5found?5?$CFd?4?5?$CFd@FNODOBFM@ 00000001400210e0     rxdevice.obj
 0001:00020130       ??_C@_0BP@BKKLPPMO@pFibContext?$DNNULL?5?$CB?$CB?5Handle?5?$CFd?6?$AA@FNODOBFM@ 0000000140021130     rxdevice.obj
 0001:00020150       ??_C@_0EI@DKKBIMEF@?$CK?5Start?5a?5timer?5to?5update?5contai@FNODOBFM@ 0000000140021150     rxdevice.obj
 0001:000201a0       ??_C@_0FE@JLKFMCPA@?$CK?5PMCPushMessageUnitQueueFib?3?5Cm@FNODOBFM@ 00000001400211a0     rxdevice.obj
 0001:00020200       ??_C@_0FE@JICOMBJP@?$CK?5PMCPushMessageUnitQueueFib?3?5Cm@FNODOBFM@ 0000000140021200     rxdevice.obj
 0001:00020260       ??_C@_0HN@JEPKAECC@?$CK?5RxSendSynchCommand?3?5Thor?5AIF?5e@FNODOBFM@ 0000000140021260     rxdevice.obj
 0001:000202e0       ??_C@_0EC@LAPIEKPJ@?$CK?5RxSendSynchCommand?3?5mailbox?$FL0?$FN@FNODOBFM@ 00000001400212e0     rxdevice.obj
 0001:00020330       ??_C@_0DJ@GJNDHOED@?$CK?5RxSendSynchCommand?3?5mailbox?$FL0?$FN@FNODOBFM@ 0000000140021330     rxdevice.obj
 0001:00020370       ??_C@_0HK@NJDHDGMI@?$CK?5RxSendSynchCommand?3?5There?5is?5a@FNODOBFM@ 0000000140021370     rxdevice.obj
 0001:000203f0       ??_C@_0HB@PLCHFMAA@?$CK?5RxSendSynchCommand?3?5synch?5cmd?3@FNODOBFM@ 00000001400213f0     rxdevice.obj
 0001:00020470       ??_C@_0FD@ECFFGBJE@?5RxSendSynchCommand?3?5FW?5doing?5IO@FNODOBFM@ 0000000140021470     rxdevice.obj
 0001:000204d0       ??_C@_0FE@DOFCONDK@?$CK?5RxSendSynchCommand?3?5wait?5for?5F@FNODOBFM@ 00000001400214d0     rxdevice.obj
 0001:00020530       ??_C@_0GF@LFEFAJKJ@?5RxSendSynchCommand?5?$CIcrash?5dump?5@FNODOBFM@ 0000000140021530     rxdevice.obj
 0001:000205a0       ??_C@_0GF@CDCMENMG@?$CK?5RxSendSynchCommand?5?$CIcrash?5dump@FNODOBFM@ 00000001400215a0     rxdevice.obj
 0001:00020610       ??_C@_0EL@HOIBIGPI@?$CK?5RxSendSynchCommand?3?5Got?5respon@FNODOBFM@ 0000000140021610     rxdevice.obj
 0001:00020660       ??_C@_0EJ@DGPABBLG@?$CK?5RxSendSynchCommand?3?5Should?5NOT@FNODOBFM@ 0000000140021660     rxdevice.obj
 0001:000206b0       ??_C@_0FA@HKIBFKMH@?$CK?5RxSendSynchCommand?3?5Still?5NO?5r@FNODOBFM@ 00000001400216b0     rxdevice.obj
 0001:00020700       ??_C@_0KI@HMCHOJIN@?5RxSendSynchCommand?$FLMSIX?5mode?$FN?5f@FNODOBFM@ 0000000140021700     rxdevice.obj
 0001:000207b0       ??_C@_0JP@JKCHEOCJ@?5RxSendSynchCommand?$FLMSIX?5mode?$FN?3?5@FNODOBFM@ 00000001400217b0     rxdevice.obj
 0001:00020850       ??_C@_0CN@BCCBJMEA@?5RxSendSynchCommand?5Failed?5?$CFd?0wa@FNODOBFM@ 0000000140021850     rxdevice.obj
 0001:00020880       ??_C@_0DB@JEAHJGPL@?$CK?5pDeviceExtension?9?$DOMaxMSIXVecto@FNODOBFM@ 0000000140021880     rxdevice.obj
 0001:000208c0       ??_C@_0CB@JPABDNKH@?$CK?5Begins?5StatusBatching?0?5Yeaaa?$CB?6@FNODOBFM@ 00000001400218c0     rxdevice.obj
 0001:000208f0       ??_C@_0CF@BPKEMKA@?$CK?5ACI2?5Command?5Delivery?5is?5enabl@FNODOBFM@ 00000001400218f0     rxdevice.obj
 0001:00020920       ??_C@_1DK@JBHFOPMP@?$AAA?$AAd?$AAa?$AAp?$AAt?$AAe?$AAr?$AA?5?$AAC?$AAo?$AAn?$AAf?$AAi?$AAg?$AAu?$AAr?$AAa?$AAt?$AAi?$AAo?$AAn?$AA?5?$AAf?$AAa?$AAi?$AAl?$AAe?$AAd?$AA?$AA@FNODOBFM@ 0000000140021920     rxdevice.obj
 0001:00020960       ??_C@_02DKCKIIND@?$CFs?$AA@FNODOBFM@ 0000000140021960     arcdebug.obj
 0001:00020970       ??_C@_06NBLAGFFP@Archba?$AA@FNODOBFM@ 0000000140021970     arcdebug.obj
 0001:00020980       ??_C@_0BC@JKBDDNDF@DelayNotification?$AA@FNODOBFM@ 0000000140021980     timer.obj
 0001:000209a0       ??_C@_0CK@BKKGBKDP@?$CK?5Scan?5Notification?5sent?5in?5?$CFs?5?$CI@FNODOBFM@ 00000001400219a0     timer.obj
 0001:000209d0       ??_C@_0GB@FAGGLJPH@?$CK?5First?58?5HBA?5devices?3?5?$CI0x?$CFx?0?$CFd?$CJ@FNODOBFM@ 00000001400219d0     timer.obj
 0001:00020a40       ??_C@_0FN@EKAEFPGA@?$CK?5HBA?5mapping?5table?5updated?0?5tim@FNODOBFM@ 0000000140021a40     timer.obj
 0001:00020aa0       ??_C@_0GF@PMGNJLIM@?$CK?5Start?5a?5timer?5to?5update?5Contai@FNODOBFM@ 0000000140021aa0     timer.obj
 0001:00020b10       ??_C@_0CK@JLKEFPAM@entering?5CheckingFWAfterPowerSta@FNODOBFM@ 0000000140021b10     timer.obj
 0001:00020b40       ??_C@_0GN@GHJFFNOA@?$CK?5set?5timer?5AGAIN?5in?5CheckingFWA@FNODOBFM@ 0000000140021b40     timer.obj
 0001:00020bb0       ??_C@_0FK@MIIMDOAD@?$CK?5set?5timer?5AGAIN?5in?5CheckingFWA@FNODOBFM@ 0000000140021bb0     timer.obj
 0001:00020c10       ??_C@_0GB@EDFGCDFC@?$CK?5set?5timer?5AGAIN?5in?5CheckingFWA@FNODOBFM@ 0000000140021c10     timer.obj
 0001:00020c80       ??_C@_0N@CGGCEMAH@7?45?40?457001?$AA?$AA@FNODOBFM@ 0000000140021c80     timer.obj
 0001:00020c90       ??_C@_0DO@GCDGNMH@?$CK?5FW?5is?5back?5from?5S3?1S4?4?5StorPor@FNODOBFM@ 0000000140021c90     timer.obj
 0001:00020cd0       ??_C@_0DM@JABFAEPO@?$CK?5?9?5Reset?5AIFSrb?5to?5NULL?5when?5ba@FNODOBFM@ 0000000140021cd0     timer.obj
 0001:00020d10       ??_C@_0DN@ELHOMNDM@?$CK?5leaving?5CheckingFWAfterPowerSt@FNODOBFM@ 0000000140021d10     timer.obj
 0001:00020d50       ??_C@_0DO@OBELKDEH@?$CK?5set?5timer?5AGAIN?5to?5check?5the?5F@FNODOBFM@ 0000000140021d50     timer.obj
 0001:00020d90       ??_C@_0CI@JPJEKICG@DPC?9Timeout?5may?5happen?5in?5ResetA@FNODOBFM@ 0000000140021d90     timer.obj
 0001:00020dc0       ??_C@_0DH@JNGKJDAE@One?5kidnapped?5FIB?5released?$CB?5FIB_@FNODOBFM@ 0000000140021dc0     timer.obj
 0001:00020e00       ??_C@_0EJ@PCDGPKJP@?$CK?5Driver?5was?5not?5able?5to?5send?5?$CFd@FNODOBFM@ 0000000140021e00     timer.obj
 0001:00020e50       ??_C@_0DM@PNDEAHOI@?$CK?5Send?5BusChangeDetected?5to?5OS?5i@FNODOBFM@ 0000000140021e50     timer.obj
 0001:00020e90       ??_C@_0EH@FCLGCKBJ@?$CK?5Start?5a?5timer?5to?5update?5HBA?5de@FNODOBFM@ 0000000140021e90     timer.obj
 0001:00020ee0       ??_C@_0GE@IFJDDHGE@?$CK?5Start?5a?5timer?5to?5update?5Contai@FNODOBFM@ 0000000140021ee0     timer.obj
 0001:00020f50       ??_C@_0DC@ODEFHEA@?$CK?5ConfigureContainersTimer?3?5Cont@FNODOBFM@ 0000000140021f50     timer.obj
 0001:00020f90       ??_C@_0DL@DODBJONE@?$CK?5SynchCommandCompletionTimer?3?5S@FNODOBFM@ 0000000140021f90     timer.obj
 0001:00020fd0       ??_C@_0EO@CBNEAKKI@?$CK?5VMCloseAllCompletionTimer?3?5sen@FNODOBFM@ 0000000140021fd0     timer.obj
 0001:00021020       ??_C@_0FI@MJCPBEAD@?$CK?5VMCloseAllCompletionTimer?3?5wai@FNODOBFM@ 0000000140022020     timer.obj
 0001:00021080       ??_C@_0DO@ELMMCKMD@?$CK?5VMCloseAllCompletionTimer?3?5SRB@FNODOBFM@ 0000000140022080     timer.obj
 0001:000210c0       ??_C@_0EH@BGEEAOIJ@?$CK?5VMCloseAllCompletionTimer?3?5Sho@FNODOBFM@ 00000001400220c0     timer.obj
 0001:00021110       ??_C@_0EF@HLMPMNBN@?$CK?5VMCloseAllCompletionTimer?3?5Syn@FNODOBFM@ 0000000140022110     timer.obj
 0001:00021160       ??_C@_0DH@IBACIAED@?$CK?5SynchFibCompletionTimer?3?5SyncF@FNODOBFM@ 0000000140022160     timer.obj
 0001:000211a0       ??_C@_0DP@OKLOLMOG@?5IBW_SWR?5register?5value?50?0?5reset@FNODOBFM@ 00000001400221a0     timer.obj
 0001:000211e0       ??_C@_0CK@IHFMNBPG@?$CK?5IOP?5Reset?5TSR?3?5State?5Machine?5s@FNODOBFM@ 00000001400221e0     timer.obj
 0001:00021210       ??_C@_0DH@KAAGAFOD@?$CK?5leaving?5Reset_IOP_CompletionTi@FNODOBFM@ 0000000140022210     timer.obj
 0001:00021250       ??_C@_0CD@MKPFBJDC@leaving?5Reset_IOP_CompletionTime@FNODOBFM@ 0000000140022250     timer.obj
 0001:00021280       ??_C@_0DL@DOEFCINE@?$CK?5HW?5SOFT?5RESET?5done?4?5StorPort?5m@FNODOBFM@ 0000000140022280     timer.obj
 0001:000212c0       ??_C@_0EA@DAIPACKH@?$CK?5RESET?5IOP?5done?5?$CFd?5times?4?5StorP@FNODOBFM@ 00000001400222c0     timer.obj
 0001:00021300       ??_C@_0CJ@HBOEHNNB@Kernel?5Panic?5BlinkLed?5Code?5?$CFx?0?5l@FNODOBFM@ 0000000140022300     timer.obj
 0001:00021330       ??_C@_0CK@CJGFOJPA@IOP_HWSOFT_RESET?3?5FW?5status?5?$CFx?0?5@FNODOBFM@ 0000000140022330     timer.obj
 0001:00021360       ??_C@_0BP@HJBLFCEF@?$CK?5PCIE?5reset?5issued?0?5line?5?$CD?$CFd?6?$AA@FNODOBFM@ 0000000140022360     timer.obj
 0001:00021380       ??_C@_0DE@KOMJIKJE@?$CK?5set?5timer?5AGAIN?5to?5check?5the?5F@FNODOBFM@ 0000000140022380     timer.obj
 0001:000213c0       ??_C@_0EF@BBNOBECH@?$CK?5set?5timer?5AGAIN?5to?5check?5the?5F@FNODOBFM@ 00000001400223c0     timer.obj
 0001:00021410       ??_C@_0EC@MICIKMJM@?$CK?5set?5timer?5AGAIN?5to?5check?5the?5F@FNODOBFM@ 0000000140022410     timer.obj
 0001:00021460       ??_C@_0DI@CMFOGNCK@?$CK?5RequestAif?3?5do?5not?5handle?5AIF?5@FNODOBFM@ 0000000140022460     timer.obj
 0001:000214a0       ??_C@_0BJ@HIBCALL@ProcessAgeOfSortingQueue?$AA@FNODOBFM@ 00000001400224a0     timer.obj
 0001:000214c0       ??_C@_0DA@GEMOEFPE@Dequeue?5Sorting?5Queue?5failed?5in?5@FNODOBFM@ 00000001400224c0     timer.obj
 0001:000214f0       ??_C@_0ID@HFHPGANL@Dequeue?5Sorting?5Queue?5failed?5whe@FNODOBFM@ 00000001400224f0     timer.obj
 0001:00021580       ??_C@_0CL@MJMGCLDD@entering?5AllocateConsumerProduce@FNODOBFM@ 0000000140022580     arcinit.obj
 0001:000215b0       ??_C@_0DK@IJIOFPFH@leaving?5AllocateConsumerProducer@FNODOBFM@ 00000001400225b0     arcinit.obj
 0001:000215f0       ??_C@_0CI@FFOEPFMJ@?$CK?5ConsumerProducerCommArea?0?5VAdd@FNODOBFM@ 00000001400225f0     arcinit.obj
 0001:00021620       ??_C@_0CN@MBHLABKL@?$CK?5Adapter?5got?5an?5invalid?5host?5me@FNODOBFM@ 0000000140022620     arcinit.obj
 0001:00021650       ??_C@_0DJ@JGKEIEFI@leaving?5AllocateConsumerProducer@FNODOBFM@ 0000000140022650     arcinit.obj
 0001:00021690       ??_C@_0CL@KCDMGIOM@entering?5AllocateMessageUnitQueu@FNODOBFM@ 0000000140022690     arcinit.obj
 0001:000216c0       ??_C@_0FP@JFBPKCDF@?$CK?5AllocateMessageUnitQueueCommAr@FNODOBFM@ 00000001400226c0     arcinit.obj
 0001:00021720       ??_C@_0DM@JMMHKBOC@?$CK?5AllocateMessageUnitQueueCommAr@FNODOBFM@ 0000000140022720     arcinit.obj
 0001:00021760       ??_C@_0DK@BKFHOPDI@leaving?5AllocateMessageUnitQueue@FNODOBFM@ 0000000140022760     arcinit.obj
 0001:000217a0       ??_C@_0DA@ICFHAOHF@?$CK?5AllocateMessageUnitQueueCommAr@FNODOBFM@ 00000001400227a0     arcinit.obj
 0001:000217d0       ??_C@_0FB@FDJPGKAF@?$CK?5StorPortAllocateContiguousMemo@FNODOBFM@ 00000001400227d0     arcinit.obj
 0001:00021830       ??_C@_0FB@MMEFOJJL@?$CK?5StorPortAllocateContiguousMemo@FNODOBFM@ 0000000140022830     arcinit.obj
 0001:00021890       ??_C@_0BJ@OICKMJHC@?$CK?5pBuf1?$DN0x?$CFp?0pBuf2?$DN0x?$CFp?6?$AA@FNODOBFM@ 0000000140022890     arcinit.obj
 0001:000218b0       ??_C@_0BO@DPONBFMO@?$CK?5MemoryPhysicalAddress?$DN0x?$CFp?6?$AA@FNODOBFM@ 00000001400228b0     arcinit.obj
 0001:000218d0       ??_C@_0EL@ELLGMDMB@?$CK?5Allocate?5big?5IOCTL?5buffer?5succ@FNODOBFM@ 00000001400228d0     arcinit.obj
 0001:00021920       ??_C@_0DJ@EGOLHGNF@leaving?5AllocateMessageUnitQueue@FNODOBFM@ 0000000140022920     arcinit.obj
 0001:00021960       ??_C@_0CF@DNFJFJLG@entering?5ConfigureContainersRunt@FNODOBFM@ 0000000140022960     arcinit.obj
 0001:00021990       ??_C@_0EJ@GFICDCBB@?$CK?5ConfigureContainersRuntime?3?5Re@FNODOBFM@ 0000000140022990     arcinit.obj
 0001:000219e0       ??_C@_0EF@KJEEMCEN@?$CK?5ConfigureContainersRuntime?3?5Ge@FNODOBFM@ 00000001400229e0     arcinit.obj
 0001:00021a30       ??_C@_0EF@JADMGPAN@?$CK?5ConfigureContainersRuntime?3?5Ge@FNODOBFM@ 0000000140022a30     arcinit.obj
 0001:00021a80       ??_C@_0EM@NKPEDKJ@?$CK?5ConfigureContainersRuntime?3?5no@FNODOBFM@ 0000000140022a80     arcinit.obj
 0001:00021ad0       ??_C@_0EF@ECHMIPBP@?$CK?5Found?5a?5new?5container?5?9?5tid?3?5?$CF@FNODOBFM@ 0000000140022ad0     arcinit.obj
 0001:00021b20       ??_C@_0DK@FCJKMAGD@ConfigureContainersRuntime?3?5UID?5@FNODOBFM@ 0000000140022b20     arcinit.obj
 0001:00021b60       ??_C@_0DK@PHPDGAOG@?$CK?5ConfigureContainersRuntime?3?5di@FNODOBFM@ 0000000140022b60     arcinit.obj
 0001:00021ba0       ??_C@_0GG@BFFFADFC@?$CK?5ConfigureContainersRuntime?3?5Fa@FNODOBFM@ 0000000140022ba0     arcinit.obj
 0001:00021c10       ??_C@_0EA@JBBLNOGE@?$CK?5ConfigureContainersRuntime?3?5RA@FNODOBFM@ 0000000140022c10     arcinit.obj
 0001:00021c50       ??_C@_0FJ@MOJFHLFO@?$CK?5ConfigureContainersRuntime?3?5Di@FNODOBFM@ 0000000140022c50     arcinit.obj
 0001:00021cb0       ??_C@_0CO@FOBCLEMJ@?$CK?5ConfigureContainersRuntime?3?5di@FNODOBFM@ 0000000140022cb0     arcinit.obj
 0001:00021ce0       ??_C@_0DO@KMBICFHC@?$CK?5ConfigureContainersRuntime?3?5Sy@FNODOBFM@ 0000000140022ce0     arcinit.obj
 0001:00021d20       ??_C@_0DB@JMFIFBDA@leaving?5ConfigureContainersRunti@FNODOBFM@ 0000000140022d20     arcinit.obj
 0001:00021d60       ??_C@_0CC@KOGKIGDL@entering?5CheckForVersionMisMatch@FNODOBFM@ 0000000140022d60     arcinit.obj
 0001:00021d90       ??_C@_0CB@BOFDNAKM@This?5is?5a?5code?5stream?5identifier@FNODOBFM@ 0000000140022d90     arcinit.obj
 0001:00021dc0       ??_C@_1CE@PCDJGPON@?$AAB?$AAa?$AAd?$AA?5?$AAV?$AAe?$AAr?$AAs?$AAi?$AAo?$AAn?$AA?5?$AAM?$AAa?$AAt?$AAc?$AAh?$AA?$AA@FNODOBFM@ 0000000140022dc0     arcinit.obj
 0001:00021df0       ??_C@_0DF@MNNMPGOO@?$CK?5Version?5Mismatch?3?5Bios?3?$CFd?0?5Fir@FNODOBFM@ 0000000140022df0     arcinit.obj
 0001:00021e30       ??_C@_0EC@DEDLMEPI@leving?5CheckForVersionMisMatch?5w@FNODOBFM@ 0000000140022e30     arcinit.obj
 0001:00021e80       ??_C@_0BN@GKEKJNDP@?$CFs?5Driver?5entry?5rtnval?5?$DN?5?$CFx?6?$AA@FNODOBFM@ 0000000140022e80     arcinit.obj
 0001:00021ea0       ??_C@_0DD@FIIKPLIC@?$CFs?3?5Driver?5FindAdapter?5?9?5invalid@FNODOBFM@ 0000000140022ea0     arcinit.obj
 0001:00021ee0       ??_C@_0M@NCHBOPE@kernalprint?$AA@FNODOBFM@ 0000000140022ee0     arcinit.obj
 0001:00021ef0       ??_C@_0BE@IDLOJBGB@?$CK?5KERNAL?5PRINT?5?$DN?51?6?$AA@FNODOBFM@ 0000000140022ef0     arcinit.obj
 0001:00021f10       ??_C@_0BG@INJAEJHE@entering?5FindAdapter?6?$AA@FNODOBFM@ 0000000140022f10     arcinit.obj
 0001:00021f30       ??_C@_0FD@NLKPIIHJ@?$CK?5This?5is?5WS03?5R2?0?5Vista?5or?5Long@FNODOBFM@ 0000000140022f30     arcinit.obj
 0001:00021f90       ??_C@_0FF@EIPBDAPC@?$CK?$CK?$CK?$CK?$CK?5Size?5of?5PORT_CONFIGURATION@FNODOBFM@ 0000000140022f90     arcinit.obj
 0001:00021ff0       ??_C@_0EF@MDPAOPOH@?$CK?5HwScsiFindAdapter?3?5DeviceExten@FNODOBFM@ 0000000140022ff0     arcinit.obj
 0001:00022040       ??_C@_0CD@BBBDOKPE@?$CK?5Returned?5PCI?5bus?5data?5length?$DN?$CF@FNODOBFM@ 0000000140023040     arcinit.obj
 0001:00022070       ??_C@_0BB@ELNGMCEN@BreakPointHelper?$AA@FNODOBFM@ 0000000140023070     arcinit.obj
 0001:00022090       ??_C@_0BN@NMODDHNP@?$CK?53?5seconds?5waiting?5is?5done?6?$AA@FNODOBFM@ 0000000140023090     arcinit.obj
 0001:000220b0       ??_C@_0DD@OAOECDIB@leaving?5FindAdapter?5?9?5StorPortGe@FNODOBFM@ 00000001400230b0     arcinit.obj
 0001:000220f0       ??_C@_0DF@ODNFGMFG@?$CK?5leaving?5FindAdapter?5?9?5StorPort@FNODOBFM@ 00000001400230f0     arcinit.obj
 0001:00022130       ??_C@_0BN@FJDEMAMC@?$CK?50x40?5PCI?5Bus?5Data?5read?5in?6?$AA@FNODOBFM@ 0000000140023130     arcinit.obj
 0001:00022150       ??_C@_0BN@INBKDNHG@?$CK?50xFF?5PCI?5Bus?5Data?5read?5in?6?$AA@FNODOBFM@ 0000000140023150     arcinit.obj
 0001:00022170       ??_C@_0DB@DAIGEFPJ@?$CK?5No?5Support?5on?5Capabilties?5list@FNODOBFM@ 0000000140023170     arcinit.obj
 0001:000221b0       ??_C@_0BM@KCLFMKNE@?$CK?5Capability_offset?5?$DN?50x?$CFx?5?$AA@FNODOBFM@ 00000001400231b0     arcinit.obj
 0001:000221d0       ??_C@_0BJ@KNABCMMM@?5?9?9?$DOcapabilty_id?5?$DN?50x?$CFx?6?$AA@FNODOBFM@ 00000001400231d0     arcinit.obj
 0001:000221f0       ??_C@_0BK@JIIOJNIO@?$CK?5Message_control?5?$DN?50x?$CFx?6?$AA@FNODOBFM@ 00000001400231f0     arcinit.obj
 0001:00022210       ??_C@_0BF@HNFCBKLM@?$CK?5HW?5supports?5MSI?9X?6?$AA@FNODOBFM@ 0000000140023210     arcinit.obj
 0001:00022230       ??_C@_0L@BLEMHNKF@archbamode?$AA@FNODOBFM@ 0000000140023230     arcinit.obj
 0001:00022240       ??_C@_0BM@OFPMAGCK@?$CK?5ARC?5HBA?5MODE?5setting?3?5?$CFd?6?$AA@FNODOBFM@ 0000000140023240     arcinit.obj
 0001:00022260       ??_C@_07IICIIOGL@fibdump?$AA@FNODOBFM@ 0000000140023260     arcinit.obj
 0001:00022270       ??_C@_0BI@NEHBJBBP@?$CK?5FIB?5DUMP?5setting?3?5?$CFd?6?$AA@FNODOBFM@ 0000000140023270     arcinit.obj
 0001:00022290       ??_C@_09LEIBFFMJ@forceintx?$AA@FNODOBFM@ 0000000140023290     arcinit.obj
 0001:000222a0       ??_C@_0N@FCLAIEBP@forcepolling?$AA@FNODOBFM@ 00000001400232a0     arcinit.obj
 0001:000222b0       ??_C@_0DI@MNEPEDIK@?$CK?5StorPortGetActiveGroupCount?5ha@FNODOBFM@ 00000001400232b0     arcinit.obj
 0001:000222f0       ??_C@_0ED@JJDFFHPI@?$CK?5StorPortGetActiveGroupCount?5re@FNODOBFM@ 00000001400232f0     arcinit.obj
 0001:00022340       ??_C@_0DJ@FDFDEBND@?$CK?5StorPortGetHighestNodeNumber?5h@FNODOBFM@ 0000000140023340     arcinit.obj
 0001:00022380       ??_C@_0EL@PIGODLHL@?$CK?5StorPortGetHighestNodeNumber?5r@FNODOBFM@ 0000000140023380     arcinit.obj
 0001:000223d0       ??_C@_0EM@HBPALBEJ@?$CK?5StorPortGetHighestNodeNumber?5r@FNODOBFM@ 00000001400233d0     arcinit.obj
 0001:00022420       ??_C@_0DF@EDOFIEGL@?$CK?5StorPortGetGroupAffinity?5has?5n@FNODOBFM@ 0000000140023420     arcinit.obj
 0001:00022460       ??_C@_0HE@CADMEBCK@?$CK?5StorPortGetGroupAffinity?5retur@FNODOBFM@ 0000000140023460     arcinit.obj
 0001:000224e0       ??_C@_0EI@OFPHCHHN@?$CK?5StorPortGetGroupAffinity?5retur@FNODOBFM@ 00000001400234e0     arcinit.obj
 0001:00022530       ??_C@_0EO@MADFJJKE@?$CK?5StorPortGetGroupAffinity?5retur@FNODOBFM@ 0000000140023530     arcinit.obj
 0001:00022580       ??_C@_0P@JECJMKHH@runspecialcode?$AA@FNODOBFM@ 0000000140023580     arcinit.obj
 0001:00022590       ??_C@_0BI@LHEEIHDL@?$CK?5RUN?5SPECIAL?5CODE?5?$DN?51?6?$AA@FNODOBFM@ 0000000140023590     arcinit.obj
 0001:000225b0       ??_C@_0BI@LGIGONAM@?$CK?5RUN?5SPECIAL?5CODE?5?$DN?50?6?$AA@FNODOBFM@ 00000001400235b0     arcinit.obj
 0001:000225d0       ??_C@_0N@DDALOBCN@enablekidnap?$AA@FNODOBFM@ 00000001400235d0     arcinit.obj
 0001:000225e0       ??_C@_0BE@NKPEGEFN@?$CK?5Catchfib?5enabled?6?$AA@FNODOBFM@ 00000001400235e0     arcinit.obj
 0001:00022600       ??_C@_0BI@PLLAPJLO@?$CK?5Catchfib?5not?5enabled?6?$AA@FNODOBFM@ 0000000140023600     arcinit.obj
 0001:00022620       ??_C@_0M@KNIKEID@kidnapvalve?$AA@FNODOBFM@ 0000000140023620     arcinit.obj
 0001:00022630       ??_C@_0BF@CEDJMGLL@?$CK?5KIDNAP?5VALVE?5?$DN?5?$CFd?6?$AA@FNODOBFM@ 0000000140023630     arcinit.obj
 0001:00022650       ??_C@_0O@OCGMBHKL@checkinterval?$AA@FNODOBFM@ 0000000140023650     arcinit.obj
 0001:00022660       ??_C@_0CM@FEFEBKKC@?$CK?5IOP?5RESET?5COMPLETION?5Check?5Int@FNODOBFM@ 0000000140023660     arcinit.obj
 0001:00022690       ??_C@_0N@MOEJGNKK@stallseconds?$AA@FNODOBFM@ 0000000140023690     arcinit.obj
 0001:000226a0       ??_C@_0BG@DLFLFJEO@?$CK?5STALL?5SECONDS?5?$DN?5?$CFd?6?$AA@FNODOBFM@ 00000001400236a0     arcinit.obj
 0001:000226c0       ??_C@_0O@BPMKJHCJ@hbaqueuedepth?$AA@FNODOBFM@ 00000001400236c0     arcinit.obj
 0001:000226d0       ??_C@_0BI@IIHNBKPK@?$CK?5HBA?5QUEUE?5DEPTH?5?$DN?5?$CFd?6?$AA@FNODOBFM@ 00000001400236d0     arcinit.obj
 0001:000226f0       ??_C@_04GGLOKIEE@dump?$AA@FNODOBFM@ 00000001400236f0     arcinit.obj
 0001:00022700       ??_C@_05FDLGEGEK@ntldr?$AA@FNODOBFM@ 0000000140023700     arcinit.obj
 0001:00022710       ??_C@_05PMICOLGA@hiber?$AA@FNODOBFM@ 0000000140023710     arcinit.obj
 0001:00022720       ??_C@_0CD@JEMNEMMP@?$CK?$CK?$CK?$CK?5dump?5?$HM?5ntldr?5?$HM?5hiber?5is?5TRU@FNODOBFM@ 0000000140023720     arcinit.obj
 0001:00022750       ??_C@_0BK@NELCFLHO@?$CK?5Switching?5to?5INTx?5mode?6?$AA@FNODOBFM@ 0000000140023750     arcinit.obj
 0001:00022770       ??_C@_09IPELKJIO@BLEDCheck?$AA@FNODOBFM@ 0000000140023770     arcinit.obj
 0001:00022780       ??_C@_0L@NIPCGJOG@DPCAllowed?$AA@FNODOBFM@ 0000000140023780     arcinit.obj
 0001:00022790       ??_C@_09CHINNNMJ@CSMI?$DNNone?$AA@FNODOBFM@ 0000000140023790     arcinit.obj
 0001:000227a0       ??_C@_0BA@BKKNJKOP@CSMI?$DNRestricted?$AA@FNODOBFM@ 00000001400237a0     arcinit.obj
 0001:000227b0       ??_C@_09PKBPEONE@CSMI?$DNFull?$AA@FNODOBFM@ 00000001400237b0     arcinit.obj
 0001:000227c0       ??_C@_0CJ@JHBMKCEI@leaving?5FindAdapter?5?9?5PCI?5Id?5not@FNODOBFM@ 00000001400237c0     arcinit.obj
 0001:000227f0       ??_C@_0CL@HDBMPJMP@?$CK?5leaving?5FindAdapter?5?9?5PCI?5Id?5n@FNODOBFM@ 00000001400237f0     arcinit.obj
 0001:00022820       ??_C@_0CH@LNPKNDMP@Rx?3?5BAR0?5Range?50x?$CFlx?5MappedSize?5@FNODOBFM@ 0000000140023820     arcinit.obj
 0001:00022850       ??_C@_0DF@OFCBAPFL@leaving?5FindAdapter?5?9?5fail?5mappi@FNODOBFM@ 0000000140023850     arcinit.obj
 0001:00022890       ??_C@_0DH@MNDLADLD@?$CK?5leaving?5FindAdapter?5?9?5fail?5map@FNODOBFM@ 0000000140023890     arcinit.obj
 0001:000228d0       ??_C@_0DC@NODBFDAD@leaving?5FindAdapter?5?9?5illegal?5FW@FNODOBFM@ 00000001400238d0     arcinit.obj
 0001:00022910       ??_C@_0EH@FLDBENFC@?$CK?5leaving?5FindAdapter?5?9?5illegal?5@FNODOBFM@ 0000000140023910     arcinit.obj
 0001:00022960       ??_C@_0CK@GPLIPCCC@?$CK?5FULL?564?5BIT?5addressing?5support@FNODOBFM@ 0000000140023960     arcinit.obj
 0001:00022990       ??_C@_0CD@NJEIKDOH@?$CK?5New?5outstanding?5number?5chose?3?$CF@FNODOBFM@ 0000000140023990     arcinit.obj
 0001:000229c0       ??_C@_0CD@CCLGIJ@?$CK?5Old?5outstanding?5number?5chose?3?$CF@FNODOBFM@ 00000001400239c0     arcinit.obj
 0001:000229f0       ??_C@_05JGHMLIKJ@devqd?$AA@FNODOBFM@ 00000001400239f0     arcinit.obj
 0001:00022a00       ??_C@_0O@EPNNFPIH@?$CK?5DEV?5QD?3?5?$CFd?6?$AA@FNODOBFM@ 0000000140023a00     arcinit.obj
 0001:00022a10       ??_C@_0N@OEGLNJCG@ioctlbufsize?$AA@FNODOBFM@ 0000000140023a10     arcinit.obj
 0001:00022a20       ??_C@_0CI@LFOBEGIG@?$CK?5This?5is?564?9bit?5Vista?5or?5Longho@FNODOBFM@ 0000000140023a20     arcinit.obj
 0001:00022a50       ??_C@_0DB@NLEKMFMO@?$CK?5This?5is?532?9bit?5WS03?5R2?0?5Vista?5@FNODOBFM@ 0000000140023a50     arcinit.obj
 0001:00022a90       ??_C@_0CA@DJAEOOFI@?$CK?5This?5is?564?9bit?5WS03?5SP1?5?4?4?4?5?6?$AA@FNODOBFM@ 0000000140023a90     arcinit.obj
 0001:00022ab0       ??_C@_0CA@IELABMFO@?$CK?5This?5is?532?9bit?5WS03?5SP1?5?4?4?4?5?6?$AA@FNODOBFM@ 0000000140023ab0     arcinit.obj
 0001:00022ad0       ??_C@_0CA@MNGBKCLD@?$CK?5This?5is?532?9bit?5WS03?5RTM?5?4?4?4?5?6?$AA@FNODOBFM@ 0000000140023ad0     arcinit.obj
 0001:00022af0       ??_C@_0BL@FPDNGGII@?$CK?5Adapter?5is?5in?5poll?5mode?6?$AA@FNODOBFM@ 0000000140023af0     arcinit.obj
 0001:00022b10       ??_C@_0CO@NGAJFGIM@?$CK?5pDeviceExtension?9?$DONewCommInter@FNODOBFM@ 0000000140023b10     arcinit.obj
 0001:00022b40       ??_C@_0CE@MCFGELJ@?$CK?5pDeviceExtension?9?$DOVendorId?3?50x@FNODOBFM@ 0000000140023b40     arcinit.obj
 0001:00022b70       ??_C@_0CE@PNKCKBKJ@?$CK?5pDeviceExtension?9?$DODeviceId?3?50x@FNODOBFM@ 0000000140023b70     arcinit.obj
 0001:00022ba0       ??_C@_0CH@NNKEKBEL@?$CK?5pDeviceExtension?9?$DOSubVendorId?3@FNODOBFM@ 0000000140023ba0     arcinit.obj
 0001:00022bd0       ??_C@_0CH@BEBMHIHH@?$CK?5pDeviceExtension?9?$DOSubSystemId?3@FNODOBFM@ 0000000140023bd0     arcinit.obj
 0001:00022c00       ??_C@_0CB@ELGCJIGA@?$CK?5Uncached?5Memory?5address?3?50x?$CFp?6@FNODOBFM@ 0000000140023c00     arcinit.obj
 0001:00022c30       ??_C@_0CH@CKCEEBMD@?$CK?5Uncached?5Memory?5allocated?3?50x?$CF@FNODOBFM@ 0000000140023c30     arcinit.obj
 0001:00022c60       ??_C@_0DK@INJPNBCP@?$CK?5MailBox?51?3?$CFx?0?5MailBox?52?3?$CFx?0?5Ma@FNODOBFM@ 0000000140023c60     arcinit.obj
 0001:00022ca0       ??_C@_0DB@DBAPOAM@?$CK?5pDeviceExtension?9?$DOMaxOutstandi@FNODOBFM@ 0000000140023ca0     arcinit.obj
 0001:00022ce0       ??_C@_0DF@CKKIGFIG@?$CK?5pDeviceExtension?9?$DOMaxMSIXVecto@FNODOBFM@ 0000000140023ce0     arcinit.obj
 0001:00022d20       ??_C@_0M@EHMNKBMA@forcev8tov7?$AA@FNODOBFM@ 0000000140023d20     arcinit.obj
 0001:00022d30       ??_C@_0CA@HGCPDEFI@?$CK?5SupportV8InitStruct?5Flag?3?5?$CFd?6?$AA@FNODOBFM@ 0000000140023d30     arcinit.obj
 0001:00022d50       ??_C@_0BA@EOIIECBM@loopbacklatency?$AA@FNODOBFM@ 0000000140023d50     arcinit.obj
 0001:00022d60       ??_C@_0BC@BDCJEMN@?$CK?5FORCE?5INTX?3?5?$CFd?6?$AA@FNODOBFM@ 0000000140023d60     arcinit.obj
 0001:00022d80       ??_C@_0BF@FJIEGFMA@?$CK?5FORCE?5POLLING?3?5?$CFd?6?$AA@FNODOBFM@ 0000000140023d80     arcinit.obj
 0001:00022da0       ??_C@_0CN@OMCAJNOM@?$CK?5?$DN?$DN?$DN?$DN?$DN?$DN?$DO?5Front?5Vector?5Number?5is@FNODOBFM@ 0000000140023da0     arcinit.obj
 0001:00022dd0       ??_C@_0CI@BJJEDHMG@?$CK?5pDeviceExtension?9?$DOVectorCapaci@FNODOBFM@ 0000000140023dd0     arcinit.obj
 0001:00022e00       ??_C@_0DE@JJAKLEJD@?$CK?5pDeviceExtension?9?$DOMSIXIoThrott@FNODOBFM@ 0000000140023e00     arcinit.obj
 0001:00022e40       ??_C@_0DF@LMKAIIEG@?$CK?5pDeviceExtension?9?$DOMSIXIoThrott@FNODOBFM@ 0000000140023e40     arcinit.obj
 0001:00022e80       ??_C@_0BK@NKHDFADJ@?$CK?5CPU?5Group?5number?5is?5?$CFd?6?$AA@FNODOBFM@ 0000000140023e80     arcinit.obj
 0001:00022ea0       ??_C@_0BJ@OBKJCBPL@?$CK?5CPU?5Node?5number?5is?5?$CFd?6?$AA@FNODOBFM@ 0000000140023ea0     arcinit.obj
 0001:00022ec0       ??_C@_0BI@KNCDOCH@?$CK?5Node?5per?5Group?5is?5?$CFd?6?$AA@FNODOBFM@ 0000000140023ec0     arcinit.obj
 0001:00022ee0       ??_C@_0BH@FMFCFLGH@?$CK?5Core?5per?5Node?5is?5?$CFd?6?$AA@FNODOBFM@ 0000000140023ee0     arcinit.obj
 0001:00022f00       ??_C@_0CB@HDFPBACC@?$CK?5System?5processor?5number?5is?5?$CFd?6@FNODOBFM@ 0000000140023f00     arcinit.obj
 0001:00022f30       ??_C@_0CI@EOOKBOFL@?$CK?5?$DN?$DN?$DN?$DN?$DN?$DN?$DO?5End?5of?5Front?5summary?5?$DM@FNODOBFM@ 0000000140023f30     arcinit.obj
 0001:00022f60       ??_C@_0DE@FBKNPKIG@?$CK?5?$DN?$DN?$DN?$DN?$DN?$DN?$DO?5inside?5finalizing?5vect@FNODOBFM@ 0000000140023f60     arcinit.obj
 0001:00022fa0       ??_C@_06DCBAGJIF@vecnum?$AA@FNODOBFM@ 0000000140023fa0     arcinit.obj
 0001:00022fb0       ??_C@_0EB@PLAOEAEF@?$CK?5Valid_MSIX_Vectors?5is?5reset?5to@FNODOBFM@ 0000000140023fb0     arcinit.obj
 0001:00023000       ??_C@_0CN@KPEBIFEO@?$CK?5?$DN?$DN?$DN?$DN?$DN?$DN?$DO?5Final?5Vector?5Number?5is@FNODOBFM@ 0000000140024000     arcinit.obj
 0001:00023030       ??_C@_0CC@CEGCGDDK@?$CK?5?$DN?$DN?$DN?$DN?$DN?$DN?$DO?5End?5of?5summary?5?$DM?$DN?$DN?$DN?$DN?$DN?$DN@FNODOBFM@ 0000000140024030     arcinit.obj
 0001:00023060       ??_C@_0EC@KMMHNEKL@?$CK?5ConfigInfo?9?$DOHwMSInterruptRouti@FNODOBFM@ 0000000140024060     arcinit.obj
 0001:000230b0       ??_C@_0BH@CDLDBOJF@?$CK?5SrbExtensionSize?3?$CFx?6?$AA@FNODOBFM@ 00000001400240b0     arcinit.obj
 0001:000230d0       ??_C@_0EK@GNODIBNL@?$CK?5MiniARC?5Interface?5?9?5?5CommandSi@FNODOBFM@ 00000001400240d0     arcinit.obj
 0001:00023120       ??_C@_0EL@HJMLPDNI@?$CK?5New?5Comm?5Interface?5?9?5?5CommandS@FNODOBFM@ 0000000140024120     arcinit.obj
 0001:00023170       ??_C@_0CM@NKHNJDEG@leaving?5FindAdapter?5?9?5fail?5initi@FNODOBFM@ 0000000140024170     arcinit.obj
 0001:000231a0       ??_C@_0CO@GHEIBKDI@?$CK?5leaving?5FindAdapter?5?9?5fail?5ini@FNODOBFM@ 00000001400241a0     arcinit.obj
 0001:000231d0       ??_C@_1EA@GNKDGDHK@?$AAA?$AAd?$AAa?$AAp?$AAt?$AAe?$AAr?$AA?5?$AAg?$AAo?$AAt?$AA?5?$AAi?$AAn?$AAv?$AAa?$AAl?$AAi?$AAd?$AA?5?$AAh?$AAo?$AAs?$AAt?$AA?5?$AAw?$AAi?$AAn?$AAd?$AAo?$AAw?$AA?$AA@FNODOBFM@ 00000001400241d0     arcinit.obj
 0001:00023210       ??_C@_1EI@NELDFHEH@?$AAA?$AAd?$AAa?$AAp?$AAt?$AAe?$AAr?$AA?5?$AAd?$AAo?$AAe?$AAs?$AA?5?$AAn?$AAo?$AAt?$AA?5?$AAs?$AAu?$AAp?$AAp?$AAo?$AAr?$AAt?$AA?5?$AA4?$AAG?$AAB?$AA?5?$AAw?$AAi?$AAn@FNODOBFM@ 0000000140024210     arcinit.obj
 0001:00023260       ??_C@_0DC@BFHJHJOO@?$CK?5fail?5SynFibCT_SET_MINIARC_HOST@FNODOBFM@ 0000000140024260     arcinit.obj
 0001:000232a0       ??_C@_0DF@KABMIJBB@?$CK?5RequestSupplementAdapterInfo?0?5@FNODOBFM@ 00000001400242a0     arcinit.obj
 0001:000232e0       ??_C@_0CE@IADADNNA@?$CK?5Use?5MU?5Register?5for?5IOP_Reset?4@FNODOBFM@ 00000001400242e0     arcinit.obj
 0001:00023310       ??_C@_0CJ@LHHNJCHI@?$CK?5Use?5inbound?5doorbell?5for?5IOP_R@FNODOBFM@ 0000000140024310     arcinit.obj
 0001:00023340       ??_C@_0DI@LGINDMLA@?$CK?5ERROR?3?5FW?5does?5not?5provide?5whi@FNODOBFM@ 0000000140024340     arcinit.obj
 0001:00023380       ??_C@_0BP@DJKPJIGJ@?$CK?5Ignore_IOP_Reset?5is?5set?5?4?4?4?6?$AA@FNODOBFM@ 0000000140024380     arcinit.obj
 0001:000233a0       ??_C@_0CK@LEDHDPPJ@?$CK?5Disk?5Power?5Management?5is?5suppo@FNODOBFM@ 00000001400243a0     arcinit.obj
 0001:000233d0       ??_C@_0CJ@PJOACPGJ@?$CK?5This?5firmware?5supports?5fast?5JB@FNODOBFM@ 00000001400243d0     arcinit.obj
 0001:00023400       ??_C@_0DB@HEHLEMPI@?$CK?5Controller?5Firmware?5supports?5S@FNODOBFM@ 0000000140024400     arcinit.obj
 0001:00023440       ??_C@_0CI@CJPAOACI@?$CK?5Controller?5Firmware?5supports?52@FNODOBFM@ 0000000140024440     arcinit.obj
 0001:00023470       ??_C@_0BM@LNCHEOOO@?$CK?5Virtual?5B?1T?1L?5?$CI?$CFd?1?$CFd?1?$CFd?$CJ?6?$AA@FNODOBFM@ 0000000140024470     arcinit.obj
 0001:00023490       ??_C@_0DA@OBMGONKI@?$CK?5Driver?5got?5SUPPORTED_NATIVE_HB@FNODOBFM@ 0000000140024490     arcinit.obj
 0001:000234c0       ??_C@_0DI@GIKAIFLA@?$CK?5Driver?5did?5not?5get?5SUPPORTED_N@FNODOBFM@ 00000001400244c0     arcinit.obj
 0001:00023500       ??_C@_0BH@LMHJIEKF@?$CK?5ExposeNonDASD?5is?5?$CFx?6?$AA@FNODOBFM@ 0000000140024500     arcinit.obj
 0001:00023520       ??_C@_0BB@JIKBMNNG@QueueDepthPerLun?$AA@FNODOBFM@ 0000000140024520     arcinit.obj
 0001:00023540       ??_C@_0N@GDDJMKFE@PauseIOLimit?$AA@FNODOBFM@ 0000000140024540     arcinit.obj
 0001:00023550       ??_C@_0O@LIIBGGCF@ResumeIOLimit?$AA@FNODOBFM@ 0000000140024550     arcinit.obj
 0001:00023560       ??_C@_0O@OKMDGJBG@ConvertSGList?$AA@FNODOBFM@ 0000000140024560     arcinit.obj
 0001:00023570       ??_C@_0BE@IIJOOEPG@QueueStartThreshold?$AA@FNODOBFM@ 0000000140024570     arcinit.obj
 0001:00023590       ??_C@_0BD@CEDPKLI@QueueDumpThreshold?$AA@FNODOBFM@ 0000000140024590     arcinit.obj
 0001:000235b0       ??_C@_0BA@NLIGFJMK@MaxIoSizeQueued?$AA@FNODOBFM@ 00000001400245b0     arcinit.obj
 0001:000235c0       ??_C@_0N@MLHJOFDC@QueueAllowed?$AA@FNODOBFM@ 00000001400245c0     arcinit.obj
 0001:000235d0       ??_C@_0BC@IEBJFOIJ@FlushSizeInBlocks?$AA@FNODOBFM@ 00000001400245d0     arcinit.obj
 0001:000235f0       ??_C@_0EA@OJJGPBKL@leaving?5FindAdapter?5?9?5fail?5Handl@FNODOBFM@ 00000001400245f0     arcinit.obj
 0001:00023630       ??_C@_0EC@HNCBOCML@?$CK?5leaving?5FindAdapter?5?9?5fail?5Han@FNODOBFM@ 0000000140024630     arcinit.obj
 0001:00023680       ??_C@_09NBOIBGGK@EnableWMI?$AA@FNODOBFM@ 0000000140024680     arcinit.obj
 0001:00023690       ??_C@_0DH@OIMAJCMK@?$CK?5?9?5Driver?5version?5?$CFs?0?5adapter?5n@FNODOBFM@ 0000000140024690     arcinit.obj
 0001:000236d0       ??_C@_0DF@NGIHOECA@?$CK?5?9?5Size?5of?5HwDevExt?$DN0x?$CFx?4?5Size?5@FNODOBFM@ 00000001400246d0     arcinit.obj
 0001:00023710       ??_C@_0IC@BPBMMOAO@?$CK?5?9?5Size?$CISrbExt?$CJ?$DN0x?$CFx?4?5sizeof?$CIFI@FNODOBFM@ 0000000140024710     arcinit.obj
 0001:000237a0       ??_C@_0CA@ENCHFGMA@?$CK?5?9?5reported?5Size?$CISrbExt?$CJ?$DN0x?$CFx?6?$AA@FNODOBFM@ 00000001400247a0     arcinit.obj
 0001:000237c0       ??_C@_0BG@JAEBOKND@?$CK?5?9?5Done?5FindAdapter?6?$AA@FNODOBFM@ 00000001400247c0     arcinit.obj
 0001:000237e0       ??_C@_0FF@LMEIGAGF@?$CK?5?9?5ConfigInfo?9?$DOMaximumTransferL@FNODOBFM@ 00000001400247e0     arcinit.obj
 0001:00023840       ??_C@_0CG@GOHAMHPA@leaving?5FindAdapter?5?9?5adapter?5fo@FNODOBFM@ 0000000140024840     arcinit.obj
 0001:00023870       ??_C@_0BN@DGMFEGDN@entering?5GetElapsedSeconds?5?6?$AA@FNODOBFM@ 0000000140024870     arcinit.obj
 0001:00023890       ??_C@_0DD@GOLHMOHG@leaving?5GetElapsedSeconds?5?9?5seco@FNODOBFM@ 0000000140024890     arcinit.obj
 0001:000238d0       ??_C@_0CJ@KCPJKGH@entering?5IsAdapterReadyForConfig@FNODOBFM@ 00000001400248d0     arcinit.obj
 0001:00023900       ??_C@_0DB@PNDBFHEI@IsAdapterReadyForConfigCommand?3?5@FNODOBFM@ 0000000140024900     arcinit.obj
 0001:00023940       ??_C@_0CH@PFKKGKLP@IsAdapterReadyForConfigCommand?3?5@FNODOBFM@ 0000000140024940     arcinit.obj
 0001:00023970       ??_C@_0DJ@FMKIDFML@?$CK?5leaving?5IsAdapterReadyForConfi@FNODOBFM@ 0000000140024970     arcinit.obj
 0001:000239b0       ??_C@_0CI@LLJGECEO@leaving?5IsAdapterReadyForConfigC@FNODOBFM@ 00000001400249b0     arcinit.obj
 0001:000239e0       ??_C@_0BD@LJONEFCN@entering?5IOPReset?6?$AA@FNODOBFM@ 00000001400249e0     arcinit.obj
 0001:00023a00       ??_C@_0EN@CPGMGMBD@?$CK?$CK?5Fail?5to?5iopreset?5the?5adapter?5@FNODOBFM@ 0000000140024a00     arcinit.obj
 0001:00023a50       ??_C@_0GF@NGDIBMBA@?$CK?5Driver?5has?5been?5waiting?55?5seco@FNODOBFM@ 0000000140024a50     arcinit.obj
 0001:00023ac0       ??_C@_1CG@OOCCJMGE@?$AAI?$AAO?$AAP?$AA?5?$AAR?$AAE?$AAS?$AAE?$AAT?$AA?5?$AAd?$AAi?$AAs?$AAa?$AAb?$AAl?$AAe?$AAd?$AA?$AA@FNODOBFM@ 0000000140024ac0     arcinit.obj
 0001:00023af0       ??_C@_1CC@HLNFBNCO@?$AAI?$AAO?$AAP?$AA?5?$AAR?$AAE?$AAS?$AAE?$AAT?$AA?5?$AAf?$AAa?$AAi?$AAl?$AAe?$AAd?$AA?$AA@FNODOBFM@ 0000000140024af0     arcinit.obj
 0001:00023b20       ??_C@_0DE@GCJLBNBN@?$CK?$CK?5Fail?5to?5iopreset?5the?5adapter?0@FNODOBFM@ 0000000140024b20     arcinit.obj
 0001:00023b60       ??_C@_0BI@DKKBLGKC@?$CK?$CK?5IOPReset?5succeeded?4?6?$AA@FNODOBFM@ 0000000140024b60     arcinit.obj
 0001:00023b80       ??_C@_0DG@MCABGJKN@Driver?5should?5not?5work?5under?5MSI@FNODOBFM@ 0000000140024b80     arcinit.obj
 0001:00023bc0       ??_C@_0DE@DDNIODIO@?$CK?5Set?5pInitStruct?9?$DONoOfMsiVector@FNODOBFM@ 0000000140024bc0     arcinit.obj
 0001:00023c00       ??_C@_0BC@JKJGEENA@leaving?5IOPReset?6?$AA@FNODOBFM@ 0000000140024c00     arcinit.obj
 0001:00023c20       ??_C@_0HE@MJKNAGNA@?$CK?$CK?5Fib2?5sent?560?5seconds?5ago?3?5B?1T@FNODOBFM@ 0000000140024c20     arcinit.obj
 0001:00023ca0       ??_C@_0HE@MLFEGAEP@?$CK?$CK?5Fib1?5sent?560?5seconds?5ago?3?5B?1T@FNODOBFM@ 0000000140024ca0     arcinit.obj
 0001:00023d20       ??_C@_0EB@NJFNJFPK@?$CK?$CK?5Driver?5internal?5AIF?5FIB?5has?5n@FNODOBFM@ 0000000140024d20     arcinit.obj
 0001:00023d70       ??_C@_0EN@EHHFOLPM@?$CK?$CK?5returned?5?$CFd?5SRB?5to?5OS?5at?5Retu@FNODOBFM@ 0000000140024d70     arcinit.obj
 0001:00023dc0       ??_C@_0EB@JKABANOB@?$CK?$CK?5Returned?5?$CFd?5SRB?5to?5OS?5at?5Retu@FNODOBFM@ 0000000140024dc0     arcinit.obj
 0001:00023e10       ??_C@_0BK@OLLEIHIC@?$CK?5Switching?5to?5MSIx?5mode?6?$AA@FNODOBFM@ 0000000140024e10     arcinit.obj
 0001:00023e30       ??_C@_0BA@EAOKKBLN@?$CK?5MSIx?5Enabled?6?$AA@FNODOBFM@ 0000000140024e30     arcinit.obj
 0001:00023e40       ??_C@_0EB@JEEKIEDM@?$CK?5Set?5pInitStruct?9?$DONoOfMsiVector@FNODOBFM@ 0000000140024e40     arcinit.obj
 0001:00023e90       ??_C@_0EA@DFHNCIMC@?$CK?5Set?5pInitStruct?9?$DONoOfMsiVector@FNODOBFM@ 0000000140024e90     arcinit.obj
 0001:00023ed0       ??_C@_0FP@EFJPBKEO@?$CK?5Valid?5Vector?$CI?$CFd?$CJ?0?5msix?5capabil@FNODOBFM@ 0000000140024ed0     arcinit.obj
 0001:00023f30       ??_C@_0CE@KCFAPPCO@?$CK?5Coalescing?5Disabled?5in?5INTx?5Mo@FNODOBFM@ 0000000140024f30     arcinit.obj
 0001:00023f60       ??_C@_0BE@OKKJEBLK@?$CK?5MSIX?5NOT?5Enabled?6?$AA@FNODOBFM@ 0000000140024f60     arcinit.obj
 0001:00023f80       ??_C@_0DJ@NFBMPICJ@?$CK?5Thor?5V8?5INIT?5structure?5sent?5su@FNODOBFM@ 0000000140024f80     arcinit.obj
 0001:00023fc0       ??_C@_0DK@LLCEGMEJ@?$CK?5NON?9Thor?5INIT?5structure?5sent?5s@FNODOBFM@ 0000000140024fc0     arcinit.obj
 0001:00024000       ??_C@_0DE@DCIDKABN@?$CK?5V8?5INIT?5structure?5sent?5success@FNODOBFM@ 0000000140025000     arcinit.obj
 0001:00024040       ??_C@_0DI@LJKDAFIG@?$CK?5NON?9V8?5INIT?5structure?5sent?5suc@FNODOBFM@ 0000000140025040     arcinit.obj
 0001:00024080       ??_C@_0ED@LLOJEJPI@leaving?5HandleAdapterGetConfig?5a@FNODOBFM@ 0000000140025080     arcinit.obj
 0001:000240d0       ??_C@_0EF@MHNEOFPB@?$CK?5leaving?5HandleAdapterGetConfig@FNODOBFM@ 00000001400250d0     arcinit.obj
 0001:00024120       ??_C@_0DP@PECHNPGJ@leaving?5HandleAdapterGetConfig?5a@FNODOBFM@ 0000000140025120     arcinit.obj
 0001:00024160       ??_C@_0EB@CHAPDLOA@?$CK?5leaving?5HandleAdapterGetConfig@FNODOBFM@ 0000000140025160     arcinit.obj
 0001:000241b0       ??_C@_0EC@JNDOKFCE@leaving?5HandleAdapterCommitConfi@FNODOBFM@ 00000001400251b0     arcinit.obj
 0001:00024200       ??_C@_0EE@HMHNBLOK@?$CK?5leaving?5HandleAdapterCommitCon@FNODOBFM@ 0000000140025200     arcinit.obj
 0001:00024250       ??_C@_0CE@FDDAIENL@entering?5HandleAdapterConfigIssu@FNODOBFM@ 0000000140025250     arcinit.obj
 0001:00024280       ??_C@_0EG@EOLGKFDM@leaving?5HandleAdapterConfigIssue@FNODOBFM@ 0000000140025280     arcinit.obj
 0001:000242d0       ??_C@_0EI@BLLNCBDL@?$CK?5leaving?5HandleAdapterConfigIss@FNODOBFM@ 00000001400252d0     arcinit.obj
 0001:00024320       ??_C@_0EC@KFDDDOGD@leaving?5HandleAdapterConfigIssue@FNODOBFM@ 0000000140025320     arcinit.obj
 0001:00024370       ??_C@_0EE@EEHAIAKN@?$CK?5leaving?5HandleAdapterConfigIss@FNODOBFM@ 0000000140025370     arcinit.obj
 0001:000243c0       ??_C@_0EC@EGKDAAOP@leaving?5HandleAdapterConfigIssue@FNODOBFM@ 00000001400253c0     arcinit.obj
 0001:00024410       ??_C@_0EE@KHOALOCB@?$CK?5leaving?5HandleAdapterConfigIss@FNODOBFM@ 0000000140025410     arcinit.obj
 0001:00024460       ??_C@_0CD@FIHDJCJC@leaving?5HandleAdapterConfigIssue@FNODOBFM@ 0000000140025460     arcinit.obj
 0001:00024490       ??_C@_0BK@LNIBADPE@?$CK?5Setting?5StatusBatching?6?$AA@FNODOBFM@ 0000000140025490     arcinit.obj
 0001:000244b0       ??_C@_0EF@JDALIICL@?$CK?5Firmware?5should?5support?5ACI2?5i@FNODOBFM@ 00000001400254b0     arcinit.obj
 0001:00024500       ??_C@_0CB@DDHFLEBF@?$CK?5FW?5sets?5KERNEL_UP_AND_RUNNING?6@FNODOBFM@ 0000000140025500     arcinit.obj
 0001:00024530       ??_C@_0CC@HECBNNJJ@?$CK?5FW?5is?5ready?5for?5config?5command@FNODOBFM@ 0000000140025530     arcinit.obj
 0001:00024560       ??_C@_0BJ@GODFBPEB@?$CK?5Get?5config?5from?5FW?5ok?6?$AA@FNODOBFM@ 0000000140025560     arcinit.obj
 0001:00024580       ??_C@_0BK@PANMBLHC@?$CK?5Commit?5config?5to?5FW?5ok?6?$AA@FNODOBFM@ 0000000140025580     arcinit.obj
 0001:000245a0       ??_C@_0CA@BDIKNGAL@?$CK?5INIT?5Structure?5sent?5to?5FW?5ok?6?$AA@FNODOBFM@ 00000001400255a0     arcinit.obj
 0001:000245c0       ??_C@_0EE@GNMBAHCA@?$CK?5Get?5FW?5debug?5buffer?5failed?0?5bu@FNODOBFM@ 00000001400255c0     arcinit.obj
 0001:00024610       ??_C@_0BH@FLOGONBD@?$CK?5?9?5Driver?5version?5?$CFs?6?$AA@FNODOBFM@ 0000000140025610     arcinit.obj
 0001:00024630       ??_C@_0DN@NNHBAELD@SMNormalModeInitAdapter?3?5Soft?5Re@FNODOBFM@ 0000000140025630     arcinit.obj
 0001:00024670       ??_C@_0BO@IEENCLHE@entering?5HwInitializeAdapter?6?$AA@FNODOBFM@ 0000000140025670     arcinit.obj
 0001:00024690       ??_C@_1CA@OFEHMOBK@?$AAB?$AAa?$AAd?$AA?5?$AAP?$AAo?$AAr?$AAt?$AA?5?$AAD?$AAr?$AAi?$AAv?$AAe?$AAr?$AA?$AA@FNODOBFM@ 0000000140025690     arcinit.obj
 0001:000246b0       ??_C@_0FM@FIFECPG@?$CK?5pDeviceExtension?9?$DOValid_MSIX_V@FNODOBFM@ 00000001400256b0     arcinit.obj
 0001:00024710       ??_C@_0EH@ONHPKJKD@?$CK?5StorPortGetMSIInfo?5returned?5Fa@FNODOBFM@ 0000000140025710     arcinit.obj
 0001:00024760       ??_C@_0EC@KLPNNIKH@?$CK?5StorPortGetMSIInfo?5returned?5st@FNODOBFM@ 0000000140025760     arcinit.obj
 0001:000247b0       ??_C@_0EE@OLLCNNAO@?$CK?5StorPortGetMSIInfo?5returned?5st@FNODOBFM@ 00000001400257b0     arcinit.obj
 0001:00024800       ??_C@_0EJ@OBPFJGIJ@?$CK?5StorPortGetMSIInfo?5returned?5st@FNODOBFM@ 0000000140025800     arcinit.obj
 0001:00024850       ??_C@_0CF@FDBIIPFF@?$CK?5This?5Tupelo?5driver?5is?5MSI?5enab@FNODOBFM@ 0000000140025850     arcinit.obj
 0001:00024880       ??_C@_0BO@FHHBMMGN@?$CK?5PerfConfigData?4Flags?3?50x?$CFx?6?$AA@FNODOBFM@ 0000000140025880     arcinit.obj
 0001:000248a0       ??_C@_0FE@LBLIGLIO@GetDoorbellMaskForIOPReset?5retur@FNODOBFM@ 00000001400258a0     arcinit.obj
 0001:00024900       ??_C@_0DN@IMFNPMPP@?$CK?5Failed?5to?5Initialize?5Adapter?5i@FNODOBFM@ 0000000140025900     arcinit.obj
 0001:00024940       ??_C@_0DE@CMNGFMDL@?$CK?5Succeed?5to?5Initialize?5Adapter?5@FNODOBFM@ 0000000140025940     arcinit.obj
 0001:00024980       ??_C@_0EG@KGJBNOFG@?$CK?5Failed?5to?5Initialize?5Adapter?5i@FNODOBFM@ 0000000140025980     arcinit.obj
 0001:000249d0       ??_C@_0BP@MCCOMIEF@?$CK?5leaving?5HwInitializeAdapter?6?$AA@FNODOBFM@ 00000001400259d0     arcinit.obj
 0001:000249f0       ??_C@_0FN@OJHBJJGK@?$CK?5StorPortAllocateContiguousMemo@FNODOBFM@ 00000001400259f0     arcinit.obj
 0001:00024a50       ??_C@_0FD@MKBBGMOP@?$CK?5PROBLEM?3?5returnedSize?5?$DN?50?5?$CISto@FNODOBFM@ 0000000140025a50     arcinit.obj
 0001:00024ab0       ??_C@_0IH@LCJNFDMG@?$CK?5StorPortAllocateContiguousMemo@FNODOBFM@ 0000000140025ab0     arcinit.obj
 0001:00024b40       ??_C@_0BI@BOGNCAIA@entering?5InitializeDPC?6?$AA@FNODOBFM@ 0000000140025b40     arcinit.obj
 0001:00024b60       ??_C@_0BL@ICGKMMAJ@?$CK?5Start?5scanning?5group?5?$CFd?6?$AA@FNODOBFM@ 0000000140025b60     arcinit.obj
 0001:00024b80       ??_C@_0CO@FDNLALKJ@?$CK?5Group?5Affinity?5for?5msix?5vector@FNODOBFM@ 0000000140025b80     arcinit.obj
 0001:00024bb0       ??_C@_0DA@FPNPLEPN@?$CK?5NUMA?5node?5for?5MSIX?5vector?5?$CFd?5i@FNODOBFM@ 0000000140025bb0     arcinit.obj
 0001:00024be0       ??_C@_0DP@MAPFHEEH@?$CK?5Outbound?5Queue?5Memory?5allocate@FNODOBFM@ 0000000140025be0     arcinit.obj
 0001:00024c20       ??_C@_0CG@GFDFODNM@?$CK?5MemoryBlock?5?$CFd?5assigned?5in?5nod@FNODOBFM@ 0000000140025c20     arcinit.obj
 0001:00024c50       ??_C@_0DG@CGCBEMEO@?$CK?5MSG?5CAP?5setup?5failed?5?$CIbecause?5@FNODOBFM@ 0000000140025c50     arcinit.obj
 0001:00024c90       ??_C@_0ED@CJAGENOE@?$CK?5we?5are?5processing?5last?5MSIX?5ve@FNODOBFM@ 0000000140025c90     arcinit.obj
 0001:00024ce0       ??_C@_0HA@GKDMKHHO@?$CK?5we?5have?5a?5problem?4?5All?5groups?1@FNODOBFM@ 0000000140025ce0     arcinit.obj
 0001:00024d50       ??_C@_0FD@LFCJJKMC@?$CK?5StorPortGetLogicalProcessorRel@FNODOBFM@ 0000000140025d50     arcinit.obj
 0001:00024db0       ??_C@_0BG@FAIHHGLA@?$CK?5Vector?5?$CFd?5is?5done?6?6?$AA@FNODOBFM@ 0000000140025db0     arcinit.obj
 0001:00024dd0       ??_C@_0DJ@MGMHFMAN@?$CK?5Failed?5to?5Initialize?5Adapter?5i@FNODOBFM@ 0000000140025dd0     arcinit.obj
 0001:00024e10       ??_C@_0DA@GDJCAINB@?$CK?5Succeed?5to?5Initialize?5Adapter?5@FNODOBFM@ 0000000140025e10     arcinit.obj
 0001:00024e40       ??_C@_0BJ@CFFELFMJ@?$CK?5MSIx?5DPCs?5initialized?6?$AA@FNODOBFM@ 0000000140025e40     arcinit.obj
 0001:00024e60       ??_C@_0BI@LAPEOFCN@?$CK?5?9?5Done?5InitializeDPC?6?$AA@FNODOBFM@ 0000000140025e60     arcinit.obj
 0001:00024e80       ??_C@_0BH@PAHICDNJ@leaving?5InitializeDPC?6?$AA@FNODOBFM@ 0000000140025e80     arcinit.obj
 0001:00024ea0       ??_C@_0CP@OJKLKHLO@entering?5InitializeConsumerProdu@FNODOBFM@ 0000000140025ea0     arcinit.obj
 0001:00024ed0       ??_C@_0DE@MJJEGAKI@leaving?5InitializeConsumerProduc@FNODOBFM@ 0000000140025ed0     arcinit.obj
 0001:00024f10       ??_C@_0CO@NEGLFCOP@leaving?5InitializeConsumerProduc@FNODOBFM@ 0000000140025f10     arcinit.obj
 0001:00024f40       ??_C@_0CP@IKCNDLML@entering?5InitializeConsumerProdu@FNODOBFM@ 0000000140025f40     arcinit.obj
 0001:00024f70       ??_C@_0DF@IICIHNDP@leaving?5InitializeConsumerProduc@FNODOBFM@ 0000000140025f70     arcinit.obj
 0001:00024fb0       ??_C@_0DE@OBANPGHF@leaving?5InitializeConsumerProduc@FNODOBFM@ 0000000140025fb0     arcinit.obj
 0001:00024ff0       ??_C@_0CP@GDFIJJML@entering?5InitializeMessageUnitQu@FNODOBFM@ 0000000140025ff0     arcinit.obj
 0001:00025020       ??_C@_0DF@CLHHLLI@leaving?5InitializeMessageUnitQue@FNODOBFM@ 0000000140026020     arcinit.obj
 0001:00025060       ??_C@_0DE@BBDIIBAC@leaving?5InitializeMessageUnitQue@FNODOBFM@ 0000000140026060     arcinit.obj
 0001:000250a0       ??_C@_0BI@PNFIHJKN@entering?5MapDeviceBase?6?$AA@FNODOBFM@ 00000001400260a0     arcinit.obj
 0001:000250c0       ??_C@_1CM@FGGDGCGC@?$AAA?$AAd?$AAa?$AAp?$AAt?$AAe?$AAr?$AA?5?$AAb?$AAo?$AAo?$AAt?$AA?5?$AAt?$AAi?$AAm?$AAe?$AA?5?$AAo?$AAu?$AAt?$AA?$AA@FNODOBFM@ 00000001400260c0     arcinit.obj
 0001:000250f0       ??_C@_0CO@NHBGNFPE@?$CK?5Driver?5got?564?5bit?5FIB?5support?5@FNODOBFM@ 00000001400260f0     arcinit.obj
 0001:00025120       ??_C@_0DG@EECBHNEJ@?$CK?5Driver?5did?5not?5get?564?5bit?5FIB?5@FNODOBFM@ 0000000140026120     arcinit.obj
 0001:00025160       ??_C@_0CB@MHHOKKDH@?$CK?5Smart?5Array?5Based?5FW?5detected?6@FNODOBFM@ 0000000140026160     arcinit.obj
 0001:00025190       ??_C@_0CG@INGLDPEA@?$CK?5This?5is?5NOT?5a?5Smart?5Array?5Base@FNODOBFM@ 0000000140026190     arcinit.obj
 0001:000251c0       ??_C@_0DL@HHJHAPNC@?$CK?5StorPortGetDeviceBase?5failed?0?5@FNODOBFM@ 00000001400261c0     arcinit.obj
 0001:00025200       ??_C@_0FM@FAGAFMJI@?$CK?5StorPortGetDeviceBaseB1?5failed@FNODOBFM@ 0000000140026200     arcinit.obj
 0001:00025260       ??_C@_0FM@DFFNMELK@?$CK?5StorPortGetDeviceBaseB0?5failed@FNODOBFM@ 0000000140026260     arcinit.obj
 0001:000252c0       ??_C@_0DH@GMHBCEJM@?$CK?5GET_MINIARC_PROPERTIES?5fails?0?5@FNODOBFM@ 00000001400262c0     arcinit.obj
 0001:00025300       ??_C@_0CE@JIIGOPEA@?$CK?5This?5is?5a?5BEDROC?5inplementatio@FNODOBFM@ 0000000140026300     arcinit.obj
 0001:00025330       ??_C@_0CF@HKNELPOC@leaving?5MapDeviceBase?5?9?5rtnval?5?$DN@FNODOBFM@ 0000000140026330     arcinit.obj
 0001:00025360       ??_C@_0BG@LOIMFNHP@entering?5MatchPciIds?6?$AA@FNODOBFM@ 0000000140026360     arcinit.obj
 0001:00025380       ??_C@_08HNOCAICB@Adaptec?5?$AA@FNODOBFM@ 0000000140026380     arcinit.obj
 0001:00025390       ??_C@_0CC@GEDCIDMJ@leaving?5MatchPciIds?0?5rtnval?5?$DN?5?$CFx@FNODOBFM@ 0000000140026390     arcinit.obj
 0001:000253c0       ??_C@_0DG@MJCHKBMN@?$CK?5Calling?5CompleteBufferedReques@FNODOBFM@ 00000001400263c0     arcinit.obj
 0001:00025400       ??_C@_0HF@LDMKNKBL@?$CK?5Calling?5DequeueRawIoReadWriteR@FNODOBFM@ 0000000140026400     arcinit.obj
 0001:00025480       ??_C@_0DO@HDLNLCMA@?$CK?5Calling?5CompleteAllSortingQueu@FNODOBFM@ 0000000140026480     arcinit.obj
 0001:000254c0       ??_C@_0CG@EHFONFB@ReturningLocalOutstandingRequest@FNODOBFM@ 00000001400264c0     arcinit.obj
 0001:000254f0       ??_C@_0CL@CGNJGHDF@?$CK?5?$CFd?5outstanding?5IO?5left?5after?5c@FNODOBFM@ 00000001400264f0     arcinit.obj
 0001:00025520       ??_C@_0DI@FDADMONL@?$CK?5CleanHostSideRRQ?3?5Host?5RRQ?5cle@FNODOBFM@ 0000000140026520     arcinit.obj
 0001:00025560       ??_C@_0CF@IKJOOFLA@?$CK?5ResetAdapter?3?5Entering?5Routine@FNODOBFM@ 0000000140026560     arcinit.obj
 0001:00025590       ??_C@_0FI@OABPGHMC@?$CK?5ResetAdapter?3?5FW?5is?5processing@FNODOBFM@ 0000000140026590     arcinit.obj
 0001:000255f0       ??_C@_0DK@DMNFFNOF@?$CK?5ResetAdapter?3?5OS?5calls?5ResetAd@FNODOBFM@ 00000001400265f0     arcinit.obj
 0001:00025630       ??_C@_0CF@DGMKAPOJ@?$CK?5ResetAdapter?3?5BlinkLed?5Code?3?50@FNODOBFM@ 0000000140026630     arcinit.obj
 0001:00025660       ??_C@_0CL@MJAGNJPB@?$CK?5ResetAdapter?3?5IOP?5RESET?5due?5to@FNODOBFM@ 0000000140026660     arcinit.obj
 0001:00025690       ??_C@_0DG@CLNGJPOA@?$CK?5ResetAdapter?3?5SendSynchFib?5fai@FNODOBFM@ 0000000140026690     arcinit.obj
 0001:000256d0       ??_C@_0FF@JLPFKNGK@?$CK?5ResetAdapter?3?5There?5is?5a?5pendi@FNODOBFM@ 00000001400266d0     arcinit.obj
 0001:00025730       ??_C@_0EC@MMLNJELN@?$CK?5ResetAdapter?3?5set?5TriggerIOPRe@FNODOBFM@ 0000000140026730     arcinit.obj
 0001:00025780       ??_C@_0EH@BGKKNIMJ@?$CK?5ResetAdapter?3?5synch?5command?5Re@FNODOBFM@ 0000000140026780     arcinit.obj
 0001:000257d0       ??_C@_0EE@KPCKIKGP@?$CK?5ResetAdapter?3?5AdapterIsAlive?5r@FNODOBFM@ 00000001400267d0     arcinit.obj
 0001:00025820       ??_C@_0DN@OJOIDCGM@?$CK?5ResetAdapter?3?5leaving?5Routine?5@FNODOBFM@ 0000000140026820     arcinit.obj
 0001:00025860       ??_C@_0DN@MKLLHNDH@?$CK?5ResetAdapter?3?5IOP?5RESET?5due?5to@FNODOBFM@ 0000000140026860     arcinit.obj
 0001:000258a0       ??_C@_0DA@IHJFMKGH@?$CK?5ResetAdapter?3?5IOP?5RESET?5due?5to@FNODOBFM@ 00000001400268a0     arcinit.obj
 0001:000258d0       ??_C@_0FJ@HDBMDLNL@?$CK?5ResetAdapter?3?5RAID?5volume?5?$CFd?5r@FNODOBFM@ 00000001400268d0     arcinit.obj
 0001:00025930       ??_C@_0DC@DFLLLKCM@?$CK?5ResetAdapter?3?5IOP_RESET_FW_FIB@FNODOBFM@ 0000000140026930     arcinit.obj
 0001:00025970       ??_C@_0DM@IMELCPEN@?$CK?5ResetAdapter?3?5Failed?5to?5send?5I@FNODOBFM@ 0000000140026970     arcinit.obj
 0001:000259b0       ??_C@_0EG@FKMCGCCN@?$CK?5ResetAdapter?3?5IOP?5RESET?5due?5to@FNODOBFM@ 00000001400269b0     arcinit.obj
 0001:00025a00       ??_C@_0DE@IDNFNJBF@?$CK?5ResetAdapter?3?5NO?5lun?5reset?5cou@FNODOBFM@ 0000000140026a00     arcinit.obj
 0001:00025a40       ??_C@_0DM@KJNOMFJC@?$CK?5ResetAdapter?3?5leaving?5Routine?0@FNODOBFM@ 0000000140026a40     arcinit.obj
 0001:00025a80       ??_C@_0EK@OOPLAGOO@?$CK?5ResetAdapter?3?5set?5timer?5to?5che@FNODOBFM@ 0000000140026a80     arcinit.obj
 0001:00025ad0       ??_C@_0DM@LMPLKKMJ@?$CK?5ResetAdapter?3?5leaving?5Routine?5@FNODOBFM@ 0000000140026ad0     arcinit.obj
 0001:00025b10       ??_C@_0EJ@DNGMPOBO@?$CK?5ResetAdapter?3?5HWSoftReset?5leav@FNODOBFM@ 0000000140026b10     arcinit.obj
 0001:00025b60       ??_C@_0CJ@PCBCCJEM@?$DMHW?$DOTD?$AI?$AA?$AA?$AA?$AA?$AA?$AA?$AA?$AA?$AADW?$AA?$AADV?$BK?$AA?$AA?$AA?$AA?$AA?$AA?$AA?$AA?$AA@FNODOBFM@ 0000000140026b60     arcinit.obj
 0001:00025b90       ??_C@_0BP@BFNIMKLC@?$CK?5SetFwTime?3?5Time?5sent?5failed?6?$AA@FNODOBFM@ 0000000140026b90     arcinit.obj
 0001:00025bb0       ??_C@_0BL@IIHDOJJO@?$CK?5Time?3?5?$CFd?4?$CFd?4?$CFd?5?$CFd?3?$CFd?3?$CFd?6?$AA@FNODOBFM@ 0000000140026bb0     arcinit.obj
 0001:00025bd0       ??_C@_0BG@NCOEMLFM@?$CK?5Driver?5version?5?$CFs?5?6?$AA@FNODOBFM@ 0000000140026bd0     arcinit.obj
 0001:00025bf0       ??_C@_0CF@KGAABJAP@?$CK?5SetFwTime?3?5Time?5sent?5successfu@FNODOBFM@ 0000000140026bf0     arcinit.obj
 0001:00025c20       ??_C@_0DB@DBHKEEOM@?$CK?5SendWellnessCommand?3?5Wellness?5@FNODOBFM@ 0000000140026c20     arcinit.obj
 0001:00025c60       ??_C@_0DG@CHJDHKJC@?$CK?5SendWellnessCommand?3?5Wellness?5@FNODOBFM@ 0000000140026c60     arcinit.obj
 0001:00025ca0       ??_C@_0N@GDIDOMEJ@?$DMHW?$DOPS?$AC?$AA?$AA?$AAZZ?$AA@FNODOBFM@ 0000000140026ca0     arcinit.obj
 0001:00025cb0       ??_C@_0CM@KDDJKBII@?$CK?5SetPciSlotNumber?3?5Update?5PCI?5S@FNODOBFM@ 0000000140026cb0     arcinit.obj
 0001:00025ce0       ??_C@_0BL@CAAHKIPO@?$CK?5PCI?5Slot?5Number?5Set?5?$CFx?5?6?$AA@FNODOBFM@ 0000000140026ce0     arcinit.obj
 0001:00025d00       ??_C@_0DB@KLKDBGPC@?$CK?5current?5ElapsedTime?5is?5?$CFx?4?5Dri@FNODOBFM@ 0000000140026d00     arcinit.obj
 0001:00025d40       ??_C@_0EE@NDLKAFLN@?$CK?5SetArcsasFwTime?3?5SendSyncFib?5F@FNODOBFM@ 0000000140026d40     arcinit.obj
 0001:00025d90       ??_C@_0DN@BMDNNOBN@?$CK?5GetThorHbaPhyDevInfo?3?5synch?5FI@FNODOBFM@ 0000000140026d90     arcinit.obj
 0001:00025dd0       ??_C@_0FG@PNEDCHMO@?$CK?5one?5dual?5port?5entry?5?$CIB?1T?1nexus@FNODOBFM@ 0000000140026dd0     arcinit.obj
 0001:00025e30       ??_C@_0EM@BKPAJHPD@?$CK?5One?5entry?5?$CIB?1T?1nexus?3?5?$CFd?1?$CFd?10x@FNODOBFM@ 0000000140026e30     arcinit.obj
 0001:00025e80       ??_C@_0BI@NKGGGHHE@?$CK?5?$CFd?5HBA?5devices?5found?6?$AA@FNODOBFM@ 0000000140026e80     arcinit.obj
 0001:00025ea0       ??_C@_0DD@PLCLGMJE@?$CK?5All?5HBA?5devices?8?5average?5Queue@FNODOBFM@ 0000000140026ea0     arcinit.obj
 0001:00025ee0       ??_C@_0BF@GFOGGOIF@GetThorHbaPhyDevInfo?$AA@FNODOBFM@ 0000000140026ee0     arcinit.obj
 0001:00025f00       ??_C@_0CL@OHPEFDNF@?$CK?5There?5is?5a?5synch?5SRB?5pending?0?5@FNODOBFM@ 0000000140026f00     arcinit.obj
 0001:00025f30       ??_C@_0DJ@HDKNIPML@?$CK?5Not?5a?5Thor?5product?5OR?5virtual?5@FNODOBFM@ 0000000140026f30     arcinit.obj
 0001:00025f70       ??_C@_1FE@JLJHJCGF@?$AAA?$AAr?$AAr?$AAa?$AAy?$AA?5?$AAm?$AAi?$AAg?$AAr?$AAa?$AAt?$AAi?$AAo?$AAn?$AA?1?$AAe?$AAx?$AAp?$AAa?$AAn?$AAs?$AAi?$AAo?$AAn?$AA?5?$AAc?$AAo?$AAm?$AAp?$AAl?$AAe@FNODOBFM@ 0000000140026f70     arcinit.obj
 0001:00025fd0       ??_C@_1CK@DJNKNDAB@?$AAR?$AAa?$AAw?$AA?5?$AAD?$AAr?$AAi?$AAv?$AAe?$AA?5?$AAr?$AAe?$AAm?$AAo?$AAv?$AAe?$AAd?$AA?0?$AA?5?$AA?$CD?$AA?$AA@FNODOBFM@ 0000000140026fd0     arcinit.obj
 0001:00026000       ??_C@_1DG@JPPGPNNE@?$AAN?$AAa?$AAt?$AAi?$AAv?$AAe?$AA?5?$AAH?$AAB?$AAA?$AA?5?$AAd?$AAe?$AAv?$AAi?$AAc?$AAe?$AA?5?$AAi?$AAs?$AA?5?$AAa?$AAd?$AAd?$AAe?$AAd?$AA?$AA@FNODOBFM@ 0000000140027000     arcinit.obj
 0001:00026040       ??_C@_1DK@DMPEAPAK@?$AAN?$AAa?$AAt?$AAi?$AAv?$AAe?$AA?5?$AAH?$AAB?$AAA?$AA?5?$AAd?$AAe?$AAv?$AAi?$AAc?$AAe?$AA?5?$AAi?$AAs?$AA?5?$AAr?$AAe?$AAm?$AAo?$AAv?$AAe?$AAd?$AA?$AA@FNODOBFM@ 0000000140027040     arcinit.obj
 0001:00026080       ??_C@_1EO@PNKAKFGH@?$AAH?$AAa?$AAr?$AAd?$AAw?$AAa?$AAr?$AAe?$AA?5?$AAn?$AAo?$AAt?$AA?5?$AAp?$AAr?$AAe?$AAs?$AAe?$AAn?$AAt?$AA?9?$AA?5?$AAB?$AAa?$AAc?$AAk?$AAu?$AAp?$AA?5?$AAn?$AAo?$AAt@FNODOBFM@ 0000000140027080     arcinit.obj
 0001:000260d0       ??_C@_1CI@IELPCEHF@?$AAS?$AAu?$AAp?$AAe?$AAr?$AAc?$AAa?$AAp?$AA?5?$AAh?$AAe?$AAa?$AAl?$AAt?$AAh?$AA?5?$AAl?$AAo?$AAw?$AA?$AA@FNODOBFM@ 00000001400270d0     arcinit.obj
 0001:00026100       ??_C@_1CK@BAADJOPA@?$AAS?$AAu?$AAp?$AAe?$AAr?$AAc?$AAa?$AAp?$AA?5?$AAh?$AAe?$AAa?$AAl?$AAt?$AAh?$AA?5?$AA?5?$AAb?$AAa?$AAd?$AA?$AA@FNODOBFM@ 0000000140027100     arcinit.obj
 0001:00026130       ??_C@_1CA@DNJAAJKJ@?$AAC?$AAa?$AAc?$AAh?$AAe?$AA?5?$AAd?$AAa?$AAt?$AAa?$AA?5?$AAl?$AAo?$AAs?$AAs?$AA?$AA@FNODOBFM@ 0000000140027130     arcinit.obj
 0001:00026150       ??_C@_1DG@KILEJPC@?$AAT?$AAe?$AAm?$AAp?$AAe?$AAr?$AAa?$AAt?$AAu?$AAr?$AAe?$AA?5?$AAB?$AAa?$AAc?$AAk?$AA?5?$AAt?$AAo?$AA?5?$AAN?$AAo?$AAr?$AAm?$AAa?$AAl?$AA?$AA@FNODOBFM@ 0000000140027150     arcinit.obj
 0001:00026190       ??_C@_1DG@IHOODPDN@?$AAS?$AAu?$AAp?$AAe?$AAr?$AAc?$AAa?$AAp?$AA?5?$AAT?$AAe?$AAm?$AAp?$AAe?$AAr?$AAa?$AAt?$AAu?$AAr?$AAe?$AA?5?$AAA?$AAl?$AAe?$AAr?$AAt?$AA?$AA@FNODOBFM@ 0000000140027190     arcinit.obj
 0001:000261d0       ??_C@_1DK@KKLIINGO@?$AAS?$AAu?$AAp?$AAe?$AAr?$AAc?$AAa?$AAp?$AA?5?$AAT?$AAe?$AAm?$AAp?$AAe?$AAr?$AAa?$AAt?$AAu?$AAr?$AAe?$AA?5?$AAW?$AAa?$AAr?$AAn?$AAi?$AAn?$AAg?$AA?$AA@FNODOBFM@ 00000001400271d0     arcinit.obj
 0001:00026210       ??_C@_1DK@HENHBAOO@?$AAB?$AAa?$AAc?$AAk?$AAu?$AAp?$AA?5?$AAu?$AAn?$AAi?$AAt?$AA?5?$AAs?$AAe?$AAl?$AAf?$AA?9?$AAt?$AAe?$AAs?$AAt?$AA?5?$AAf?$AAa?$AAi?$AAl?$AAe?$AAd?$AA?$AA@FNODOBFM@ 0000000140027210     arcinit.obj
 0001:00026250       ??_C@_1DK@GKIHJFEC@?$AAF?$AAa?$AAt?$AAa?$AAl?$AA?5?$AAE?$AAr?$AAr?$AAo?$AAr?$AA?3?$AA?5?$AAB?$AAa?$AAc?$AAk?$AAu?$AAp?$AA?5?$AAd?$AAi?$AAs?$AAa?$AAb?$AAl?$AAe?$AAd?$AA?$AA@FNODOBFM@ 0000000140027250     arcinit.obj
 0001:00026290       ??_C@_1CO@DFMHCOAI@?$AAL?$AAo?$AAg?$AAi?$AAc?$AAa?$AAl?$AA?5?$AAD?$AAr?$AAi?$AAv?$AAe?$AA?5?$AAa?$AAd?$AAd?$AAe?$AAd?$AA?0?$AA?5?$AA?$CD?$AA?$AA@FNODOBFM@ 0000000140027290     arcinit.obj
 0001:000262c0       ??_C@_1DC@CMPCKFLI@?$AAL?$AAo?$AAg?$AAi?$AAc?$AAa?$AAl?$AA?5?$AAD?$AAr?$AAi?$AAv?$AAe?$AA?5?$AAd?$AAe?$AAl?$AAe?$AAt?$AAe?$AAd?$AA?0?$AA?5?$AA?$CD?$AA?$AA@FNODOBFM@ 00000001400272c0     arcinit.obj
 0001:00026300       ??_C@_1CI@JDGBIDGK@?$AAA?$AA?5?$AAn?$AAe?$AAw?$AA?5?$AAJ?$AAB?$AAO?$AAD?$AA?5?$AAi?$AAs?$AA?5?$AAa?$AAd?$AAd?$AAe?$AAd?$AA?$AA@FNODOBFM@ 0000000140027300     arcinit.obj
 0001:00026330       ??_C@_1CE@CICPDMOD@?$AAA?$AA?5?$AAJ?$AAB?$AAO?$AAD?$AA?5?$AAi?$AAs?$AA?5?$AAd?$AAe?$AAl?$AAe?$AAt?$AAe?$AAd?$AA?$AA@FNODOBFM@ 0000000140027330     arcinit.obj
 0001:00026360       ??_C@_1DI@CCPBOJAM@?$AAL?$AAu?$AAn?$AA?5?$AAR?$AAe?$AAs?$AAe?$AAt?$AA?5?$AAt?$AAh?$AAr?$AAe?$AAs?$AAh?$AAo?$AAl?$AAd?$AA?5?$AAr?$AAe?$AAa?$AAc?$AAh?$AAe?$AAd?$AA?$AA@FNODOBFM@ 0000000140027360     arcinit.obj
 0001:000263a0       ??_C@_1DG@OJKKJGHC@?$AAA?$AAd?$AAa?$AAp?$AAt?$AAe?$AAr?$AA?5?$AAa?$AAl?$AAi?$AAv?$AAe?$AA?5?$AAr?$AAe?$AAt?$AAu?$AAr?$AAn?$AA?5?$AAf?$AAa?$AAl?$AAs?$AAe?$AA?$AA@FNODOBFM@ 00000001400273a0     arcinit.obj
 0001:000263e0       ??_C@_1FC@MIPJHMMM@?$AAR?$AAe?$AAq?$AAu?$AAe?$AAs?$AAt?$AAA?$AAd?$AAa?$AAp?$AAt?$AAe?$AAr?$AAI?$AAn?$AAf?$AAo?$AA?5?$AAs?$AAy?$AAn?$AAc?$AAh?$AA?5?$AAc?$AAo?$AAm?$AAm?$AAa?$AAn?$AAd@FNODOBFM@ 00000001400273e0     arcinit.obj
 0001:00026440       ??_C@_1DC@FGMGNGA@?$AAF?$AAW?$AA?5?$AAK?$AAe?$AAr?$AAn?$AAe?$AAl?$AA?5?$AAP?$AAa?$AAn?$AAi?$AAc?$AA?5?$AAd?$AAe?$AAt?$AAe?$AAc?$AAt?$AAe?$AAd?$AA?$AA@FNODOBFM@ 0000000140027440     arcinit.obj
 0001:00026480       ??_C@_1CA@BBEOIBOD@?$AAU?$AAn?$AAd?$AAe?$AAf?$AAi?$AAn?$AAe?$AAd?$AA?5?$AAE?$AAv?$AAe?$AAn?$AAt?$AA?$AA@FNODOBFM@ 0000000140027480     arcinit.obj
 0001:000264a0       ??_C@_1EG@MMOHKHFO@?$AAC?$AAT?$AA_?$AAC?$AAO?$AAN?$AAF?$AAI?$AAG?$AA_?$AAS?$AAT?$AAA?$AAT?$AAU?$AAS?$AA_?$AAR?$AAE?$AAA?$AAD?$AAY?$AA?$CI?$AA?5?$AA?5?$AA?5?$AA?$CJ?$AA?5?$AAF?$AAa?$AAi?$AAl@FNODOBFM@ 00000001400274a0     arcinit.obj
 0001:000264f0       ??_C@_1EC@LINPOIBA@?$AAC?$AAT?$AA_?$AAG?$AAE?$AAT?$AA_?$AAC?$AAO?$AAN?$AAF?$AAI?$AAG?$AA_?$AAS?$AAT?$AAA?$AAT?$AAU?$AAS?$AA?$CI?$AA?5?$AA?5?$AA?5?$AA?$CJ?$AA?5?$AAF?$AAa?$AAi?$AAl?$AAe?$AAd@FNODOBFM@ 00000001400274f0     arcinit.obj
 0001:00026540       ??_C@_1DI@OLCGHNCB@?$AAC?$AAT?$AA_?$AAC?$AAO?$AAM?$AAM?$AAI?$AAT?$AA_?$AAC?$AAO?$AAN?$AAF?$AAI?$AAG?$AA?$CI?$AA?5?$AA?5?$AA?5?$AA?$CJ?$AAF?$AAa?$AAi?$AAl?$AAe?$AAd?$AA?$AA@FNODOBFM@ 0000000140027540     arcinit.obj
 0001:00026580       ??_C@_1FA@NIJNEMHE@?$AAA?$AAD?$AAA?$AAP?$AAT?$AAE?$AAR?$AA_?$AAI?$AAN?$AAI?$AAT?$AA_?$AAS?$AAT?$AAR?$AAU?$AAC?$AAT?$AA_?$AAR?$AAE?$AAV?$AAI?$AAS?$AAI?$AAO?$AAN?$AA?$CI?$AA?5?$AA?5?$AA?$CJ@FNODOBFM@ 0000000140027580     arcinit.obj
 0001:000265d0       ??_C@_1DM@EFGMNBLE@?$AAV?$AAM?$AA_?$AAC?$AAo?$AAn?$AAt?$AAa?$AAi?$AAn?$AAe?$AAr?$AAC?$AAo?$AAn?$AAf?$AAi?$AAg?$AA?$CI?$AA?5?$AA?5?$AA?$CJ?$AA?5?$AAF?$AAa?$AAi?$AAl?$AAe?$AAd?$AA?$AA@FNODOBFM@ 00000001400275d0     arcinit.obj
 0001:00026610       ??_C@_1DC@PCLINFGL@?$AAT?$AAi?$AAm?$AAe?$AAd?$AAo?$AAu?$AAt?$AA?0?$AA?5?$AAI?$AAn?$AAi?$AAt?$AA?5?$AAS?$AAt?$AAa?$AAg?$AAe?$AA?5?$AA?$CD?$AA?5?$AA?5?$AA?$AA@FNODOBFM@ 0000000140027610     arcinit.obj
 0001:00026650       ??_C@_1FE@PCKFJNFD@?$AAR?$AAe?$AAs?$AAe?$AAt?$AA?5?$AAf?$AAr?$AAo?$AAm?$AA?5?$AAO?$AAS?$AA?3?$AAp?$AAa?$AAt?$AAh?$AA?5?$AA?$CD?$AA?5?$AA?5?$AA?0?$AAo?$AAu?$AAt?$AAs?$AAt?$AAa?$AAn?$AAd?$AAi@FNODOBFM@ 0000000140027650     arcinit.obj
 0001:000266b0       ??_C@_1FC@CLHIPIHG@?$AAG?$AAo?$AAt?$AA?5?$AAL?$AAU?$AAN?$AA?5?$AAR?$AAE?$AAS?$AAE?$AAT?$AA?5?$AAf?$AAo?$AAr?$AA?5?$AAp?$AAa?$AAt?$AAh?$AA?5?$AA?$CD?$AA?5?$AA?5?$AA?0?$AA?5?$AAt?$AAa?$AAr?$AAg@FNODOBFM@ 00000001400276b0     arcinit.obj
 0001:00026710       ??_C@_1FI@HJHKOPPE@?$AAG?$AAo?$AAt?$AA?5?$AAT?$AAa?$AAr?$AAg?$AAe?$AAt?$AA?5?$AAR?$AAE?$AAS?$AAE?$AAT?$AA?5?$AAf?$AAo?$AAr?$AA?5?$AAp?$AAa?$AAt?$AAh?$AA?5?$AA?$CD?$AA?5?$AA?5?$AA?0?$AA?5?$AAt@FNODOBFM@ 0000000140027710     arcinit.obj
 0001:00026770       ??_C@_1EC@DEFLMBHE@?$AAI?$AAO?$AAP?$AA?5?$AAR?$AAE?$AAS?$AAE?$AAT?$AA?5?$AAb?$AAe?$AAc?$AAa?$AAu?$AAs?$AAe?$AA?5?$AAo?$AAf?$AA?5?$AAF?$AAW?$AA?5?$AAB?$AAl?$AAi?$AAn?$AAk?$AAL?$AAE?$AAD@FNODOBFM@ 0000000140027770     arcinit.obj
 0001:000267c0       ??_C@_1FA@GLBMBCFD@?$AAR?$AAe?$AAq?$AAu?$AAe?$AAs?$AAt?$AAA?$AAd?$AAa?$AAp?$AAt?$AAe?$AAr?$AAI?$AAn?$AAf?$AAo?$AA?5?$AAp?$AAe?$AAn?$AAd?$AAi?$AAn?$AAg?$AA?5?$AA?5?$AA?5?$AA?5?$AA?5?$AA?5@FNODOBFM@ 00000001400277c0     arcinit.obj
 0001:00026810       ??_C@_1EK@DPFNMDNI@?$AAI?$AAO?$AAP?$AAR?$AAE?$AAS?$AAE?$AAT?$AA?3?$AA?5?$AAR?$AAe?$AAq?$AAu?$AAe?$AAs?$AAt?$AAA?$AAd?$AAa?$AAp?$AAt?$AAe?$AAr?$AAI?$AAn?$AAf?$AAo?$AA?5?$AAt?$AAi?$AAm@FNODOBFM@ 0000000140027810     arcinit.obj
 0001:00026860       ??_C@_1EC@JONMGECF@?$AAR?$AAA?$AA?3?$AA?5?$AAA?$AAd?$AAa?$AAp?$AAt?$AAe?$AAr?$AAI?$AAs?$AAA?$AAl?$AAi?$AAv?$AAe?$AA?5?$AAr?$AAe?$AAt?$AAu?$AAr?$AAn?$AAs?$AA?5?$AAf?$AAa?$AAl?$AAs?$AAe@FNODOBFM@ 0000000140027860     arcinit.obj
 0001:000268b0       ??_C@_1EA@KMCOFCE@?$AAI?$AAO?$AAP?$AA?5?$AAR?$AAE?$AAS?$AAE?$AAT?$AA?5?$AAf?$AAo?$AAr?$AA?5?$AAS?$AAm?$AAa?$AAr?$AAt?$AAH?$AAB?$AAA?$AA?5?$AAp?$AAa?$AAt?$AAh?$AA?5?$AA?$CD?$AA?5?$AA?5?$AA?$AA@FNODOBFM@ 00000001400278b0     arcinit.obj
 0001:000268f0       ??_C@_1EK@EBJJOFBF@?$AAR?$AAE?$AAS?$AAE?$AAT?$AA?$CI?$AAc?$AAn?$AAt?$AA?$DO?$AA?$DN?$AA5?$AA?$CJ?$AA?3?$AA?5?$AAp?$AAa?$AAt?$AAh?$AA?5?$AA?$CD?$AA?5?$AA?5?$AA?0?$AA?5?$AAt?$AAa?$AAr?$AAg?$AAe?$AAt?$AA?5@FNODOBFM@ 00000001400278f0     arcinit.obj
 0001:00026940       ??_C@_1DA@EFMGPIMG@?$AAS?$AAO?$AAF?$AAT?$AA?5?$AAR?$AAE?$AAS?$AAE?$AAT?$AA?5?$AAI?$AAs?$AAs?$AAu?$AAe?$AAd?$AA?5?$AAt?$AAo?$AA?5?$AAF?$AAW?$AA?$AA@FNODOBFM@ 0000000140027940     arcinit.obj
 0001:00026970       ??_C@_1CO@GBDEAPLE@?$AAI?$AAO?$AAP?$AA?5?$AAR?$AAE?$AAS?$AAE?$AAT?$AA?5?$AAI?$AAs?$AAs?$AAu?$AAe?$AAd?$AA?5?$AAt?$AAo?$AA?5?$AAF?$AAW?$AA?$AA@FNODOBFM@ 0000000140027970     arcinit.obj
 0001:000269a0       ??_C@_1EI@KMCCOKBI@?$AAF?$AAW?$AA?5?$AAK?$AAE?$AAR?$AAN?$AAE?$AAL?$AA?5?$AAP?$AAA?$AAN?$AAI?$AAC?$AA?5?$AAD?$AAe?$AAt?$AAe?$AAc?$AAt?$AAe?$AAd?$AA?0?$AA?5?$AAB?$AAL?$AAE?$AAD?$AA?5?$AA?$CD@FNODOBFM@ 00000001400279a0     arcinit.obj
 0001:000269f0       ??_C@_1EK@GGMELPLN@?$AAF?$AAW?$AA?5?$AAN?$AAo?$AAt?$AA?5?$AAU?$AAp?$AA?5?$AA?$CG?$AA?5?$AAR?$AAu?$AAn?$AAn?$AAi?$AAn?$AAg?$AA?0?$AA?5?$AAB?$AAL?$AAE?$AAD?$AA?5?$AA0?$AAx?$AA?5?$AA?5?$AA?5?$AA?5@FNODOBFM@ 00000001400279f0     arcinit.obj
 0001:00026a40       ??_C@_0BG@HHGGAPDG@entering?5HWSoftReset?6?$AA@FNODOBFM@ 0000000140027a40     arcinit.obj
 0001:00026a60       ??_C@_0CB@CNHAMPIN@HwSoftReset?3?5Soft?5Reset?5Issued?4?6@FNODOBFM@ 0000000140027a60     arcinit.obj
 0001:00026a90       ??_C@_0DJ@CBPNBDFH@?$CK?5Set?5pInitStruct?9?$DONoOfMsiVector@FNODOBFM@ 0000000140027a90     arcinit.obj
 0001:00026ad0       ??_C@_0BG@FGBHCKJG@CompleteQueuedRequest?$AA@FNODOBFM@ 0000000140027ad0     cmddelivery.obj
 0001:00026af0       ??_C@_0DM@OFFCECMD@IN?5?$CFs?0?5WE?5ARE?5SEEING?5AIF?5FIB?4?5DO@FNODOBFM@ 0000000140027af0     cmddelivery.obj
 0001:00026b30       ??_C@_0L@ENAJINDB@Management?$AA@FNODOBFM@ 0000000140027b30     cmddelivery.obj
 0001:00026b40       ??_C@_0BB@JIADCMFJ@Array?5?5?5?5?5?5?5?5?5?5?5?$AA@FNODOBFM@ 0000000140027b40     cmddelivery.obj
 0001:00026b60       ??_C@_0BB@HJODFKJH@ARRAY?5?5?5?5?5?5?5?5?5?5?5?$AA@FNODOBFM@ 0000000140027b60     cmddelivery.obj
 0001:00026b80       ??_C@_0CB@IIENMBOI@?$CK?5Got?5an?5AIF?5in?5crash?5dump?5mode?6@FNODOBFM@ 0000000140027b80     cmddelivery.obj
 0001:00026bb0       ??_C@_0DO@NPBDNHBG@?$CK?5Should?5not?5be?5here?0?5we?5should?5@FNODOBFM@ 0000000140027bb0     cmddelivery.obj
 0001:00026bf0       ??_C@_0CO@PDPAIINM@?$CK?5PollSmartHBAFIBCompletion?3?5wai@FNODOBFM@ 0000000140027bf0     cmddelivery.obj
 0001:00026c20       ??_C@_0FC@DFPAPIBO@?$CK?5?9?9?5SCSIOP_START_STOP_UNIT?3?5Pat@FNODOBFM@ 0000000140027c20     cmddelivery.obj
 0001:00026c80       ??_C@_0CP@GPLNGCJB@?$CK?5?9?5Cannot?5start?1stop?5a?5unit?0?5er@FNODOBFM@ 0000000140027c80     cmddelivery.obj
 0001:00026cb0       ??_C@_0FM@ENJACBOF@?$CK?5SCSIOP_SYNCHRONIZE_CACHE?$CICDM?$CJ?3@FNODOBFM@ 0000000140027cb0     cmddelivery.obj
 0001:00026d10       ??_C@_0GA@MEOEEOJH@?$CK?5SCSIOP_SYNCHRONIZE_CACHE?$CICDM?$CJ?3@FNODOBFM@ 0000000140027d10     cmddelivery.obj
 0001:00026d70       ??_C@_0GO@DFFGFOPL@?$CK?$CK?57?124?5SendFib?3?5Line?5?$CFd?5Outstat@FNODOBFM@ 0000000140027d70     cmddelivery.obj
 0001:00026de0       ??_C@_0EI@ELGPOPDD@?$CK?$CK?57?124?5SendFib?3?5Line?5?$CFd?5MsgCap?$FL@FNODOBFM@ 0000000140027de0     cmddelivery.obj
 0001:00026e30       ??_C@_0GF@HHOGHLFF@?$CK?5This?5should?5not?5happen?4?5Srb?5po@FNODOBFM@ 0000000140027e30     cmddelivery.obj
 0001:00026ea0       ??_C@_0DC@IHNBNMNO@?$CK?$CK?5One?5FIB?5kidnapped?0?5FIB_Contex@FNODOBFM@ 0000000140027ea0     cmddelivery.obj
 0001:00026ee0       ??_C@_0HI@CALKOMHC@?$CK?5SendSynchFib?3?5There?5is?5a?5pendi@FNODOBFM@ 0000000140027ee0     cmddelivery.obj
 0001:00026f60       ??_C@_0FM@IHOMFPBM@?$CK?5In?5StartIo?0?5FW?5is?5still?5NOT?5ba@FNODOBFM@ 0000000140027f60     cmddelivery.obj
 0001:00026fc0       ??_C@_0CN@EPOHBMBH@?$CK?5path?5?$CFd?5target?5?$CFd?5reset?5counte@FNODOBFM@ 0000000140027fc0     cmddelivery.obj
 0001:00026ff0       ??_C@_0CB@KIAHGGON@?5RESET?5is?5for?5Smart?5HBA?5device?5?6@FNODOBFM@ 0000000140027ff0     cmddelivery.obj
 0001:00027020       ??_C@_0BP@PAHACOBL@?$CK?5Got?5path?5?$CFd?5target?5?$CFd?5reset?6?$AA@FNODOBFM@ 0000000140028020     cmddelivery.obj
 0001:00027040       ??_C@_0CC@BGHDODBG@?$CK?5SRB_FUNCTION_POWER?3?5action?3?5?$CFd@FNODOBFM@ 0000000140028040     cmddelivery.obj
 0001:00027070       ??_C@_0BP@DFKLHFDI@?$CK?5SRB_FUNCTION_POWER?3?5sleep?51?6?$AA@FNODOBFM@ 0000000140028070     cmddelivery.obj
 0001:00027090       ??_C@_0DL@PCKMOFFE@?$CK?5SRB_FUNCTION_POWER?3?5coming?5bac@FNODOBFM@ 0000000140028090     cmddelivery.obj
 0001:000270d0       ??_C@_0CG@NCNALCOB@?$CK?5SRB_FUNCTION_POWER?3?5going?5to?5S@FNODOBFM@ 00000001400280d0     cmddelivery.obj
 0001:00027100       ??_C@_0CA@IBGDOHDE@?$CK?5SRB_FUNCTION_POWER?3?5shutdown?6?$AA@FNODOBFM@ 0000000140028100     cmddelivery.obj
 0001:00027120       ??_C@_0CD@NOANDIPK@?$CK?5SRB_FUNCTION_POWER?3?5shutdownOf@FNODOBFM@ 0000000140028120     cmddelivery.obj
 0001:00027150       ??_C@_0BO@KPPCGIPP@?$CK?5SRB_FUNCTION_POWER?3?5reboot?6?$AA@FNODOBFM@ 0000000140028150     cmddelivery.obj
 0001:00027170       ??_C@_0BJ@NDPKABON@entering?5AdapterControl?6?$AA@FNODOBFM@ 0000000140028170     cmdproc.obj
 0001:00027190       ??_C@_0CF@FDIANAIH@?$CK?5?9?5AdapterControl?3?5ScsiStopAdap@FNODOBFM@ 0000000140028190     cmdproc.obj
 0001:000271c0       ??_C@_0FJ@DLLPOCIO@?$CK?5?9?5AdapterControl?3?5ScsiStopAdap@FNODOBFM@ 00000001400281c0     cmdproc.obj
 0001:00027220       ??_C@_0DK@JIECJOFO@?$CK?5Set?5pInitStruct?9?$DONoOfMsiVector@FNODOBFM@ 0000000140028220     cmdproc.obj
 0001:00027260       ??_C@_0HA@BIJAMPMG@?$CK?5?9?5AdapterControl?3?5ScsiSetBootC@FNODOBFM@ 0000000140028260     cmdproc.obj
 0001:000272d0       ??_C@_0DL@CMAPNHGC@?$CK?5?9?5AdapterControl?3?5ScsiSetBootC@FNODOBFM@ 00000001400282d0     cmdproc.obj
 0001:00027310       ??_C@_0DI@IPKKLNPP@?$CK?5?9?5AdapterControl?3?5ScsiSetBootC@FNODOBFM@ 0000000140028310     cmdproc.obj
 0001:00027350       ??_C@_0HE@CIFLMEO@?$CK?5?9?5AdapterControl?3?5ScsiSetRunni@FNODOBFM@ 0000000140028350     cmdproc.obj
 0001:000273d0       ??_C@_0CI@NDPGKLNN@?$CK?5?9?5AdapterControl?3?5ScsiRestartA@FNODOBFM@ 00000001400283d0     cmdproc.obj
 0001:00027400       ??_C@_0CM@CNGCOMHH@?$CK?5Before?5checking?5Adapter?5Health@FNODOBFM@ 0000000140028400     cmdproc.obj
 0001:00027430       ??_C@_0BF@GMFKAGLA@?$CK?$CK?5BlinLed?5Code?3?5?$CFx?6?$AA@FNODOBFM@ 0000000140028430     cmdproc.obj
 0001:00027450       ??_C@_1CE@ENBAPEOO@?$AAB?$AAl?$AAi?$AAn?$AAk?$AAL?$AAE?$AAD?$AA?5?$AAd?$AAe?$AAt?$AAe?$AAc?$AAt?$AAe?$AAd?$AA?$AA@FNODOBFM@ 0000000140028450     cmdproc.obj
 0001:00027480       ??_C@_0DM@EBNPFHJD@?$CK?5set?5timer?5to?5check?5the?5FW?5stat@FNODOBFM@ 0000000140028480     cmdproc.obj
 0001:000274c0       ??_C@_0CM@LGOLDMAP@?$CK?5leaving?5AdapterControl?5Routine@FNODOBFM@ 00000001400284c0     cmdproc.obj
 0001:000274f0       ??_C@_0EF@MIBINBLP@?$CK?5Hw?5Soft?5Reset?5Set?5Timer?0?5leavi@FNODOBFM@ 00000001400284f0     cmdproc.obj
 0001:00027540       ??_C@_0CG@MHIDKAIN@?$CK?5HW?5Soft?5Reset?0?5Set?5Timer?0?5line@FNODOBFM@ 0000000140028540     cmdproc.obj
 0001:00027570       ??_C@_0IF@DDPMHFDG@?$CK?5SMNormalModeInitAdapter?5failed@FNODOBFM@ 0000000140028570     cmdproc.obj
 0001:00027600       ??_C@_0IE@BILJPPDJ@?$CK?5SMNormalModeInitAdapter?5failed@FNODOBFM@ 0000000140028600     cmdproc.obj
 0001:00027690       ??_C@_0CO@CEANCDOF@?$CK?5?9?5AdapterControl?3?5Reset?5HostRR@FNODOBFM@ 0000000140028690     cmdproc.obj
 0001:000276c0       ??_C@_0CN@OHJICFOG@?$CK?5?9?5AdapterControl?3?5ScsiQuery?5wi@FNODOBFM@ 00000001400286c0     cmdproc.obj
 0001:000276f0       ??_C@_0DA@CMHNEFAA@?$CK?5?9?5AdapterControl?3?5ScsiQuery?5WI@FNODOBFM@ 00000001400286f0     cmdproc.obj
 0001:00027720       ??_C@_0DB@DKFDCCOB@?$CK?5Unsupported?5AdapterControl?5cod@FNODOBFM@ 0000000140028720     cmdproc.obj
 0001:00027760       ??_C@_0BI@MBKDPNLO@leaving?5AdapterControl?6?$AA@FNODOBFM@ 0000000140028760     cmdproc.obj
 0001:00027780       ??_C@_0EC@JJCHBELF@?$CI?$CFx?0?$CFx?0?$CFx?$CJ?0?5Function?5?$DN?5?$CFx?0?5Opcod@FNODOBFM@ 0000000140028780     cmdproc.obj
 0001:000277d0       ??_C@_0EG@JJEEJEDP@?$CI?$CFx?0?$CFx?0?$CFx?$CJ?0?5Function?5?$DN?5?$CFx?0?5Opcod@FNODOBFM@ 00000001400287d0     cmdproc.obj
 0001:00027820       ??_C@_0CO@NKBJPPMA@?$CK?5buildio?3?5LBA?5OUT?5OF?5RANGE?0?5sen@FNODOBFM@ 0000000140028820     cmdproc.obj
 0001:00027850       ??_C@_0FN@LKLFGDKL@?$CK?5buildio?3?5LBA?5OUT?5OF?5RANGE?0?5sen@FNODOBFM@ 0000000140028850     cmdproc.obj
 0001:000278b0       ??_C@_0FA@MOKLGDID@?$CK?5buildio?3?5LBA?5OUT?5OF?5RANGE?0?5sen@FNODOBFM@ 00000001400288b0     cmdproc.obj
 0001:00027900       ??_C@_0GA@IGOANHED@?$CK?5buildio?3?5LBA?5OUT?5OF?5RANGE?0?5sen@FNODOBFM@ 0000000140028900     cmdproc.obj
 0001:00027960       ??_C@_0DM@NPKIKBA@?$CK?5IOP?5RESET?5is?5done?5in?5ProcessIo@FNODOBFM@ 0000000140028960     ioctl.obj
 0001:000279a0       ??_C@_0DH@EIBEBELL@?$CK?5ProcessIoctl?3?5HWSoftReset?5leav@FNODOBFM@ 00000001400289a0     ioctl.obj
 0001:000279e0       ??_C@_0DL@IOLCNFHG@?$CK?5IOP?5RESET?5failed?5in?5ProcessIoc@FNODOBFM@ 00000001400289e0     ioctl.obj
 0001:00027a20       ??_C@_07MPDDHOMN@CSMIALL?$AA@FNODOBFM@ 0000000140028a20     ioctl.obj
 0001:00027a30       ??_C@_07OODOBGKD@CSMIARY?$AA@FNODOBFM@ 0000000140028a30     ioctl.obj
 0001:00027a40       ??_C@_07PAKBHMBE@CSMISAS?$AA@FNODOBFM@ 0000000140028a40     ioctl.obj
 0001:00027a50       ??_C@_07BHCKAAPP@CSMIPHY?$AA@FNODOBFM@ 0000000140028a50     ioctl.obj
 0001:00027a60       ??_C@_0ED@COAGKFGB@?$CK?5IOP?5RESET?5is?5in?5progress?4?5Reje@FNODOBFM@ 0000000140028a60     ioctl.obj
 0001:00027ab0       ??_C@_0CF@JOCBDLKJ@?$CK?5Allocate?5big?5IOCTL?5buffer?5fail@FNODOBFM@ 0000000140028ab0     ioctl.obj
 0001:00027ae0       ??_C@_0DF@CHPLNPBM@?$CK?5ProcessIoctl?3?5Internal?5Print?5B@FNODOBFM@ 0000000140028ae0     ioctl.obj
 0001:00027b20       ??_C@_0CE@NGAHOGLJ@?$CK?5ProcessIoctl?3?5private?5cdb?8s?5he@FNODOBFM@ 0000000140028b20     ioctl.obj
 0001:00027b50       ??_C@_0CH@HPKPAOCF@?$CK?5ProcessIoctl?3?5DBG_IO_TRACE?5fla@FNODOBFM@ 0000000140028b50     ioctl.obj
 0001:00027b80       ??_C@_0CK@OFFABCEM@?$CK?5ProcessIoctl?3?5DBG_IOCTL_TRACE?5@FNODOBFM@ 0000000140028b80     ioctl.obj
 0001:00027bb0       ??_C@_0CM@CGIIOCGI@?$CK?5ProcessIoctl?3?5DBG_CLUSTER_TRAC@FNODOBFM@ 0000000140028bb0     ioctl.obj
 0001:00027be0       ??_C@_0CI@LPOJHEHM@?$CK?5ProcessIoctl?3?5DBG_ISR_TRACE?5fl@FNODOBFM@ 0000000140028be0     ioctl.obj
 0001:00027c10       ??_C@_0DC@NOLFHCLF@?$CK?5ProcessIoctl?3?5DBG_IO_FUNC_ENTR@FNODOBFM@ 0000000140028c10     ioctl.obj
 0001:00027c50       ??_C@_0DE@PFEFFOBG@?$CK?5ProcessIoctl?3?5DBG_INIT_FUNC_EN@FNODOBFM@ 0000000140028c50     ioctl.obj
 0001:00027c90       ??_C@_0DF@DPLBBPBM@?$CK?5ProcessIoctl?3?5DBG_IOCTL_FUNC_E@FNODOBFM@ 0000000140028c90     ioctl.obj
 0001:00027cd0       ??_C@_0CL@GAIHEBC@?$CK?5ProcessIoctl?3?5DBG_IO_TRACE?5fla@FNODOBFM@ 0000000140028cd0     ioctl.obj
 0001:00027d00       ??_C@_0CO@NGOEBBKH@?$CK?5ProcessIoctl?3?5DBG_IOCTL_TRACE?5@FNODOBFM@ 0000000140028d00     ioctl.obj
 0001:00027d30       ??_C@_0DA@HPMIGAD@?$CK?5ProcessIoctl?3?5DBG_CLUSTER_TRAC@FNODOBFM@ 0000000140028d30     ioctl.obj
 0001:00027d60       ??_C@_0CM@NECMPDIP@?$CK?5ProcessIoctl?3?5DBG_ISR_TRACE?5fl@FNODOBFM@ 0000000140028d60     ioctl.obj
 0001:00027d90       ??_C@_0DG@PHFPGNCH@?$CK?5ProcessIoctl?3?5DBG_IO_FUNC_ENTR@FNODOBFM@ 0000000140028d90     ioctl.obj
 0001:00027dd0       ??_C@_0DI@CBNGHMLF@?$CK?5ProcessIoctl?3?5DBG_INIT_FUNC_EN@FNODOBFM@ 0000000140028dd0     ioctl.obj
 0001:00027e10       ??_C@_0DJ@DEFCHEDB@?$CK?5ProcessIoctl?3?5DBG_IOCTL_FUNC_E@FNODOBFM@ 0000000140028e10     ioctl.obj
 0001:00027e50       ??_C@_0CC@ELKJFKAD@?$CK?5ProcessIoctl?3?5DebugFlags?3?50x?$CFx@FNODOBFM@ 0000000140028e50     ioctl.obj
 0001:00027e80       ??_C@_0DI@PNEPHAGL@?$CK?5Set?5pInitStruct?9?$DONoOfMsiVector@FNODOBFM@ 0000000140028e80     ioctl.obj
 0001:00027ec0       ??_C@_0DF@KDDHBOCK@?$CK?5when?5back?5from?5IOP_RESET?0?5we?5w@FNODOBFM@ 0000000140028ec0     ioctl.obj
 0001:00027f00       ??_C@_0DO@IBFHJCIJ@?$CK?5IOP?5RESET?5is?5done?5in?5ProcessIo@FNODOBFM@ 0000000140028f00     ioctl.obj
 0001:00027f40       ??_C@_0DN@EJCEJBIF@?$CK?5IOP?5RESET?5failed?5in?5ProcessIoc@FNODOBFM@ 0000000140028f40     ioctl.obj
 0001:00027f80       ??_C@_0CF@GENCHGED@?$CK?5ProcessIoctl?3?5coalescing?5disab@FNODOBFM@ 0000000140028f80     ioctl.obj
 0001:00027fb0       ??_C@_0CE@KOEFFOB@?$CK?5ProcessIoctl?3?5coalescing?5enabl@FNODOBFM@ 0000000140028fb0     ioctl.obj
 0001:00027fe0       ??_C@_0GG@KLCLOEBM@?$CK?5ProcessIoctl?3?5Get?5a?5request?5fo@FNODOBFM@ 0000000140028fe0     ioctl.obj
 0001:00028050       ??_C@_0IA@OEPDMML@?$CK?5ProcessIoctl?3?5Get?5a?5request?5fo@FNODOBFM@ 0000000140029050     ioctl.obj
 0001:000280d0       ??_C@_0GG@JMGDPGEE@?$CK?5ProcessIoctl?3?5Get?5a?5request?5fo@FNODOBFM@ 00000001400290d0     ioctl.obj
 0001:00028140       ??_C@_0IA@HMGAPIGO@?$CK?5ProcessIoctl?3?5Get?5a?5request?5fo@FNODOBFM@ 0000000140029140     ioctl.obj
 0001:000281c0       ??_C@_0DH@GFOJOHEG@?$CK?5ProcessIoctl?3?5TTYPE_CHANGE_IO_@FNODOBFM@ 00000001400291c0     ioctl.obj
 0001:00028200       ??_C@_0CN@FFFLABJM@?$CK?5ProcessIoctl?3?5AIF?5commands?5pri@FNODOBFM@ 0000000140029200     ioctl.obj
 0001:00028230       ??_C@_0CO@EKDJMEJG@?$CK?5ProcessIoctl?3?5AIF?5commands?5pri@FNODOBFM@ 0000000140029230     ioctl.obj
 0001:00028260       ??_C@_0CP@DNDOBHJJ@?$CK?5ProcessIoctl?3?5synch?5commands?5p@FNODOBFM@ 0000000140029260     ioctl.obj
 0001:00028290       ??_C@_0DA@DKDLFFAP@?$CK?5ProcessIoctl?3?5synch?5commands?5p@FNODOBFM@ 0000000140029290     ioctl.obj
 0001:000282c0       ??_C@_0DD@OCMBIILM@?$CK?5ProcessIoctl?3?5RUN_CODE_IN_SPEC@FNODOBFM@ 00000001400292c0     ioctl.obj
 0001:00028300       ??_C@_0FD@PBJMMHDI@?$CK?5ProcessIoctl?3?5RUN_CODE_IN_SPEC@FNODOBFM@ 0000000140029300     ioctl.obj
 0001:00028360       ??_C@_0EG@IJGFKELB@?$CK?5ProcessIoctl?3?5bus?$DN?$CFd?0?5target?$DN?$CF@FNODOBFM@ 0000000140029360     ioctl.obj
 0001:000283b0       ??_C@_0GB@LAAKBHJK@?$CK?5ProcessIoctl?3?5wrong?5parameters@FNODOBFM@ 00000001400293b0     ioctl.obj
 0001:00028420       ??_C@_0DA@LCPJHFEI@?$CK?5ProcessIoctl?3?5Max?5Data?5Transfe@FNODOBFM@ 0000000140029420     ioctl.obj
 0001:00028450       ??_C@_0CE@DJCKDJAF@?$CK?5ProcessIoctl?3?5Max?5SG?5items?3?50x@FNODOBFM@ 0000000140029450     ioctl.obj
 0001:00028480       ??_C@_0BF@JHMLOOKE@?$CK?5outstanding?5IO?3?$CFd?6?$AA@FNODOBFM@ 0000000140029480     ioctl.obj
 0001:000284a0       ??_C@_0BL@BDGJNAIM@?$CK?5Sorting?5Q?4?5CalledCnt?3?$CFd?6?$AA@FNODOBFM@ 00000001400294a0     ioctl.obj
 0001:000284c0       ??_C@_0BO@FHMIKIJB@?$CK?5Sorting?5Q?4?5OverlapCase1?3?$CFd?6?$AA@FNODOBFM@ 00000001400294c0     ioctl.obj
 0001:000284e0       ??_C@_0BO@NBFMNKDP@?$CK?5Sorting?5Q?4?5OverlapCase2?3?$CFd?6?$AA@FNODOBFM@ 00000001400294e0     ioctl.obj
 0001:00028500       ??_C@_0CK@EPAOGNLF@?$CK?5ProcessIoctl?3?5BUILDIO?5LOOPBACK@FNODOBFM@ 0000000140029500     ioctl.obj
 0001:00028530       ??_C@_0CK@DADBMBLL@?$CK?5ProcessIoctl?3?5STARTIO?5LOOPBACK@FNODOBFM@ 0000000140029530     ioctl.obj
 0001:00028560       ??_C@_0CK@BMBGJMJA@?$CK?5ProcessIoctl?3?5PUSHFIB?5LOOPBACK@FNODOBFM@ 0000000140029560     ioctl.obj
 0001:00028590       ??_C@_0CL@DANMEPHG@?$CK?5ProcessIoctl?3?5BUILDIO?5LOOPBACK@FNODOBFM@ 0000000140029590     ioctl.obj
 0001:000285c0       ??_C@_0CL@NHBLFNNN@?$CK?5ProcessIoctl?3?5STARTIO?5LOOPBACK@FNODOBFM@ 00000001400295c0     ioctl.obj
 0001:000285f0       ??_C@_0CL@HLILIDMA@?$CK?5ProcessIoctl?3?5PUSHFIB?5LOOPBACK@FNODOBFM@ 00000001400295f0     ioctl.obj
 0001:00028620       ??_C@_0DB@MDNCKDFE@?$CK?5ProcessIoctl?3?5Simulate?5SCSI?5sm@FNODOBFM@ 0000000140029620     ioctl.obj
 0001:00028660       ??_C@_0EC@KMBGJBEG@?$CK?5ProcessIoctl?3?5Simulate?5FW?5Targ@FNODOBFM@ 0000000140029660     ioctl.obj
 0001:000286b0       ??_C@_0BI@COAKNOP@?$CK?5?9?5IOCTL?5MESSAGE?3?5?$CFs?5?6?$AA@FNODOBFM@ 00000001400296b0     ioctl.obj
 0001:000286d0       ??_C@_0BP@PHOOCPMJ@?$CK?5?9?5IOCTL?3?5FSAMPCTL_RESET_IOP?6?$AA@FNODOBFM@ 00000001400296d0     ioctl.obj
 0001:000286f0       ??_C@_0CE@ONNDCLIE@FSAMPCTL_RESET_IOP?5?3?5ResetFlag?5?$CF@FNODOBFM@ 00000001400296f0     ioctl.obj
 0001:00028720       ??_C@_0CM@ILCOJJDE@FSAMPCTL_RESET_IOP?3?5IOP?5Reset?5On@FNODOBFM@ 0000000140029720     ioctl.obj
 0001:00028750       ??_C@_0CP@PMFIDFBA@?$CK?5IOP?5RESET?5is?5done?5in?5ProcessIo@FNODOBFM@ 0000000140029750     ioctl.obj
 0001:00028780       ??_C@_0EB@EJNKCDGF@?$CK?5IOP?5RESET?5failed?5in?5ProcessIoc@FNODOBFM@ 0000000140029780     ioctl.obj
 0001:000287d0       ??_C@_0DA@ILCCCIHD@FSAMPCTL_RESET_IOP?3?5HW?5Soft?5Rese@FNODOBFM@ 00000001400297d0     ioctl.obj
 0001:00028800       ??_C@_0DI@EHOOKHPF@?$CK?5when?5back?5from?5HWSOFT_RESET?0?5w@FNODOBFM@ 0000000140029800     ioctl.obj
 0001:00028840       ??_C@_0DN@BHCOMBAH@?$CK?5set?5timer?5to?5check?5the?5FW?5stat@FNODOBFM@ 0000000140029840     ioctl.obj
 0001:00028880       ??_C@_0DD@GMMMAFI@?$CK?5HW?5SOFT?5RESET?5is?5done?5in?5Proce@FNODOBFM@ 0000000140029880     ioctl.obj
 0001:000288c0       ??_C@_0DJ@HKOHJJPL@HW?5SOFT?5RESET?5is?5not?5support?4?5In@FNODOBFM@ 00000001400298c0     ioctl.obj
 0001:00028900       ??_C@_0EM@EEFCGCAM@FSAMPCTL_RESET_IOP?3?5IOP?5Reset?5Fo@FNODOBFM@ 0000000140029900     ioctl.obj
 0001:00028950       ??_C@_0DC@MOKOJMEO@?$CK?5HW?5IOP?5RESET?5is?5done?5in?5Proces@FNODOBFM@ 0000000140029950     ioctl.obj
 0001:00028990       ??_C@_0EF@IPKPNMPC@?$CK?5HW?5SOFT?5RESET?5failed?5in?5Proces@FNODOBFM@ 0000000140029990     ioctl.obj
 0001:000289e0       ??_C@_0DP@HKHFJHOF@ProcessIoctl?5FSAMPCTL_RESET_IOP?0@FNODOBFM@ 00000001400299e0     ioctl.obj
 0001:00028a20       ??_C@_0L@BGLGDCOP@archba?4sys?$AA@FNODOBFM@ 0000000140029a20     ioctl.obj
 0001:00028a30       ??_C@_0CA@HJMENHI@Adaptec?5SAS?5HBA?5Storport?5Driver?$AA@FNODOBFM@ 0000000140029a30     ioctl.obj
 0001:00028a50       ??_C@_0DJ@MIENLJJJ@OMR?5value?5in?5Check?5Adapter?5Healt@FNODOBFM@ 0000000140029a50     comm.obj
 0001:00028a90       ??_C@_0DB@LCMFMKOG@?$CK?5Event?5array?5FULL?4?5Event?5?$CI?$CFd?$CJ?5n@FNODOBFM@ 0000000140029a90     comm.obj
 0001:00028ad0       ??_C@_0EJ@PCHGGBBF@?$CK?5ProcessAif?3?5request?5timer?5for?5@FNODOBFM@ 0000000140029ad0     comm.obj
 0001:00028b20       ??_C@_0BL@NHJOLJMJ@AIF?5EVENT?5?$CIThor?$CJ?3?5HotPlug?6?$AA@FNODOBFM@ 0000000140029b20     comm.obj
 0001:00028b40       ??_C@_0CD@EMEGIPDM@AIF?5EVENT?5?$CIThor?$CJ?3?5Hardware?5chang@FNODOBFM@ 0000000140029b40     comm.obj
 0001:00028b70       ??_C@_0DC@LGHJMKLE@AIF?5EVENT?5?$CIThor?$CJ?3?5Physical?5Devic@FNODOBFM@ 0000000140029b70     comm.obj
 0001:00028bb0       ??_C@_0DB@CEOPCOBC@AIF?5EVENT?5?$CIThor?$CJ?3?5Logical?5Device@FNODOBFM@ 0000000140029bb0     comm.obj
 0001:00028bf0       ??_C@_0DC@PEAKFMNI@AIF?5EVENT?5?$CIThor?$CJ?3?5FW?5IO?5bypass?5s@FNODOBFM@ 0000000140029bf0     comm.obj
 0001:00028c30       ??_C@_0DK@MABGHGOH@AIF?5EVENT?5?$CIThor?$CJ?3?5FW?5IO?5bypass?5c@FNODOBFM@ 0000000140029c30     comm.obj
 0001:00028c70       ??_C@_0CP@MLBBLAGJ@AIF?5EVENT?5?$CIThor?$CJ?3?5Not?5a?5recogniz@FNODOBFM@ 0000000140029c70     comm.obj
 0001:00028ca0       ??_C@_0DL@CJKFCOBN@?$CK?5ProcessAif?3?5request?5timer?5to?5s@FNODOBFM@ 0000000140029ca0     comm.obj
 0001:00028ce0       ??_C@_0CH@PCLLKGG@?$CK?5ProcessAif?3?5Physical?5Drives?5sc@FNODOBFM@ 0000000140029ce0     comm.obj
 0001:00028d10       ??_C@_0DK@NNFHFOND@?$CK?5ProcessAif?3?5request?5timer?5to?5s@FNODOBFM@ 0000000140029d10     comm.obj
 0001:00028d50       ??_C@_0CG@CDKKDOHL@?$CK?5ProcessAif?3?5Logical?5Drives?5sca@FNODOBFM@ 0000000140029d50     comm.obj
 0001:00028d80       ??_C@_0CM@GEHGCFFI@?$CK?5ProcessAif?3?5AIF?5cmd?3?5?$CFd?0?5AIF?5s@FNODOBFM@ 0000000140029d80     comm.obj
 0001:00028db0       ??_C@_0CJ@ELNMEDDG@AIF?5EVENT?3?5Container?5?$CD?$CFd?5Morph?5c@FNODOBFM@ 0000000140029db0     comm.obj
 0001:00028de0       ??_C@_0CF@GOGNODAJ@AIF?5EVENT?3?5a?5RAW?5device?5?$CD?$CFd?5remo@FNODOBFM@ 0000000140029de0     comm.obj
 0001:00028e10       ??_C@_0CL@PFPKJCEB@AIF?5EVENT?3?5AifEnNativeHBADeviceA@FNODOBFM@ 0000000140029e10     comm.obj
 0001:00028e40       ??_C@_0CO@KNHKMPNF@AIF?5EVENT?3?5AifEnNativeHBADeviceR@FNODOBFM@ 0000000140029e40     comm.obj
 0001:00028e70       ??_C@_0DD@GCBHPPGK@AIF?5EVENT?3?5Hardware?5not?5present?9@FNODOBFM@ 0000000140029e70     comm.obj
 0001:00028eb0       ??_C@_0EJ@OLDMFEFC@AIF?5EVENT?3?5Super?5cap?5health?5is?5l@FNODOBFM@ 0000000140029eb0     comm.obj
 0001:00028f00       ??_C@_0DM@BNKBKMII@AIF?5EVENT?3?5Super?5cap?5health?5is?5b@FNODOBFM@ 0000000140029f00     comm.obj
 0001:00028f40       ??_C@_0BM@DGCCGGOI@AIF?5EVENT?3?5Cache?5data?5loss?6?$AA@FNODOBFM@ 0000000140029f40     comm.obj
 0001:00028f60       ??_C@_0CH@EOEMJJE@AIF?5EVENT?3?5Temperature?5Back?5to?5N@FNODOBFM@ 0000000140029f60     comm.obj
 0001:00028f90       ??_C@_0EA@EGACBNC@AIF?5EVENT?3?5Temperature?5has?5cross@FNODOBFM@ 0000000140029f90     comm.obj
 0001:00028fd0       ??_C@_0ED@CGHEBKG@AIF?5EVENT?3?5Temperature?5is?5in?5the@FNODOBFM@ 0000000140029fd0     comm.obj
 0001:00029020       ??_C@_0CJ@JLLJHFCM@AIF?5EVENT?3?5Backup?5unit?5self?9test@FNODOBFM@ 000000014002a020     comm.obj
 0001:00029050       ??_C@_0CJ@NHDLILDM@AIF?5EVENT?3?5Fatal?5Error?3?5Backup?5d@FNODOBFM@ 000000014002a050     comm.obj
 0001:00029080       ??_C@_0CA@GLOIGEIG@AIF?5EVENT?3?5Container?5?$CD?$CFd?5added?6?$AA@FNODOBFM@ 000000014002a080     comm.obj
 0001:000290a0       ??_C@_0CC@IGLGEBDK@AIF?5EVENT?3?5Container?5?$CD?$CFd?5removed@FNODOBFM@ 000000014002a0a0     comm.obj
 0001:000290d0       ??_C@_0FE@GFLJPFDG@AIF?5EVENT?3?5AifEnEnclosureManagem@FNODOBFM@ 000000014002a0d0     comm.obj
 0001:00029130       ??_C@_0BJ@NJMLAEMO@AIF?5EVENT?3?5a?5JBOD?5added?6?$AA@FNODOBFM@ 000000014002a130     comm.obj
 0001:00029150       ??_C@_0BL@PDKEFHEM@AIF?5EVENT?3?5a?5JBOD?5removed?6?$AA@FNODOBFM@ 000000014002a150     comm.obj
 0001:00029170       ??_C@_0DO@DNJOKEFB@AIF?5EVENT?3?5AifCmdJobProgress?5for@FNODOBFM@ 000000014002a170     comm.obj
 0001:000291b0       ??_C@_0EM@MHLKFBIP@AIF?5EVENT?3?5AifCmdJobProgress?5for@FNODOBFM@ 000000014002a1b0     comm.obj
 0001:00029200       ??_C@_0EO@LMDDDIBO@?$CK?5RestoreBMIC15Srb?3?5QD?5limitatio@FNODOBFM@ 000000014002a200     comm.obj
 0001:00029250       ??_C@_0EI@IBBGKNJF@?$CK?5ProcessNormalFib?9Set?5QD?54?5HBA?5@FNODOBFM@ 000000014002a250     comm.obj
 0001:000292a0       ??_C@_0CG@IPLFJLPL@Smart?5HBA?5Scsi?5response?5Status?5?$DN@FNODOBFM@ 000000014002a2a0     comm.obj
 0001:000292d0       ??_C@_0DO@HNDDHFGA@?5HBA?5Error?5HBA_MODE_DISABLED?5Srb@FNODOBFM@ 000000014002a2d0     comm.obj
 0001:00029310       ??_C@_0DA@CPGPCCBA@?5HBA?5Error?5code?5?$CFx?5For?5Path?5ID?5?$CF@FNODOBFM@ 000000014002a310     comm.obj
 0001:00029340       ??_C@_0FA@CPHJLELC@?5HBA?5Error?5SCSI_COMPL_TRANSL_STA@FNODOBFM@ 000000014002a340     comm.obj
 0001:00029390       ??_C@_0FE@JFIIIBKF@?5HBA?5Error?5SCSI_COMPL_TRANSL_STA@FNODOBFM@ 000000014002a390     comm.obj
 0001:000293f0       ??_C@_0EO@DHIENLOG@?5HBA?5Error?3?5Length?5from?5OS?$CI0x?$CFx?$CJ@FNODOBFM@ 000000014002a3f0     comm.obj
 0001:00029440       ??_C@_0HP@ECKDIFKN@?5HBA?5Error?3?5hbaCmd?9?$DOdata_length?$CI@FNODOBFM@ 000000014002a440     comm.obj
 0001:000294c0       ??_C@_0FK@IBAGLEPN@?5HBA?5Error?5SCSI_COMPL_TRANSL_STA@FNODOBFM@ 000000014002a4c0     comm.obj
 0001:00029520       ??_C@_0FJ@DMCDLFNM@?5HBA?5Error?5SCSI_COMPL_TRANSL_STA@FNODOBFM@ 000000014002a520     comm.obj
 0001:00029580       ??_C@_0EP@JHLDIODO@?$CK?5NO?5ERROR?5handling?5for?5pHbaResp@FNODOBFM@ 000000014002a580     comm.obj
 0001:000295d0       ??_C@_0CG@PJJANG@TMF?5Function?5Completed?5Successfu@FNODOBFM@ 000000014002a5d0     comm.obj
 0001:00029600       ??_C@_0FJ@OIALMBME@?$CK?5NO?5ERROR?5handling?5for?5pHbaResp@FNODOBFM@ 000000014002a600     comm.obj
 0001:00029660       ??_C@_1BI@BHAHBMFJ@?$AAM?$AAo?$AAf?$AAR?$AAe?$AAs?$AAo?$AAu?$AAr?$AAc?$AAe?$AA?$AA@FNODOBFM@ 000000014002a660     wmi.obj
 0002:00000000       __imp_KeQueryPerformanceCounter 000000014002b000     hal:HAL.dll
 0002:00000008       \177HAL_NULL_THUNK_DATA    000000014002b008     hal:HAL.dll
 0002:00000010       __imp_RtlTimeToTimeFields  000000014002b010     ntoskrnl:ntoskrnl.exe
 0002:00000018       __imp_ExSystemTimeToLocalTime 000000014002b018     ntoskrnl:ntoskrnl.exe
 0002:00000020       \177ntoskrnl_NULL_THUNK_DATA 000000014002b020     ntoskrnl:ntoskrnl.exe
 0002:00000028       __imp_StorPortGetPhysicalAddress 000000014002b028     storport:storport.sys
 0002:00000030       __imp_StorPortPause        000000014002b030     storport:storport.sys
 0002:00000038       __imp_StorPortNotification 000000014002b038     storport:storport.sys
 0002:00000040       __imp_StorPortStallExecution 000000014002b040     storport:storport.sys
 0002:00000048       __imp_StorPortDebugPrint   000000014002b048     storport:storport.sys
 0002:00000050       __imp_StorPortExtendedFunction 000000014002b050     storport:storport.sys
 0002:00000058       __imp_StorPortGetDeviceBase 000000014002b058     storport:storport.sys
 0002:00000060       __imp_StorPortResume       000000014002b060     storport:storport.sys
 0002:00000068       __imp_StorPortInitialize   000000014002b068     storport:storport.sys
 0002:00000070       __imp_StorPortFreeDeviceBase 000000014002b070     storport:storport.sys
 0002:00000078       __imp_StorPortGetBusData   000000014002b078     storport:storport.sys
 0002:00000080       __imp_StorPortGetUncachedExtension 000000014002b080     storport:storport.sys
 0002:00000088       __imp_StorPortSetDeviceQueueDepth 000000014002b088     storport:storport.sys
 0002:00000090       __imp_StorPortQuerySystemTime 000000014002b090     storport:storport.sys
 0002:00000098       __imp_StorPortPauseDevice  000000014002b098     storport:storport.sys
 0002:000000a0       __imp_StorPortResumeDevice 000000014002b0a0     storport:storport.sys
 0002:000000a8       __imp_StorPortBusy         000000014002b0a8     storport:storport.sys
 0002:000000b0       __imp_StorPortGetScatterGatherList 000000014002b0b0     storport:storport.sys
 0002:000000b8       \177storport_NULL_THUNK_DATA 000000014002b0b8     storport:storport.sys
 0002:000000c0       __guard_check_icall_fptr   000000014002b0c0     BufferOverflowFastFailK:guard_support.obj
 0002:000000c8       __guard_dispatch_icall_fptr 000000014002b0c8     BufferOverflowFastFailK:guard_support.obj
 0002:000000d0       __guard_fids_table         000000014002b0d0     <linker-defined>
 0002:00000180       RevCompareTable            000000014002b180     revision.obj
 0002:00000280       RevCompareTableLength      000000014002b280     revision.obj
 0002:00000288       WPP_ThisDir_CTLGUID_archba 000000014002b288     arcdebug.obj
 0002:00000298       ??_C@_1O@IJPMNEG@?$AAa?$AAr?$AAc?$AAh?$AAb?$AAa?$AA?$AA@ 000000014002b298     arcdebug.obj
 0002:000002b0       ??_C@_1DKM@GBPEPNNL@?$AA?5?$AAM?$AAd?$AAD?$AAb?$AAg?$AAI?$AAn?$AAi?$AAt?$AA?5?$AAM?$AAd?$AAD?$AAb?$AAg?$AAP?$AAn?$AAp?$AA?5?$AAM?$AAd?$AAD?$AAb?$AAg?$AAP?$AAo?$AAw?$AAe?$AAr?$AA?5?$AAM@ 000000014002b2b0     arcdebug.obj
 0002:00000660       WPP_564d9f83b95836092d7383fb0050d933_Traceguids 000000014002b660     arcdebug.obj
 0002:00000670       ??_C@_08HNOCAICB@Adaptec?5?$AA@ 000000014002b670     archba.obj
 0002:0000067c       ??_C@_04ODJNANJC@9005?$AA@ 000000014002b67c     archba.obj
 0002:00000684       ??_C@_04EKJHPGNA@0285?$AA@ 000000014002b684     archba.obj
 0002:0000068c       ??_C@_04GBLKKFBD@0286?$AA@ 000000014002b68c     archba.obj
 0002:00000694       ??_C@_04PPDJIIJN@0288?$AA@ 000000014002b694     archba.obj
 0002:0000069c       ??_C@_04LPGNDNED@028b?$AA@ 000000014002b69c     archba.obj
 0002:000006a4       ??_C@_04KGHGAMAC@028c?$AA@ 000000014002b6a4     archba.obj
 0002:000006ac       ??_C@_04OJDHJKMF@028d?$AA@ 000000014002b6ac     archba.obj
 0002:000006b8       ??_C@_0BB@BOPAMEAE@ARC?9HBA?5?5?5?5?5?5?5?5?5?$AA@ 000000014002b6b8     archba.obj
 0002:000006cc       ??_C@_06DFBHEALI@AACAPI?$AA@ 000000014002b6cc     archba.obj
 0002:000006d8       ??_C@_1BK@EPHGJNJ@?$AAS?$AAc?$AAs?$AAi?$AAM?$AAi?$AAn?$AAi?$AAP?$AAo?$AAr?$AAt?$AA?$AA@ 000000014002b6d8     scsiwmi:wmilib.obj
 0002:00000740       _load_config_used          000000014002b740     BufferOverflowFastFailK:loadcfg.obj
 0003:00000000       pfnWppTraceMessage         000000014002d000     arcdebug.obj
 0003:00000008       WPP_GLOBAL_Control         000000014002d008     arcdebug.obj
 0003:00000040       gDebugFlags                000000014002d040     arcdebug.obj
 0003:00000050       gNativeModeAdapters        000000014002d050     archba.obj
 0003:00000380       gNumNativeModeAdapters     000000014002d380     archba.obj
 0003:00000384       gARCOEMFlags               000000014002d384     archba.obj
 0003:00000388       gARCProductId              000000014002d388     archba.obj
 0003:00000390       gARCApiId                  000000014002d390     archba.obj
 0003:000003a0       gARCSASRxSubsystemInfo     000000014002d3a0     archba.obj
 0003:000006b0       gARCSASRktSubsystemInfo    000000014002d6b0     archba.obj
 0003:00000720       gARCSASArkSubsystemInfo    000000014002d720     archba.obj
 0003:00000750       gARCSASPMCSubsystemInfo    000000014002d750     archba.obj
 0003:00000a70       gARCVendor                 000000014002da70     arcinit.obj
 0003:00000a78       gAdapterGuid               000000014002da78     wmi.obj
 0003:00000a88       gIoChannelGuid             000000014002da88     wmi.obj
 0003:00000a98       gDiskArrayGuid             000000014002da98     wmi.obj
 0003:00000aa8       gPhysicalDiskGuid          000000014002daa8     wmi.obj
 0003:00000ab8       gAdapterMethodGuid         000000014002dab8     wmi.obj
 0003:00000ad0       __security_cookie          000000014002dad0     BufferOverflowFastFailK:gs_support.obj
 0003:00000ad8       __security_cookie_complement 000000014002dad8     BufferOverflowFastFailK:gs_support.obj
 0003:00000b10       gAdapterAddCount           000000014002db10     arcinit.obj
 0003:00000b14       gLatency                   000000014002db14     arcinit.obj
 0003:00000b18       gLoopbackInPushFib         000000014002db18     arcinit.obj
 0003:00000b20       gTraceContext              000000014002db20     arcinit.obj
 0003:00000bc0       gAdapterTable              000000014002dbc0     <common>
 0003:00000dc0       gDriverObject              000000014002ddc0     <common>
 0005:00000000       GsDriverEntry              000000014002f000 f   BufferOverflowFastFailK:gs_driverentry.obj
 0005:0000002c       __security_init_cookie     000000014002f02c f   BufferOverflowFastFailK:gs_support.obj
 0005:0000005c       __IMPORT_DESCRIPTOR_ntoskrnl 000000014002f05c     ntoskrnl:ntoskrnl.exe
 0005:00000070       __IMPORT_DESCRIPTOR_HAL    000000014002f070     hal:HAL.dll
 0005:00000084       __IMPORT_DESCRIPTOR_storport 000000014002f084     storport:storport.sys
 0005:00000098       __NULL_IMPORT_DESCRIPTOR   000000014002f098     ntoskrnl:ntoskrnl.exe

 entry point at        0005:00000000

 Static symbols

 0002:fffd4fff       __guard_fids__guard_icall_checks_enforced 000000023fffffff     BufferOverflowFastFailK:guard_support.obj
 0002:fffd4fff       __guard_fids__             000000023fffffff     BufferOverflowFastFailK:guard_support.obj
 0000:fffcd000       .debug$S                   0000000140000000     storport:storport.sys
 0000:fffcd000       .debug$S                   0000000140000000     hal:HAL.dll
 0002:fffd5000       __guard_fids_InitializeDPCs 0000000140000000     arcinit.obj
 0002:fffd5000       __guard_fids_FindAdapter   0000000140000000     arcinit.obj
 0002:fffd5000       __guard_fids_WppInitKm     0000000140000000     arcinit.obj
 0002:fffd5000       __guard_fids_HwInitializeAdapter 0000000140000000     arcinit.obj
 0002:fffd5000       __guard_fids_DriverEntry   0000000140000000     arcinit.obj
 0002:fffd5000       __guard_fids_InitializeWmiInterface 0000000140000000     wmi.obj
 0002:fffd5000       __guard_fids__             0000000140000000     archba.obj
 0002:fffd5000       __guard_fids_RequestTimer  0000000140000000     timer.obj
 0002:fffd5000       __guard_fids_UpdateThorHBAMappingTable 0000000140000000     timer.obj
 0002:fffd5000       __guard_fids__             0000000140000000     arcdebug.obj
 0000:fffcd000       .debug$S                   0000000140000000     storport:storport.sys
 0000:fffcd000       .debug$S                   0000000140000000     storport:storport.sys
 0000:fffcd000       .debug$S                   0000000140000000     storport:storport.sys
 0000:fffcd000       .debug$S                   0000000140000000     storport:storport.sys
 0000:fffcd000       .debug$S                   0000000140000000     storport:storport.sys
 0000:fffcd000       .debug$S                   0000000140000000     storport:storport.sys
 0000:fffcd000       .debug$S                   0000000140000000     storport:storport.sys
 0000:fffcd000       .debug$S                   0000000140000000     storport:storport.sys
 0000:fffcd000       .debug$S                   0000000140000000     storport:storport.sys
 0000:fffcd000       .debug$S                   0000000140000000     storport:storport.sys
 0000:fffcd000       .debug$S                   0000000140000000     storport:storport.sys
 0000:fffcd000       .debug$S                   0000000140000000     storport:storport.sys
 0000:fffcd000       .debug$S                   0000000140000000     storport:storport.sys
 0000:fffcd000       .debug$S                   0000000140000000     storport:storport.sys
 0000:fffcd000       .debug$S                   0000000140000000     storport:storport.sys
 0000:fffcd000       .debug$S                   0000000140000000     storport:storport.sys
 0000:fffcd000       .debug$S                   0000000140000000     storport:storport.sys
 0000:fffcd000       .debug$S                   0000000140000000     storport:storport.sys
 0000:fffcd000       .debug$S                   0000000140000000     ntoskrnl:ntoskrnl.exe
 0000:fffcd000       .debug$S                   0000000140000000     ntoskrnl:ntoskrnl.exe
 0001:00001d80       $LN72                      0000000140002d80     rxdevice.obj
 0001:00004cf4       $LN194                     0000000140005cf4     arcdebug.obj
 0001:00004d0c       $LN193                     0000000140005d0c     arcdebug.obj
 0001:000090d0       $LN14                      000000014000a0d0     arcinit.obj
 0001:0000fc40       $LN43                      0000000140010c40     arcinit.obj
 0001:0001011c       $LN67                      000000014001111c     arcinit.obj
 0001:00010a7c       $LN231                     0000000140011a7c     arcinit.obj
 0001:00010f50       $LN125                     0000000140011f50     arcinit.obj
 0001:00011644       $LN319                     0000000140012644     arcinit.obj
 0001:0001259c       $LN28                      000000014001359c     arcinit.obj
 0001:00014174       $LN132                     0000000140015174     cmddelivery.obj
 0001:0001419c       $LN131                     000000014001519c     cmddelivery.obj
 0001:00014238       $LN130                     0000000140015238     cmddelivery.obj
 0001:0001425c       $LN129                     000000014001525c     cmddelivery.obj
 0001:00015ac4       $LN157                     0000000140016ac4     cmddelivery.obj
 0001:00015adc       $LN156                     0000000140016adc     cmddelivery.obj
 0001:000174c8       $LN191                     00000001400184c8     cmdproc.obj
 0001:000174e0       $LN190                     00000001400184e0     cmdproc.obj
 0001:00017508       $LN189                     0000000140018508     cmdproc.obj
 0001:00017518       $LN188                     0000000140018518     cmdproc.obj
 0001:00019b08       $LN102                     000000014001ab08     ioctl.obj
 0001:0001c470       $LN382                     000000014001d470     ioctl.obj
 0001:0001c4b0       $LN381                     000000014001d4b0     ioctl.obj
 0001:0001d3c8       $LN132                     000000014001e3c8     comm.obj
 0001:0001d3e8       $LN131                     000000014001e3e8     comm.obj
 0001:0001d410       $LN130                     000000014001e410     comm.obj
 0001:0001d9b4       $LN34                      000000014001e9b4     comm.obj
 0001:0001d9d0       $LN33                      000000014001e9d0     comm.obj
 0001:0001f0b0       $$000000                   00000001400200b0     BufferOverflowFastFailK:amdsecgs.obj
 0001:0001f860       $$000000                   0000000140020860     BufferOverflowFastFailK:guard_dispatch.obj
 0001:0001f880       $$000000                   0000000140020880     ntoskrnl:memcpy.obj
 0001:0001fbc0       $$000000                   0000000140020bc0     ntoskrnl:memset.obj
 0002:000009f0       $unwind$RxCheckAdapterHealth 000000014002b9f0     rxdevice.obj
 0002:000009fc       $unwind$RxNewCommProcessInterrupt 000000014002b9fc     rxdevice.obj
 0002:00000a14       $chain$0$RxNewCommProcessInterrupt 000000014002ba14     rxdevice.obj
 0002:00000a28       $chain$3$RxNewCommProcessInterrupt 000000014002ba28     rxdevice.obj
 0002:00000a44       $chain$6$RxNewCommProcessInterrupt 000000014002ba44     rxdevice.obj
 0002:00000a44       $chain$4$RxNewCommProcessInterrupt 000000014002ba44     rxdevice.obj
 0002:00000a58       $chain$5$RxNewCommProcessInterrupt 000000014002ba58     rxdevice.obj
 0002:00000a74       $chain$7$RxNewCommProcessInterrupt 000000014002ba74     rxdevice.obj
 0002:00000a88       $unwind$RxInterruptHandler 000000014002ba88     rxdevice.obj
 0002:00000a98       $chain$0$RxInterruptHandler 000000014002ba98     rxdevice.obj
 0002:00000ab0       $chain$2$RxInterruptHandler 000000014002bab0     rxdevice.obj
 0002:00000ab0       $chain$6$RxInterruptHandler 000000014002bab0     rxdevice.obj
 0002:00000ab0       $chain$4$RxInterruptHandler 000000014002bab0     rxdevice.obj
 0002:00000ac8       $chain$8$RxInterruptHandler 000000014002bac8     rxdevice.obj
 0002:00000adc       $chain$9$RxInterruptHandler 000000014002badc     rxdevice.obj
 0002:00000af0       $unwind$NonMSIXInterruptHandler 000000014002baf0     rxdevice.obj
 0002:00000b04       $chain$3$NonMSIXInterruptHandler 000000014002bb04     rxdevice.obj
 0002:00000b24       $chain$4$NonMSIXInterruptHandler 000000014002bb24     rxdevice.obj
 0002:00000b38       $unwind$PMCDpcResponseHandler 000000014002bb38     rxdevice.obj
 0002:00000b44       $chain$5$PMCDpcResponseHandler 000000014002bb44     rxdevice.obj
 0002:00000b6c       $chain$6$PMCDpcResponseHandler 000000014002bb6c     rxdevice.obj
 0002:00000b80       $chain$8$PMCDpcResponseHandler 000000014002bb80     rxdevice.obj
 0002:00000b94       $chain$9$PMCDpcResponseHandler 000000014002bb94     rxdevice.obj
 0002:00000ba8       $unwind$PMCInterruptHandler 000000014002bba8     rxdevice.obj
 0002:00000bb8       $chain$2$PMCInterruptHandler 000000014002bbb8     rxdevice.obj
 0002:00000bd4       $chain$3$PMCInterruptHandler 000000014002bbd4     rxdevice.obj
 0002:00000bec       $unwind$RxPullMessageUnitQueueCompletedFib 000000014002bbec     rxdevice.obj
 0002:00000c08       $chain$1$RxPullMessageUnitQueueCompletedFib 000000014002bc08     rxdevice.obj
 0002:00000c20       $chain$2$RxPullMessageUnitQueueCompletedFib 000000014002bc20     rxdevice.obj
 0002:00000c34       $unwind$RxPushMessageUnitQueueFib 000000014002bc34     rxdevice.obj
 0002:00000c44       $chain$0$RxPushMessageUnitQueueFib 000000014002bc44     rxdevice.obj
 0002:00000c58       $chain$1$RxPushMessageUnitQueueFib 000000014002bc58     rxdevice.obj
 0002:00000c6c       $unwind$PMCPushMessageUnitQueueFib 000000014002bc6c     rxdevice.obj
 0002:00000c78       $chain$0$PMCPushMessageUnitQueueFib 000000014002bc78     rxdevice.obj
 0002:00000c8c       $chain$1$PMCPushMessageUnitQueueFib 000000014002bc8c     rxdevice.obj
 0002:00000ca4       $chain$2$PMCPushMessageUnitQueueFib 000000014002bca4     rxdevice.obj
 0002:00000cb8       $unwind$RxSendSynchCommand 000000014002bcb8     rxdevice.obj
 0002:00000cd4       $unwind$RxStartAdapter     000000014002bcd4     rxdevice.obj
 0002:00000cf0       $unwind$RxWaitForAdapterToBoot 000000014002bcf0     rxdevice.obj
 0002:00000cfc       $chain$0$RxWaitForAdapterToBoot 000000014002bcfc     rxdevice.obj
 0002:00000d14       $chain$1$RxWaitForAdapterToBoot 000000014002bd14     rxdevice.obj
 0002:00000d28       $unwind$DumpHandles        000000014002bd28     rxdevice.obj
 0002:00000d28       $unwind$DumpHandlesZeroPointer 000000014002bd28     rxdevice.obj
 0002:00000d44       $unwind$RevCheckCompatibility 000000014002bd44     revision.obj
 0002:00000d54       $unwind$GetDriverParameter 000000014002bd54     helpers.obj
 0002:00000d70       $unwind$MatchRegistryString 000000014002bd70     helpers.obj
 0002:00000d80       $unwind$LongToAscii        000000014002bd80     helpers.obj
 0002:00000d94       $unwind$CompareStrings     000000014002bd94     helpers.obj
 0002:00000da0       $unwind$ArcPrintf          000000014002bda0     arcdebug.obj
 0002:00000db8       $chain$3$ArcPrintf         000000014002bdb8     arcdebug.obj
 0002:00000dd8       $chain$4$ArcPrintf         000000014002bdd8     arcdebug.obj
 0002:00000dec       $unwind$RealSprintf        000000014002bdec     arcdebug.obj
 0002:00000dfc       $chain$1$RealSprintf       000000014002bdfc     arcdebug.obj
 0002:00000e14       $chain$6$RealSprintf       000000014002be14     arcdebug.obj
 0002:00000e38       $chain$7$RealSprintf       000000014002be38     arcdebug.obj
 0002:00000e48       $chain$8$RealSprintf       000000014002be48     arcdebug.obj
 0002:00000e5c       $unwind$MainTimeThread     000000014002be5c     timer.obj
 0002:00000e74       $chain$4$MainTimeThread    000000014002be74     timer.obj
 0002:00000e98       $chain$5$MainTimeThread    000000014002be98     timer.obj
 0002:00000eb8       $chain$6$MainTimeThread    000000014002beb8     timer.obj
 0002:00000ecc       $chain$7$MainTimeThread    000000014002becc     timer.obj
 0002:00000ee0       $unwind$VMCloseAllCompletionTimer 000000014002bee0     timer.obj
 0002:00000eec       $chain$0$VMCloseAllCompletionTimer 000000014002beec     timer.obj
 0002:00000f04       $chain$1$VMCloseAllCompletionTimer 000000014002bf04     timer.obj
 0002:00000f18       $unwind$UpdateThorHBAMappingTable 000000014002bf18     timer.obj
 0002:00000f28       $chain$0$UpdateThorHBAMappingTable 000000014002bf28     timer.obj
 0002:00000f3c       $chain$2$UpdateThorHBAMappingTable 000000014002bf3c     timer.obj
 0002:00000f54       $chain$3$UpdateThorHBAMappingTable 000000014002bf54     timer.obj
 0002:00000f64       $chain$4$UpdateThorHBAMappingTable 000000014002bf64     timer.obj
 0002:00000f78       $unwind$Reset_IOP_CompletionTimer 000000014002bf78     timer.obj
 0002:00000f84       $chain$0$Reset_IOP_CompletionTimer 000000014002bf84     timer.obj
 0002:00000f9c       $chain$2$Reset_IOP_CompletionTimer 000000014002bf9c     timer.obj
 0002:00000fb4       $chain$4$Reset_IOP_CompletionTimer 000000014002bfb4     timer.obj
 0002:00000fc8       $chain$5$Reset_IOP_CompletionTimer 000000014002bfc8     timer.obj
 0002:00000fdc       $unwind$StopTimer          000000014002bfdc     timer.obj
 0002:00000ff0       $unwind$RequestTimer       000000014002bff0     timer.obj
 0002:00001008       $unwind$CheckingFWAfterPowerStateChange 000000014002c008     timer.obj
 0002:00001018       $chain$0$CheckingFWAfterPowerStateChange 000000014002c018     timer.obj
 0002:00001030       $chain$3$CheckingFWAfterPowerStateChange 000000014002c030     timer.obj
 0002:00001048       $chain$4$CheckingFWAfterPowerStateChange 000000014002c048     timer.obj
 0002:0000105c       $unwind$StorWmiTraceMessage 000000014002c05c     arcinit.obj
 0002:00001068       $unwind$DriverEntry        000000014002c068     arcinit.obj
 0002:00001080       $chain$0$DriverEntry       000000014002c080     arcinit.obj
 0002:00001094       $chain$1$DriverEntry       000000014002c094     arcinit.obj
 0002:000010a8       $chain$2$DriverEntry       000000014002c0a8     arcinit.obj
 0002:000010b8       $chain$3$DriverEntry       000000014002c0b8     arcinit.obj
 0002:000010cc       $unwind$HwInitializeAdapter 000000014002c0cc     arcinit.obj
 0002:000010f4       $unwind$FindAdapter        000000014002c0f4     arcinit.obj
 0002:00001110       $chain$1$FindAdapter       000000014002c110     arcinit.obj
 0002:00001128       $chain$2$FindAdapter       000000014002c128     arcinit.obj
 0002:0000113c       $unwind$ResetAdapter       000000014002c13c     arcinit.obj
 0002:00001150       $chain$5$ResetAdapter      000000014002c150     arcinit.obj
 0002:00001178       $chain$6$ResetAdapter      000000014002c178     arcinit.obj
 0002:0000118c       $unwind$SMNormalModeInitAdapter 000000014002c18c     arcinit.obj
 0002:00001198       $chain$1$SMNormalModeInitAdapter 000000014002c198     arcinit.obj
 0002:000011b0       $chain$2$SMNormalModeInitAdapter 000000014002c1b0     arcinit.obj
 0002:000011c4       $unwind$InitializeDPCs     000000014002c1c4     arcinit.obj
 0002:000011d8       $chain$1$InitializeDPCs    000000014002c1d8     arcinit.obj
 0002:000011f0       $chain$2$InitializeDPCs    000000014002c1f0     arcinit.obj
 0002:00001204       $unwind$ReturningLocalOutstandingRequestsToOS 000000014002c204     arcinit.obj
 0002:00001204       $unwind$HWSoftReset        000000014002c204     arcinit.obj
 0002:00001214       $unwind$CleanHostSideRRQ   000000014002c214     arcinit.obj
 0002:00001220       $unwind$ScsiPortWmiPostProcess 000000014002c220     scsiwmi:wmilib.obj
 0002:00001220       $unwind$EventTracingCleanup 000000014002c220     arcinit.obj
 0002:0000122c       $unwind$AllocateConsumerProducerCommArea 000000014002c22c     arcinit.obj
 0002:00001248       $unwind$AllocateMessageUnitQueueCommArea 000000014002c248     arcinit.obj
 0002:00001264       $unwind$ConfigureContainersRuntime 000000014002c264     arcinit.obj
 0002:00001288       $chain$0$ConfigureContainersRuntime 000000014002c288     arcinit.obj
 0002:0000129c       $chain$1$ConfigureContainersRuntime 000000014002c29c     arcinit.obj
 0002:000012ac       $unwind$SendEvent2OSDelayed 000000014002c2ac     arcinit.obj
 0002:000012c4       $unwind$HwScsiWmiExecuteMethod 000000014002c2c4     wmi.obj
 0002:000012c4       $unwind$GsDriverEntry      000000014002c2c4     BufferOverflowFastFailK:gs_driverentry.obj
 0002:000012c4       $unwind$GetElapsedSeconds  000000014002c2c4     arcinit.obj
 0002:000012d4       $unwind$HandleAdapterGetConfig 000000014002c2d4     arcinit.obj
 0002:000012d4       $unwind$IsAdapterReadyForConfigCommand 000000014002c2d4     arcinit.obj
 0002:000012d4       $unwind$HandleAdapterConfigIssues 000000014002c2d4     arcinit.obj
 0002:000012d4       $unwind$HandleAdapterCommitConfig 000000014002c2d4     arcinit.obj
 0002:000012ec       $unwind$CheckMSIxPossibility 000000014002c2ec     arcinit.obj
 0002:000012f4       $chain$0$CheckMSIxPossibility 000000014002c2f4     arcinit.obj
 0002:00001308       $chain$1$CheckMSIxPossibility 000000014002c308     arcinit.obj
 0002:0000131c       $chain$2$CheckMSIxPossibility 000000014002c31c     arcinit.obj
 0002:00001334       $chain$3$CheckMSIxPossibility 000000014002c334     arcinit.obj
 0002:00001348       $unwind$SendInitStructure  000000014002c348     arcinit.obj
 0002:00001360       $unwind$InitializeConsumerProducerCommRegion 000000014002c360     arcinit.obj
 0002:00001374       $unwind$MapDeviceBase      000000014002c374     arcinit.obj
 0002:00001390       $unwind$IOPReset           000000014002c390     arcinit.obj
 0002:000013ac       $unwind$DumpFibsSentToFW60SecondsBefore 000000014002c3ac     arcinit.obj
 0002:000013b8       $chain$4$DumpFibsSentToFW60SecondsBefore 000000014002c3b8     arcinit.obj
 0002:000013dc       $chain$5$DumpFibsSentToFW60SecondsBefore 000000014002c3dc     arcinit.obj
 0002:000013f0       $unwind$ReturningOutstandingSentToFWBeforeIOPResetToOS 000000014002c3f0     arcinit.obj
 0002:000013fc       $chain$3$ReturningOutstandingSentToFWBeforeIOPResetToOS 000000014002c3fc     arcinit.obj
 0002:0000141c       $chain$4$ReturningOutstandingSentToFWBeforeIOPResetToOS 000000014002c41c     arcinit.obj
 0002:00001430       $chain$5$ReturningOutstandingSentToFWBeforeIOPResetToOS 000000014002c430     arcinit.obj
 0002:00001440       $chain$6$ReturningOutstandingSentToFWBeforeIOPResetToOS 000000014002c440     arcinit.obj
 0002:00001454       $unwind$ReturnOutstandingFibOnTargetDevice 000000014002c454     arcinit.obj
 0002:00001464       $chain$2$ReturnOutstandingFibOnTargetDevice 000000014002c464     arcinit.obj
 0002:00001480       $chain$3$ReturnOutstandingFibOnTargetDevice 000000014002c480     arcinit.obj
 0002:00001494       $chain$4$ReturnOutstandingFibOnTargetDevice 000000014002c494     arcinit.obj
 0002:000014a4       $chain$5$ReturnOutstandingFibOnTargetDevice 000000014002c4a4     arcinit.obj
 0002:000014b8       $unwind$SetFwTime          000000014002c4b8     arcinit.obj
 0002:000014d0       $chain$0$SetFwTime         000000014002c4d0     arcinit.obj
 0002:000014e4       $chain$4$SetFwTime         000000014002c4e4     arcinit.obj
 0002:00001504       $chain$5$SetFwTime         000000014002c504     arcinit.obj
 0002:0000151c       $chain$6$SetFwTime         000000014002c51c     arcinit.obj
 0002:0000152c       $chain$7$SetFwTime         000000014002c52c     arcinit.obj
 0002:00001540       $unwind$SetArcsasFwTime    000000014002c540     arcinit.obj
 0002:00001550       $unwind$SetPciSlotNumber   000000014002c550     arcinit.obj
 0002:00001564       $unwind$SendWellnessCmnd   000000014002c564     arcinit.obj
 0002:00001580       $unwind$GetThorHbaPhyDevInfo 000000014002c580     arcinit.obj
 0002:0000159c       $unwind$ArcLogEventString  000000014002c59c     arcinit.obj
 0002:000015a8       $unwind$LogSystemEvent     000000014002c5a8     arcinit.obj
 0002:000015b4       $unwind$SendEvent2OS       000000014002c5b4     arcinit.obj
 0002:000015d4       $unwind$WppTraceCallback   000000014002c5d4     arcinit.obj
 0002:000015e4       $chain$2$WppTraceCallback  000000014002c5e4     arcinit.obj
 0002:00001604       $chain$3$WppTraceCallback  000000014002c604     arcinit.obj
 0002:00001620       $unwind$DynamicallyThrottleLunQueueDepth 000000014002c620     arcinit.obj
 0002:00001640       $unwind$SA4StatusBatching  000000014002c640     arcinit.obj
 0002:00001650       $unwind$SA4ACI2Interface   000000014002c650     arcinit.obj
 0002:00001660       $unwind$SMCrashDumpModeInitAdapter 000000014002c660     arcinit.obj
 0002:00001678       $unwind$SendEvent2OSChild  000000014002c678     arcinit.obj
 0002:00001694       $unwind$StartIo            000000014002c694     cmddelivery.obj
 0002:000016b0       $chain$0$StartIo           000000014002c6b0     cmddelivery.obj
 0002:000016c4       $chain$1$StartIo           000000014002c6c4     cmddelivery.obj
 0002:000016d8       $unwind$PostProcessScsiCommand 000000014002c6d8     cmddelivery.obj
 0002:000016f0       $unwind$SendFib            000000014002c6f0     cmddelivery.obj
 0002:0000170c       $unwind$HandleMSIXInterrupt 000000014002c70c     cmddelivery.obj
 0002:0000171c       $unwind$QueueRawIoReadWriteRequest 000000014002c71c     cmddelivery.obj
 0002:00001728       $chain$1$QueueRawIoReadWriteRequest 000000014002c728     cmddelivery.obj
 0002:00001744       $chain$3$QueueRawIoReadWriteRequest 000000014002c744     cmddelivery.obj
 0002:0000175c       $chain$4$QueueRawIoReadWriteRequest 000000014002c75c     cmddelivery.obj
 0002:00001770       $chain$5$QueueRawIoReadWriteRequest 000000014002c770     cmddelivery.obj
 0002:00001780       $chain$6$QueueRawIoReadWriteRequest 000000014002c780     cmddelivery.obj
 0002:00001794       $unwind$CompleteQueuedRequest 000000014002c794     cmddelivery.obj
 0002:000017a8       $unwind$DequeueRawIoReadWriteRequest 000000014002c7a8     cmddelivery.obj
 0002:000017bc       $chain$0$DequeueRawIoReadWriteRequest 000000014002c7bc     cmddelivery.obj
 0002:000017d0       $chain$1$DequeueRawIoReadWriteRequest 000000014002c7d0     cmddelivery.obj
 0002:000017e4       $unwind$ProcessContainerInquiry 000000014002c7e4     cmddelivery.obj
 0002:00001804       $unwind$ProcessScsiCommand 000000014002c804     cmddelivery.obj
 0002:0000182c       $unwind$QueuePrintf        000000014002c82c     cmddelivery.obj
 0002:00001840       $unwind$SendRawIoFib       000000014002c840     cmddelivery.obj
 0002:00001860       $unwind$SendSynchFib       000000014002c860     cmddelivery.obj
 0002:00001878       $chain$0$SendSynchFib      000000014002c878     cmddelivery.obj
 0002:0000188c       $chain$1$SendSynchFib      000000014002c88c     cmddelivery.obj
 0002:000018a0       $unwind$DequeueCertainLD   000000014002c8a0     cmddelivery.obj
 0002:000018b4       $chain$0$DequeueCertainLD  000000014002c8b4     cmddelivery.obj
 0002:000018c8       $chain$1$DequeueCertainLD  000000014002c8c8     cmddelivery.obj
 0002:000018dc       $unwind$PollSmartHBAFIBCompletion 000000014002c8dc     cmddelivery.obj
 0002:000018f8       $unwind$AdapterControl     000000014002c8f8     cmdproc.obj
 0002:0000190c       $unwind$BuildIo            000000014002c90c     cmdproc.obj
 0002:00001930       $unwind$BuildHBAFib        000000014002c930     cmdproc.obj
 0002:0000194c       $unwind$BuildRawIoFib      000000014002c94c     cmdproc.obj
 0002:00001964       $unwind$BuildRawIoScatterGather 000000014002c964     cmdproc.obj
 0002:0000197c       $chain$0$BuildRawIoScatterGather 000000014002c97c     cmdproc.obj
 0002:00001990       $chain$1$BuildRawIoScatterGather 000000014002c990     cmdproc.obj
 0002:000019a4       $chain$2$BuildRawIoScatterGather 000000014002c9a4     cmdproc.obj
 0002:000019b8       $chain$3$BuildRawIoScatterGather 000000014002c9b8     cmdproc.obj
 0002:000019c8       $unwind$BuildRawIo2ScatterGather 000000014002c9c8     cmdproc.obj
 0002:000019e8       $unwind$ConvertRawIo2ScatterGather 000000014002c9e8     cmdproc.obj
 0002:000019f4       $chain$1$ConvertRawIo2ScatterGather 000000014002c9f4     cmdproc.obj
 0002:00001a0c       $chain$3$ConvertRawIo2ScatterGather 000000014002ca0c     cmdproc.obj
 0002:00001a24       $chain$4$ConvertRawIo2ScatterGather 000000014002ca24     cmdproc.obj
 0002:00001a34       $chain$5$ConvertRawIo2ScatterGather 000000014002ca34     cmdproc.obj
 0002:00001a48       $unwind$BuildReadWriteFib  000000014002ca48     cmdproc.obj
 0002:00001a64       $unwind$BuildScatterGather 000000014002ca64     cmdproc.obj
 0002:00001a64       $unwind$SendConsumerProducerFib 000000014002ca64     comm.obj
 0002:00001a64       $unwind$BuildScatterGather64 000000014002ca64     cmdproc.obj
 0002:00001a80       $unwind$BuildRawIo2ScatterGather4HBAIoctl 000000014002ca80     cmdproc.obj
 0002:00001a9c       $unwind$BuildHBAIoctlFib   000000014002ca9c     cmdproc.obj
 0002:00001ab8       $unwind$BuildSrbFib        000000014002cab8     cmdproc.obj
 0002:00001ad4       $unwind$InitializeFib      000000014002cad4     cmdproc.obj
 0002:00001ae0       $unwind$PrepareBMIC15      000000014002cae0     cmdproc.obj
 0002:00001afc       $unwind$ProcessIoctl       000000014002cafc     ioctl.obj
 0002:00001b24       $unwind$BuildRawScatterGather 000000014002cb24     ioctl.obj
 0002:00001b38       $chain$1$BuildRawScatterGather 000000014002cb38     ioctl.obj
 0002:00001b50       $chain$2$BuildRawScatterGather 000000014002cb50     ioctl.obj
 0002:00001b64       $unwind$BuildRawScatterGather64 000000014002cb64     ioctl.obj
 0002:00001b80       $unwind$CSMIGetRAIDConfig  000000014002cb80     ioctl.obj
 0002:00001b98       $chain$0$CSMIGetRAIDConfig 000000014002cb98     ioctl.obj
 0002:00001bb0       $chain$1$CSMIGetRAIDConfig 000000014002cbb0     ioctl.obj
 0002:00001bc4       $unwind$CSMIGetRAIDInfo    000000014002cbc4     ioctl.obj
 0002:00001be4       $unwind$CSMISTPPassThru    000000014002cbe4     ioctl.obj
 0002:00001bfc       $chain$0$CSMISTPPassThru   000000014002cbfc     ioctl.obj
 0002:00001c10       $chain$1$CSMISTPPassThru   000000014002cc10     ioctl.obj
 0002:00001c28       $unwind$HandleCSMI         000000014002cc28     ioctl.obj
 0002:00001c4c       $unwind$QueueEvent         000000014002cc4c     comm.obj
 0002:00001c64       $unwind$AdapterIsAlive     000000014002cc64     comm.obj
 0002:00001c70       $unwind$ServiceHostResponseNormalQueue 000000014002cc70     comm.obj
 0002:00001c78       $chain$6$ServiceHostResponseNormalQueue 000000014002cc78     comm.obj
 0002:00001ca4       $chain$7$ServiceHostResponseNormalQueue 000000014002cca4     comm.obj
 0002:00001cb8       $unwind$FreeConsumerProducerAif 000000014002ccb8     comm.obj
 0002:00001cb8       $unwind$CompleteBufferedRequest 000000014002ccb8     comm.obj
 0002:00001ccc       $chain$0$FreeConsumerProducerAif 000000014002cccc     comm.obj
 0002:00001ce0       $chain$1$FreeConsumerProducerAif 000000014002cce0     comm.obj
 0002:00001cf4       $unwind$ProcessAif         000000014002ccf4     comm.obj
 0002:00001d0c       $unwind$SubDeQueueSortingQueue 000000014002cd0c     comm.obj
 0002:00001d1c       $chain$0$SubDeQueueSortingQueue 000000014002cd1c     comm.obj
 0002:00001d34       $chain$1$SubDeQueueSortingQueue 000000014002cd34     comm.obj
 0002:00001d48       $unwind$DeQueueSortingQueue 000000014002cd48     comm.obj
 0002:00001d68       $unwind$CompleteAllSortingQueue 000000014002cd68     comm.obj
 0002:00001d74       $chain$5$CompleteAllSortingQueue 000000014002cd74     comm.obj
 0002:00001d9c       $chain$6$CompleteAllSortingQueue 000000014002cd9c     comm.obj
 0002:00001db0       $chain$0$CompleteBufferedRequest 000000014002cdb0     comm.obj
 0002:00001dc4       $chain$1$CompleteBufferedRequest 000000014002cdc4     comm.obj
 0002:00001dd8       $unwind$ServiceHostCommandNormalQueue 000000014002cdd8     comm.obj
 0002:00001de0       $chain$3$ServiceHostCommandNormalQueue 000000014002cde0     comm.obj
 0002:00001e00       $chain$4$ServiceHostCommandNormalQueue 000000014002ce00     comm.obj
 0002:00001e14       $unwind$DpcDequeueRawIoReadWriteRequest 000000014002ce14     comm.obj
 0002:00001e20       $unwind$ProcessNormalFib   000000014002ce20     comm.obj
 0002:00001e2c       $chain$3$ProcessNormalFib  000000014002ce2c     comm.obj
 0002:00001e4c       $chain$5$ProcessNormalFib  000000014002ce4c     comm.obj
 0002:00001e64       $chain$6$ProcessNormalFib  000000014002ce64     comm.obj
 0002:00001e74       $chain$7$ProcessNormalFib  000000014002ce74     comm.obj
 0002:00001e88       $chain$8$ProcessNormalFib  000000014002ce88     comm.obj
 0002:00001eb0       $unwind$ServiceInternalAifQueue 000000014002ceb0     comm.obj
 0002:00001ec4       $unwind$ProcessHbaErrors   000000014002cec4     comm.obj
 0002:00001ee0       $chain$3$ProcessHbaErrors  000000014002cee0     comm.obj
 0002:00001f00       $chain$4$ProcessHbaErrors  000000014002cf00     comm.obj
 0002:00001f1c       $unwind$ProcessWmi         000000014002cf1c     wmi.obj
 0002:00001f2c       $unwind$__GSHandlerCheck   000000014002cf2c     ntoskrnl:gshandler.obj
 0002:00001f2c       $unwind$__GSHandlerCheckCommon 000000014002cf2c     ntoskrnl:gshandler.obj
 0002:00001f2c       $unwind$HwScsiWmiFunctionControl 000000014002cf2c     wmi.obj
 0002:00001f2c       $unwind$HwScsiWmiQueryDataBlock 000000014002cf2c     wmi.obj
 0002:00001f38       $xdatasym                  000000014002cf38     BufferOverflowFastFailK:amdsecgs.obj
 0002:00001f40       $xdatasym                  000000014002cf40     BufferOverflowFastFailK:guard_dispatch.obj
 0002:00001f48       $xdatasym                  000000014002cf48     ntoskrnl:memcpy.obj
 0002:00001f50       $xdatasym                  000000014002cf50     ntoskrnl:memset.obj
 0002:00001f54       $unwind$ScsiPortWmiDispatchFunction 000000014002cf54     scsiwmi:wmilib.obj
 0002:00001f64       $unwind$ScsiWmipProcessRequest 000000014002cf64     scsiwmi:wmilib.obj
 0002:00001f84       $unwind$ScsiWmipPostProcess 000000014002cf84     scsiwmi:wmilib.obj
 0002:00001f98       $unwind$ScsiWmipFindGuid   000000014002cf98     scsiwmi:wmilib.obj
 0003:00000044       ?NeedToReadStatus@?1??CheckingFWAfterPowerStateChange@@9@9 000000014002d044     timer.obj
 0003:00000045       ?NeedToCheckMSIX@?1??CheckingFWAfterPowerStateChange@@9@9 000000014002d045     timer.obj
 0003:00000ae0       ?CalledCnt@?1??CheckForDupHandles@@9@9 000000014002dae0     rxdevice.obj
 0003:00000ae8       ?CalledCnt@?1??CheckFWPulseInCrashDumpMode@@9@9 000000014002dae8     timer.obj
 0003:00000aec       ?TimerAge@?1??CheckingFWAfterPowerStateChange@@9@9 000000014002daec     timer.obj
 0003:00000af0       ?status@?1??CheckingFWAfterPowerStateChange@@9@9 000000014002daf0     timer.obj
 0003:00000af4       ?DelayCnt4DualFWFlushSoftReset@?1??CheckingFWAfterPowerStateChange@@9@9 000000014002daf4     timer.obj
 0003:00000af8       ?pSavedDevExt@?1??CheckingFWAfterPowerStateChange@@9@9 000000014002daf8     timer.obj
 0003:00000b00       ?TimerAge@?1??Reset_IOP_CompletionTimer@@9@9 000000014002db00     timer.obj
 0003:00000b28       ?NewScanStarted@?1??ConfigureContainersRuntime@@9@9 000000014002db28     arcinit.obj
 0003:00000b29       ?LoopCount@?1??ConfigureContainersRuntime@@9@9 000000014002db29     arcinit.obj
 0003:00000b2a       ?busChange@?1??ConfigureContainersRuntime@@9@9 000000014002db2a     arcinit.obj
 0003:00000b2b       ?initialized@?1??DriverEntry@@9@9 000000014002db2b     arcinit.obj
 0003:00000b2c       ?containerCount@?1??ConfigureContainersRuntime@@9@9 000000014002db2c     arcinit.obj
 0003:00000b30       ?diskInfoResponse@?1??ConfigureContainersRuntime@@9@9 000000014002db30     arcinit.obj
 0003:00000b98       ?pSavedDevExt@?1??ConfigureContainersRuntime@@9@9 000000014002db98     arcinit.obj
 0003:00000ba0       ?SkipSecondSynchCmd@?1??ConfigureContainersRuntime@@9@9 000000014002dba0     arcinit.obj
 0003:00000ba4       ?ShutdownSent@?1??BuildIo@@9@9 000000014002dba4     cmdproc.obj
 0004:00000000       $pdata$RxCheckAdapterHealth 000000014002e000     rxdevice.obj
 0004:0000000c       $pdata$RxNewCommProcessInterrupt 000000014002e00c     rxdevice.obj
 0004:00000018       $pdata$0$RxNewCommProcessInterrupt 000000014002e018     rxdevice.obj
 0004:00000024       $pdata$3$RxNewCommProcessInterrupt 000000014002e024     rxdevice.obj
 0004:00000030       $pdata$4$RxNewCommProcessInterrupt 000000014002e030     rxdevice.obj
 0004:0000003c       $pdata$5$RxNewCommProcessInterrupt 000000014002e03c     rxdevice.obj
 0004:00000048       $pdata$6$RxNewCommProcessInterrupt 000000014002e048     rxdevice.obj
 0004:00000054       $pdata$7$RxNewCommProcessInterrupt 000000014002e054     rxdevice.obj
 0004:00000060       $pdata$RxInterruptHandler  000000014002e060     rxdevice.obj
 0004:0000006c       $pdata$0$RxInterruptHandler 000000014002e06c     rxdevice.obj
 0004:00000078       $pdata$2$RxInterruptHandler 000000014002e078     rxdevice.obj
 0004:00000084       $pdata$4$RxInterruptHandler 000000014002e084     rxdevice.obj
 0004:00000090       $pdata$6$RxInterruptHandler 000000014002e090     rxdevice.obj
 0004:0000009c       $pdata$8$RxInterruptHandler 000000014002e09c     rxdevice.obj
 0004:000000a8       $pdata$9$RxInterruptHandler 000000014002e0a8     rxdevice.obj
 0004:000000b4       $pdata$NonMSIXInterruptHandler 000000014002e0b4     rxdevice.obj
 0004:000000c0       $pdata$3$NonMSIXInterruptHandler 000000014002e0c0     rxdevice.obj
 0004:000000cc       $pdata$4$NonMSIXInterruptHandler 000000014002e0cc     rxdevice.obj
 0004:000000d8       $pdata$PMCDpcResponseHandler 000000014002e0d8     rxdevice.obj
 0004:000000e4       $pdata$5$PMCDpcResponseHandler 000000014002e0e4     rxdevice.obj
 0004:000000f0       $pdata$6$PMCDpcResponseHandler 000000014002e0f0     rxdevice.obj
 0004:000000fc       $pdata$8$PMCDpcResponseHandler 000000014002e0fc     rxdevice.obj
 0004:00000108       $pdata$9$PMCDpcResponseHandler 000000014002e108     rxdevice.obj
 0004:00000114       $pdata$PMCInterruptHandler 000000014002e114     rxdevice.obj
 0004:00000120       $pdata$2$PMCInterruptHandler 000000014002e120     rxdevice.obj
 0004:0000012c       $pdata$3$PMCInterruptHandler 000000014002e12c     rxdevice.obj
 0004:00000138       $pdata$RxPullMessageUnitQueueCompletedFib 000000014002e138     rxdevice.obj
 0004:00000144       $pdata$1$RxPullMessageUnitQueueCompletedFib 000000014002e144     rxdevice.obj
 0004:00000150       $pdata$2$RxPullMessageUnitQueueCompletedFib 000000014002e150     rxdevice.obj
 0004:0000015c       $pdata$RxPushMessageUnitQueueFib 000000014002e15c     rxdevice.obj
 0004:00000168       $pdata$0$RxPushMessageUnitQueueFib 000000014002e168     rxdevice.obj
 0004:00000174       $pdata$1$RxPushMessageUnitQueueFib 000000014002e174     rxdevice.obj
 0004:00000180       $pdata$PMCPushMessageUnitQueueFib 000000014002e180     rxdevice.obj
 0004:0000018c       $pdata$0$PMCPushMessageUnitQueueFib 000000014002e18c     rxdevice.obj
 0004:00000198       $pdata$1$PMCPushMessageUnitQueueFib 000000014002e198     rxdevice.obj
 0004:000001a4       $pdata$2$PMCPushMessageUnitQueueFib 000000014002e1a4     rxdevice.obj
 0004:000001b0       $pdata$RxSendSynchCommand  000000014002e1b0     rxdevice.obj
 0004:000001bc       $pdata$RxStartAdapter      000000014002e1bc     rxdevice.obj
 0004:000001c8       $pdata$RxWaitForAdapterToBoot 000000014002e1c8     rxdevice.obj
 0004:000001d4       $pdata$0$RxWaitForAdapterToBoot 000000014002e1d4     rxdevice.obj
 0004:000001e0       $pdata$1$RxWaitForAdapterToBoot 000000014002e1e0     rxdevice.obj
 0004:000001ec       $pdata$DumpHandles         000000014002e1ec     rxdevice.obj
 0004:000001f8       $pdata$DumpHandlesZeroPointer 000000014002e1f8     rxdevice.obj
 0004:00000204       $pdata$RevCheckCompatibility 000000014002e204     revision.obj
 0004:00000210       $pdata$GetDriverParameter  000000014002e210     helpers.obj
 0004:0000021c       $pdata$MatchRegistryString 000000014002e21c     helpers.obj
 0004:00000228       $pdata$LongToAscii         000000014002e228     helpers.obj
 0004:00000234       $pdata$CompareStrings      000000014002e234     helpers.obj
 0004:00000240       $pdata$ArcPrintf           000000014002e240     arcdebug.obj
 0004:0000024c       $pdata$3$ArcPrintf         000000014002e24c     arcdebug.obj
 0004:00000258       $pdata$4$ArcPrintf         000000014002e258     arcdebug.obj
 0004:00000264       $pdata$RealSprintf         000000014002e264     arcdebug.obj
 0004:00000270       $pdata$1$RealSprintf       000000014002e270     arcdebug.obj
 0004:0000027c       $pdata$6$RealSprintf       000000014002e27c     arcdebug.obj
 0004:00000288       $pdata$7$RealSprintf       000000014002e288     arcdebug.obj
 0004:00000294       $pdata$8$RealSprintf       000000014002e294     arcdebug.obj
 0004:000002a0       $pdata$MainTimeThread      000000014002e2a0     timer.obj
 0004:000002ac       $pdata$4$MainTimeThread    000000014002e2ac     timer.obj
 0004:000002b8       $pdata$5$MainTimeThread    000000014002e2b8     timer.obj
 0004:000002c4       $pdata$6$MainTimeThread    000000014002e2c4     timer.obj
 0004:000002d0       $pdata$7$MainTimeThread    000000014002e2d0     timer.obj
 0004:000002dc       $pdata$VMCloseAllCompletionTimer 000000014002e2dc     timer.obj
 0004:000002e8       $pdata$0$VMCloseAllCompletionTimer 000000014002e2e8     timer.obj
 0004:000002f4       $pdata$1$VMCloseAllCompletionTimer 000000014002e2f4     timer.obj
 0004:00000300       $pdata$UpdateThorHBAMappingTable 000000014002e300     timer.obj
 0004:0000030c       $pdata$0$UpdateThorHBAMappingTable 000000014002e30c     timer.obj
 0004:00000318       $pdata$2$UpdateThorHBAMappingTable 000000014002e318     timer.obj
 0004:00000324       $pdata$3$UpdateThorHBAMappingTable 000000014002e324     timer.obj
 0004:00000330       $pdata$4$UpdateThorHBAMappingTable 000000014002e330     timer.obj
 0004:0000033c       $pdata$Reset_IOP_CompletionTimer 000000014002e33c     timer.obj
 0004:00000348       $pdata$0$Reset_IOP_CompletionTimer 000000014002e348     timer.obj
 0004:00000354       $pdata$2$Reset_IOP_CompletionTimer 000000014002e354     timer.obj
 0004:00000360       $pdata$4$Reset_IOP_CompletionTimer 000000014002e360     timer.obj
 0004:0000036c       $pdata$5$Reset_IOP_CompletionTimer 000000014002e36c     timer.obj
 0004:00000378       $pdata$StopTimer           000000014002e378     timer.obj
 0004:00000384       $pdata$RequestTimer        000000014002e384     timer.obj
 0004:00000390       $pdata$CheckingFWAfterPowerStateChange 000000014002e390     timer.obj
 0004:0000039c       $pdata$0$CheckingFWAfterPowerStateChange 000000014002e39c     timer.obj
 0004:000003a8       $pdata$3$CheckingFWAfterPowerStateChange 000000014002e3a8     timer.obj
 0004:000003b4       $pdata$4$CheckingFWAfterPowerStateChange 000000014002e3b4     timer.obj
 0004:000003c0       $pdata$StorWmiTraceMessage 000000014002e3c0     arcinit.obj
 0004:000003cc       $pdata$DriverEntry         000000014002e3cc     arcinit.obj
 0004:000003d8       $pdata$0$DriverEntry       000000014002e3d8     arcinit.obj
 0004:000003e4       $pdata$1$DriverEntry       000000014002e3e4     arcinit.obj
 0004:000003f0       $pdata$2$DriverEntry       000000014002e3f0     arcinit.obj
 0004:000003fc       $pdata$3$DriverEntry       000000014002e3fc     arcinit.obj
 0004:00000408       $pdata$HwInitializeAdapter 000000014002e408     arcinit.obj
 0004:00000414       $pdata$FindAdapter         000000014002e414     arcinit.obj
 0004:00000420       $pdata$1$FindAdapter       000000014002e420     arcinit.obj
 0004:0000042c       $pdata$2$FindAdapter       000000014002e42c     arcinit.obj
 0004:00000438       $pdata$ResetAdapter        000000014002e438     arcinit.obj
 0004:00000444       $pdata$5$ResetAdapter      000000014002e444     arcinit.obj
 0004:00000450       $pdata$6$ResetAdapter      000000014002e450     arcinit.obj
 0004:0000045c       $pdata$SMNormalModeInitAdapter 000000014002e45c     arcinit.obj
 0004:00000468       $pdata$1$SMNormalModeInitAdapter 000000014002e468     arcinit.obj
 0004:00000474       $pdata$2$SMNormalModeInitAdapter 000000014002e474     arcinit.obj
 0004:00000480       $pdata$InitializeDPCs      000000014002e480     arcinit.obj
 0004:0000048c       $pdata$1$InitializeDPCs    000000014002e48c     arcinit.obj
 0004:00000498       $pdata$2$InitializeDPCs    000000014002e498     arcinit.obj
 0004:000004a4       $pdata$ReturningLocalOutstandingRequestsToOS 000000014002e4a4     arcinit.obj
 0004:000004b0       $pdata$CleanHostSideRRQ    000000014002e4b0     arcinit.obj
 0004:000004bc       $pdata$EventTracingCleanup 000000014002e4bc     arcinit.obj
 0004:000004c8       $pdata$AllocateConsumerProducerCommArea 000000014002e4c8     arcinit.obj
 0004:000004d4       $pdata$AllocateMessageUnitQueueCommArea 000000014002e4d4     arcinit.obj
 0004:000004e0       $pdata$ConfigureContainersRuntime 000000014002e4e0     arcinit.obj
 0004:000004ec       $pdata$0$ConfigureContainersRuntime 000000014002e4ec     arcinit.obj
 0004:000004f8       $pdata$1$ConfigureContainersRuntime 000000014002e4f8     arcinit.obj
 0004:00000504       $pdata$SendEvent2OSDelayed 000000014002e504     arcinit.obj
 0004:00000510       $pdata$GetElapsedSeconds   000000014002e510     arcinit.obj
 0004:0000051c       $pdata$IsAdapterReadyForConfigCommand 000000014002e51c     arcinit.obj
 0004:00000528       $pdata$CheckMSIxPossibility 000000014002e528     arcinit.obj
 0004:00000534       $pdata$0$CheckMSIxPossibility 000000014002e534     arcinit.obj
 0004:00000540       $pdata$1$CheckMSIxPossibility 000000014002e540     arcinit.obj
 0004:0000054c       $pdata$2$CheckMSIxPossibility 000000014002e54c     arcinit.obj
 0004:00000558       $pdata$3$CheckMSIxPossibility 000000014002e558     arcinit.obj
 0004:00000564       $pdata$HandleAdapterConfigIssues 000000014002e564     arcinit.obj
 0004:00000570       $pdata$SendInitStructure   000000014002e570     arcinit.obj
 0004:0000057c       $pdata$HandleAdapterGetConfig 000000014002e57c     arcinit.obj
 0004:00000588       $pdata$HandleAdapterCommitConfig 000000014002e588     arcinit.obj
 0004:00000594       $pdata$InitializeConsumerProducerCommRegion 000000014002e594     arcinit.obj
 0004:000005a0       $pdata$MapDeviceBase       000000014002e5a0     arcinit.obj
 0004:000005ac       $pdata$IOPReset            000000014002e5ac     arcinit.obj
 0004:000005b8       $pdata$HWSoftReset         000000014002e5b8     arcinit.obj
 0004:000005c4       $pdata$DumpFibsSentToFW60SecondsBefore 000000014002e5c4     arcinit.obj
 0004:000005d0       $pdata$4$DumpFibsSentToFW60SecondsBefore 000000014002e5d0     arcinit.obj
 0004:000005dc       $pdata$5$DumpFibsSentToFW60SecondsBefore 000000014002e5dc     arcinit.obj
 0004:000005e8       $pdata$ReturningOutstandingSentToFWBeforeIOPResetToOS 000000014002e5e8     arcinit.obj
 0004:000005f4       $pdata$3$ReturningOutstandingSentToFWBeforeIOPResetToOS 000000014002e5f4     arcinit.obj
 0004:00000600       $pdata$4$ReturningOutstandingSentToFWBeforeIOPResetToOS 000000014002e600     arcinit.obj
 0004:0000060c       $pdata$5$ReturningOutstandingSentToFWBeforeIOPResetToOS 000000014002e60c     arcinit.obj
 0004:00000618       $pdata$6$ReturningOutstandingSentToFWBeforeIOPResetToOS 000000014002e618     arcinit.obj
 0004:00000624       $pdata$ReturnOutstandingFibOnTargetDevice 000000014002e624     arcinit.obj
 0004:00000630       $pdata$2$ReturnOutstandingFibOnTargetDevice 000000014002e630     arcinit.obj
 0004:0000063c       $pdata$3$ReturnOutstandingFibOnTargetDevice 000000014002e63c     arcinit.obj
 0004:00000648       $pdata$4$ReturnOutstandingFibOnTargetDevice 000000014002e648     arcinit.obj
 0004:00000654       $pdata$5$ReturnOutstandingFibOnTargetDevice 000000014002e654     arcinit.obj
 0004:00000660       $pdata$SetFwTime           000000014002e660     arcinit.obj
 0004:0000066c       $pdata$0$SetFwTime         000000014002e66c     arcinit.obj
 0004:00000678       $pdata$4$SetFwTime         000000014002e678     arcinit.obj
 0004:00000684       $pdata$5$SetFwTime         000000014002e684     arcinit.obj
 0004:00000690       $pdata$6$SetFwTime         000000014002e690     arcinit.obj
 0004:0000069c       $pdata$7$SetFwTime         000000014002e69c     arcinit.obj
 0004:000006a8       $pdata$SetArcsasFwTime     000000014002e6a8     arcinit.obj
 0004:000006b4       $pdata$SetPciSlotNumber    000000014002e6b4     arcinit.obj
 0004:000006c0       $pdata$SendWellnessCmnd    000000014002e6c0     arcinit.obj
 0004:000006cc       $pdata$GetThorHbaPhyDevInfo 000000014002e6cc     arcinit.obj
 0004:000006d8       $pdata$ArcLogEventString   000000014002e6d8     arcinit.obj
 0004:000006e4       $pdata$LogSystemEvent      000000014002e6e4     arcinit.obj
 0004:000006f0       $pdata$SendEvent2OS        000000014002e6f0     arcinit.obj
 0004:000006fc       $pdata$WppTraceCallback    000000014002e6fc     arcinit.obj
 0004:00000708       $pdata$2$WppTraceCallback  000000014002e708     arcinit.obj
 0004:00000714       $pdata$3$WppTraceCallback  000000014002e714     arcinit.obj
 0004:00000720       $pdata$DynamicallyThrottleLunQueueDepth 000000014002e720     arcinit.obj
 0004:0000072c       $pdata$SA4StatusBatching   000000014002e72c     arcinit.obj
 0004:00000738       $pdata$SA4ACI2Interface    000000014002e738     arcinit.obj
 0004:00000744       $pdata$SMCrashDumpModeInitAdapter 000000014002e744     arcinit.obj
 0004:00000750       $pdata$SendEvent2OSChild   000000014002e750     arcinit.obj
 0004:0000075c       $pdata$StartIo             000000014002e75c     cmddelivery.obj
 0004:00000768       $pdata$0$StartIo           000000014002e768     cmddelivery.obj
 0004:00000774       $pdata$1$StartIo           000000014002e774     cmddelivery.obj
 0004:00000780       $pdata$PostProcessScsiCommand 000000014002e780     cmddelivery.obj
 0004:0000078c       $pdata$SendFib             000000014002e78c     cmddelivery.obj
 0004:00000798       $pdata$HandleMSIXInterrupt 000000014002e798     cmddelivery.obj
 0004:000007a4       $pdata$QueueRawIoReadWriteRequest 000000014002e7a4     cmddelivery.obj
 0004:000007b0       $pdata$1$QueueRawIoReadWriteRequest 000000014002e7b0     cmddelivery.obj
 0004:000007bc       $pdata$3$QueueRawIoReadWriteRequest 000000014002e7bc     cmddelivery.obj
 0004:000007c8       $pdata$4$QueueRawIoReadWriteRequest 000000014002e7c8     cmddelivery.obj
 0004:000007d4       $pdata$5$QueueRawIoReadWriteRequest 000000014002e7d4     cmddelivery.obj
 0004:000007e0       $pdata$6$QueueRawIoReadWriteRequest 000000014002e7e0     cmddelivery.obj
 0004:000007ec       $pdata$CompleteQueuedRequest 000000014002e7ec     cmddelivery.obj
 0004:000007f8       $pdata$DequeueRawIoReadWriteRequest 000000014002e7f8     cmddelivery.obj
 0004:00000804       $pdata$0$DequeueRawIoReadWriteRequest 000000014002e804     cmddelivery.obj
 0004:00000810       $pdata$1$DequeueRawIoReadWriteRequest 000000014002e810     cmddelivery.obj
 0004:0000081c       $pdata$ProcessContainerInquiry 000000014002e81c     cmddelivery.obj
 0004:00000828       $pdata$ProcessScsiCommand  000000014002e828     cmddelivery.obj
 0004:00000834       $pdata$QueuePrintf         000000014002e834     cmddelivery.obj
 0004:00000840       $pdata$SendRawIoFib        000000014002e840     cmddelivery.obj
 0004:0000084c       $pdata$SendSynchFib        000000014002e84c     cmddelivery.obj
 0004:00000858       $pdata$0$SendSynchFib      000000014002e858     cmddelivery.obj
 0004:00000864       $pdata$1$SendSynchFib      000000014002e864     cmddelivery.obj
 0004:00000870       $pdata$DequeueCertainLD    000000014002e870     cmddelivery.obj
 0004:0000087c       $pdata$0$DequeueCertainLD  000000014002e87c     cmddelivery.obj
 0004:00000888       $pdata$1$DequeueCertainLD  000000014002e888     cmddelivery.obj
 0004:00000894       $pdata$PollSmartHBAFIBCompletion 000000014002e894     cmddelivery.obj
 0004:000008a0       $pdata$AdapterControl      000000014002e8a0     cmdproc.obj
 0004:000008ac       $pdata$BuildIo             000000014002e8ac     cmdproc.obj
 0004:000008b8       $pdata$BuildHBAFib         000000014002e8b8     cmdproc.obj
 0004:000008c4       $pdata$BuildRawIoFib       000000014002e8c4     cmdproc.obj
 0004:000008d0       $pdata$BuildRawIoScatterGather 000000014002e8d0     cmdproc.obj
 0004:000008dc       $pdata$0$BuildRawIoScatterGather 000000014002e8dc     cmdproc.obj
 0004:000008e8       $pdata$1$BuildRawIoScatterGather 000000014002e8e8     cmdproc.obj
 0004:000008f4       $pdata$2$BuildRawIoScatterGather 000000014002e8f4     cmdproc.obj
 0004:00000900       $pdata$3$BuildRawIoScatterGather 000000014002e900     cmdproc.obj
 0004:0000090c       $pdata$BuildRawIo2ScatterGather 000000014002e90c     cmdproc.obj
 0004:00000918       $pdata$ConvertRawIo2ScatterGather 000000014002e918     cmdproc.obj
 0004:00000924       $pdata$1$ConvertRawIo2ScatterGather 000000014002e924     cmdproc.obj
 0004:00000930       $pdata$3$ConvertRawIo2ScatterGather 000000014002e930     cmdproc.obj
 0004:0000093c       $pdata$4$ConvertRawIo2ScatterGather 000000014002e93c     cmdproc.obj
 0004:00000948       $pdata$5$ConvertRawIo2ScatterGather 000000014002e948     cmdproc.obj
 0004:00000954       $pdata$BuildReadWriteFib   000000014002e954     cmdproc.obj
 0004:00000960       $pdata$BuildScatterGather  000000014002e960     cmdproc.obj
 0004:0000096c       $pdata$BuildScatterGather64 000000014002e96c     cmdproc.obj
 0004:00000978       $pdata$BuildRawIo2ScatterGather4HBAIoctl 000000014002e978     cmdproc.obj
 0004:00000984       $pdata$BuildHBAIoctlFib    000000014002e984     cmdproc.obj
 0004:00000990       $pdata$BuildSrbFib         000000014002e990     cmdproc.obj
 0004:0000099c       $pdata$InitializeFib       000000014002e99c     cmdproc.obj
 0004:000009a8       $pdata$PrepareBMIC15       000000014002e9a8     cmdproc.obj
 0004:000009b4       $pdata$ProcessIoctl        000000014002e9b4     ioctl.obj
 0004:000009c0       $pdata$BuildRawScatterGather 000000014002e9c0     ioctl.obj
 0004:000009cc       $pdata$1$BuildRawScatterGather 000000014002e9cc     ioctl.obj
 0004:000009d8       $pdata$2$BuildRawScatterGather 000000014002e9d8     ioctl.obj
 0004:000009e4       $pdata$BuildRawScatterGather64 000000014002e9e4     ioctl.obj
 0004:000009f0       $pdata$CSMIGetRAIDConfig   000000014002e9f0     ioctl.obj
 0004:000009fc       $pdata$0$CSMIGetRAIDConfig 000000014002e9fc     ioctl.obj
 0004:00000a08       $pdata$1$CSMIGetRAIDConfig 000000014002ea08     ioctl.obj
 0004:00000a14       $pdata$CSMIGetRAIDInfo     000000014002ea14     ioctl.obj
 0004:00000a20       $pdata$CSMISTPPassThru     000000014002ea20     ioctl.obj
 0004:00000a2c       $pdata$0$CSMISTPPassThru   000000014002ea2c     ioctl.obj
 0004:00000a38       $pdata$1$CSMISTPPassThru   000000014002ea38     ioctl.obj
 0004:00000a44       $pdata$HandleCSMI          000000014002ea44     ioctl.obj
 0004:00000a50       $pdata$QueueEvent          000000014002ea50     comm.obj
 0004:00000a5c       $pdata$AdapterIsAlive      000000014002ea5c     comm.obj
 0004:00000a68       $pdata$ServiceHostResponseNormalQueue 000000014002ea68     comm.obj
 0004:00000a74       $pdata$6$ServiceHostResponseNormalQueue 000000014002ea74     comm.obj
 0004:00000a80       $pdata$7$ServiceHostResponseNormalQueue 000000014002ea80     comm.obj
 0004:00000a8c       $pdata$FreeConsumerProducerAif 000000014002ea8c     comm.obj
 0004:00000a98       $pdata$0$FreeConsumerProducerAif 000000014002ea98     comm.obj
 0004:00000aa4       $pdata$1$FreeConsumerProducerAif 000000014002eaa4     comm.obj
 0004:00000ab0       $pdata$ProcessAif          000000014002eab0     comm.obj
 0004:00000abc       $pdata$SendConsumerProducerFib 000000014002eabc     comm.obj
 0004:00000ac8       $pdata$SubDeQueueSortingQueue 000000014002eac8     comm.obj
 0004:00000ad4       $pdata$0$SubDeQueueSortingQueue 000000014002ead4     comm.obj
 0004:00000ae0       $pdata$1$SubDeQueueSortingQueue 000000014002eae0     comm.obj
 0004:00000aec       $pdata$DeQueueSortingQueue 000000014002eaec     comm.obj
 0004:00000af8       $pdata$CompleteAllSortingQueue 000000014002eaf8     comm.obj
 0004:00000b04       $pdata$5$CompleteAllSortingQueue 000000014002eb04     comm.obj
 0004:00000b10       $pdata$6$CompleteAllSortingQueue 000000014002eb10     comm.obj
 0004:00000b1c       $pdata$CompleteBufferedRequest 000000014002eb1c     comm.obj
 0004:00000b28       $pdata$0$CompleteBufferedRequest 000000014002eb28     comm.obj
 0004:00000b34       $pdata$1$CompleteBufferedRequest 000000014002eb34     comm.obj
 0004:00000b40       $pdata$ServiceHostCommandNormalQueue 000000014002eb40     comm.obj
 0004:00000b4c       $pdata$3$ServiceHostCommandNormalQueue 000000014002eb4c     comm.obj
 0004:00000b58       $pdata$4$ServiceHostCommandNormalQueue 000000014002eb58     comm.obj
 0004:00000b64       $pdata$DpcDequeueRawIoReadWriteRequest 000000014002eb64     comm.obj
 0004:00000b70       $pdata$ProcessNormalFib    000000014002eb70     comm.obj
 0004:00000b7c       $pdata$3$ProcessNormalFib  000000014002eb7c     comm.obj
 0004:00000b88       $pdata$5$ProcessNormalFib  000000014002eb88     comm.obj
 0004:00000b94       $pdata$6$ProcessNormalFib  000000014002eb94     comm.obj
 0004:00000ba0       $pdata$7$ProcessNormalFib  000000014002eba0     comm.obj
 0004:00000bac       $pdata$8$ProcessNormalFib  000000014002ebac     comm.obj
 0004:00000bb8       $pdata$ServiceInternalAifQueue 000000014002ebb8     comm.obj
 0004:00000bc4       $pdata$ProcessHbaErrors    000000014002ebc4     comm.obj
 0004:00000bd0       $pdata$3$ProcessHbaErrors  000000014002ebd0     comm.obj
 0004:00000bdc       $pdata$4$ProcessHbaErrors  000000014002ebdc     comm.obj
 0004:00000be8       $pdata$ProcessWmi          000000014002ebe8     wmi.obj
 0004:00000bf4       $pdata$HwScsiWmiExecuteMethod 000000014002ebf4     wmi.obj
 0004:00000c00       $pdata$HwScsiWmiQueryDataBlock 000000014002ec00     wmi.obj
 0004:00000c00       $pdata$HwScsiWmiFunctionControl 000000014002ec00     wmi.obj
 0004:00000c0c       $pdata$GsDriverEntry       000000014002ec0c     BufferOverflowFastFailK:gs_driverentry.obj
 0004:00000c30       $pdata$__GSHandlerCheckCommon 000000014002ec30     ntoskrnl:gshandler.obj
 0004:00000c3c       $pdata$__GSHandlerCheck    000000014002ec3c     ntoskrnl:gshandler.obj
 0004:00000c60       $pdata$ScsiPortWmiDispatchFunction 000000014002ec60     scsiwmi:wmilib.obj
 0004:00000c6c       $pdata$ScsiWmipProcessRequest 000000014002ec6c     scsiwmi:wmilib.obj
 0004:00000c78       $pdata$ScsiPortWmiPostProcess 000000014002ec78     scsiwmi:wmilib.obj
 0004:00000c84       $pdata$ScsiWmipPostProcess 000000014002ec84     scsiwmi:wmilib.obj
 0004:00000c90       $pdata$ScsiWmipFindGuid    000000014002ec90     scsiwmi:wmilib.obj
 0005:000001a0       .idata$6                   000000014002f1a0     ntoskrnl:ntoskrnl.exe
 0005:000001ca       .idata$6                   000000014002f1ca     hal:HAL.dll
 0005:0000038a       .idata$6                   000000014002f38a     storport:storport.sys
 0006:000000d0       $R000000                   00000001400300d0     archba.res
 0006:00000420       $R000350                   0000000140030420     archba.res
